:020000040800F2
:1000000000200010ED08030825B60108E5EB000804
:1000100021B601081DB6010819B60108000000004C
:1000200000000000000000000000000015B60108FC
:1000300011B60108000000000DB60108D147010803
:10004000550903085509030855090308550903080C
:10005000550903085509030839DF000865E0000861
:1000600029E00008EDDF0008B1DF00080DFA020802
:100070001DFA020881F9020871F9020861F9020803
:1000800039F902084DF90208550903085509030812
:10009000B1B90108550903085509030875DF0008BF
:1000A00025F9000875F90008550903089DF90008AD
:1000B00065F9000855F900085509030855090308B2
:1000C000550903085509030855090308550903088C
:1000D00055090308B9FA0208ADFA0208DDFA020868
:1000E000FDDE000855090308FDB5010855090308A0
:1000F00035F900085509030845F9000855090308B2
:100100000000000000000000000000005509030886
:10011000C5FA0208D1FA020855090308550903086F
:10012000F9F9020891F90208A5F90208B9F90208DB
:10013000D9F902085509030800000000000000007A
:100140005509030855090308550903080000000074
:10015000000000000000000000000000000000009F
:1001600000000000000000005509030855090308BD
:100170005509030800000000000000000000000016
:0801800000000000550903080E
:100190002DE9F04FA64C23681A688DB00646D26947
:1001A00018469047C8B96768A24BA3FB07239B0872
:1001B00003EB8303791CFF1A616011D02068036888
:1001C000DB689847236843B193F90830002B04DDBE
:1001D000994D2B7823F001032B700DB0BDE8F08F03
:1001E000954D237A2A7802F00402934200F0D581DB
:1001F000002A76D0D4F80080D8F8003040469B68BA
:100200009847FF23206888F8073002688B4BD2F8A4
:100210001490012288F806200C210722C847DFF835
:1002200058C2278206214FF4FA724FF06309BE4686
:10023000A781A782BA463846ACF80010E281A4F83C
:1002400012902B7803F0040323720028BCBF002017
:10025000A0817B48DFF824820088DFF818B2904242
:10026000D8F80020B8BFE0818BFB027BD217C2EB2D
:100270006B1212B25245C8BF2282A27D4A45B8BF56
:100280006282704A92697245C8BFA2828BB1DFF860
:10029000F0E194F81790AEFB067ECEF3874EF14561
:1002A00007D0B4F8189084F817E009F1010EA4F80B
:1002B00018E0002900F0E880634AB2F9060040F235
:1002C000D663984200F3A780B2F902209A4200F365
:1002D000A280013989B2ACF8001000297FF472AF16
:1002E0009CE027683B6838469B689847FF23206856
:1002F000FB710268554BD2F8148001210222B971BA
:100300001146C047524B1B789A0700F1AA81072378
:100310000293062303934FF005084FF004094FF0B2
:10032000030A04AF20684B4B02680221D2F814B0D4
:100330005246D847B4F90E304748484980FB03205D
:10034000DA17C2EBA00202EB8200A3EB40031BB260
:1003500012B238462DF0D0FE2068036852461621AE
:10036000D3F814A03B46D04720683D4B02680221D9
:10037000D2F814A04A46D0473946B4F912001DF00D
:100380007FFD38462FF0CCFB364A236812883A525C
:1003900019684A461846D1F814903B461621C847BA
:1003A000314B1B681B0500F17D8120682F4B0268D3
:1003B0000221D2F814904246C8472D4BB4F91400DC
:1003C00093F87A34002B40F0F78000EB800300EBC9
:1003D000C300284AC00082FB0031C317D3EB611170
:1003E00000F1238182FB012ECA17C2EB6E124FF07F
:1003F0006409DFF864E0DFF88CC009FB12128EFBA1
:1004000002E1D2178CFB00E0C2EBA101C3EB203369
:1004100020220F20EBE00023ACF8003025682B6889
:1004200028469B6898470122FF23AA71EB71C9E611
:1004300070180020CDCCCCCC744F0020D4790308A8
:10044000941A0020401A00206C1A0020DC7903085E
:100450002E1B0020007A030867666666147A03087C
:100460001C7A0308A4830308504F0020607A030815
:10047000744500201F85EB51C06300209C1A0020AA
:1004800083DE1B43AD8BDB68A649DFF8D492D4F83A
:1004900000B0B609A1FB0616C6F3801689F8006005
:1004A000BBF1000F04D09BF9081000293FF791AE73
:1004B0009D4D95F87A1449B94FF4A4719B4E01FBF8
:1004C00002F286FB0261D217C2EB6112DFF894A23E
:1004D000964EBAF800E0DFF890C286FB02766421FF
:1004E000D217934F01FB0EF1C2EB661295F872E43E
:1004F000904EC1F387218E45A175B7F800E03168B1
:100500008CBF41F0010121F0010170458A48B5F826
:1005100076E40078B5BF41F4001121F4001141F0F8
:10052000020121F002018707208BACFB007054BF51
:1005300041F4804121F48041BEEB501F00F2EF8076
:10054000002B00F0EC8041F040037C49B5F87404C6
:1005500009688842B5F87814D4BF43F4805323F473
:1005600080538A42DBF80020ACBF43F4004323F4FD
:1005700000433360584693689847714B1B680121CC
:10058000FF2258038BF806108BF8072040F1F28009
:10059000206803681B6A984714E6DFF8D0C1B4F9F5
:1005A0000C00BCF80010B4F90E20B4F910A0B4F996
:1005B0001290B4F914E048E65C4B624983FB0023D7
:1005C000C217C2EB6313642202FB130281FB021EFB
:1005D000D1170028C1EBAE01ACBF20222D2200298B
:1005E000B8BF4942002B4FF00C00B8BF5B420190EE
:1005F0000091384654492DF07FFD206801683B4644
:1006000042464F691621B847DFF860C1B4F90C00C3
:10061000B4F90E20B4F910A0B4F91290B4F914E0B2
:100620004FF43471ACF800100BE682FB012EDFF8BA
:1006300040C1CA17C2EB6E124FF0640E0EFB1212CD
:100640008CFB00E03F49C3EB203381FB02E1002B30
:100650004FEAE272A2EBA101B8BF5B420F202D224C
:10066000C5E72068394B02680221D2F8148004AF34
:100670000322C0473946B4F90C001DF001FC206884
:1006800003680322D3F8148016213B46C047082391
:100690000293072303934FF006084FF005094FF02C
:1006A000040A3FE620682A4B02680221D2F814901F
:1006B0004246C8473946B4F910001DF0E1FB384600
:1006C0002FF02EFA234A236812883A5219684246BC
:1006D0001846D1F814803B461621C0472068DDF843
:1006E0000C9002681C4BD2F8148002214A46C04785
:1006F000124B394618681DF0C3FB38462FF010FA2C
:10070000164A236812883A5219681846D1F814809C
:100710004A463B461621C047DDF8088045E621F0F1
:10072000400312E7632D3E05744500201F85EB5101
:10073000082D0020BC6300202E1B0020A01A0020E2
:10074000681A002067666666747A0308EC79030805
:10075000307A0308447A0308487A03085C7A03086D
:10076000000000202C1B002089888888C06300209E
:10077000AD8BDB68B74B1B68990705D423684BB179
:1007800093F90830002B05DD03202CF065FE0220D4
:100790002CF062FEB5F848B41BF4006F25D0336826
:1007A0009A0702D599F80030FBB9AB4BAB4A1B88CE
:1007B000AB49A2FB0302D20802EB8200A3EB400389
:1007C0000CA807469BB24FF0910E0DF1110007F8EF
:1007D00020ED2DF091FC2068026852693B460BF039
:1007E0001F011746CBF34412B847B5F846B41BF4C3
:1007F000006F23D03368DB0702D599F80030EBB9DE
:10080000BAF800309749642202FB03F292120DF10C
:10081000300A632A4FF00103A8BF63220DF11100D3
:100820000AF8203D2DF068FC2068026853460BF062
:100830001F01D2F814A0CBF34412D047B5F852A44C
:100840001AF4006F24D033685F0602D599F800309F
:10085000F3B9238B844A8549A2FB03025209C2EBF8
:1008600002100DF1300BA3EB80039BB24FF09C0EF6
:100870000DF111000BF820ED2DF03EFC2068026810
:100880005B460AF01F01D2F814B0CAF34412D847ED
:10089000B5F850B41BF4006F2FD03368980602D51A
:1008A00099F800304BBB13F0EDFE714B6E4ADFF848
:1008B000E4E16E49A3FB00739B0CA2FB03724FEAB9
:1008C000102C50090DF1300AAEFB0C72C0EB001079
:1008D000A3EB8003920A4FF09B0E0DF111000AF872
:1008E00020ED2DF009FC2068026853460BF01F0133
:1008F000D2F814A0CBF34412D047B5F854341905FC
:1009000020D53268120602D599F80020D2B9594A8A
:10091000106803F01F01C3F34412030140F18C81FE
:10092000554B56480088470500F18481C70700F100
:100930008D81DFF864E110F0020F18BF7346206864
:100940000DF0C6FBB5F858A41AF4006F30D0336828
:100950009F0502D599F8003053BB494B494AB3F97A
:1009600006304049B3F5FA6FA8BF4FF4FA63B3F508
:100970007A7FB8BF4FF47A73A3F57A7382FB0302D0
:10098000DB17C3EBA2024FF0040E05230DF112009A
:100990008DF811308DF810E02DF0AEFB2068036863
:1009A000CAF34412D3F814B00AF01F0104ABD847BD
:1009B000B5F85CA41AF4006F28D03368180502D586
:1009C00099F8003013BBD8F800302F482F49002B7E
:1009D000B8BF5B4280FB0320DA17C2EB60120DF157
:1009E000300B642000FB12334FF09A0E0DF1110012
:1009F0000BF820ED2DF080FB206802685B460AF0C2
:100A00001F01D2F814B0CAF34412D847B5F85EA457
:100A10001AF4006F42D03368D90403D599F8003036
:100A2000002B3BD11A4B0F491A680DF1300B0723ED
:100A30000DF111000BF8203D2DF05EFB20680268DF
:100A40005B460AF01F01D2F814B0CAF34412D8472B
:100A500024E000BF601B0020941A0020CDCCCCCC39
:100A6000147A0308BCA8030889888888807A030858
:100A700083DE1B43681A0020C0790308061B002090
:100A80006C1A0020676666661F85EB518C7A030836
:100A9000A01A0020C7541E01D079030808202CF0AA
:100AA000DBFC0F202CF0D8FCB5F866A41AF4006F1C
:100AB00019D03368DA0302D599F800309BB9644B3A
:100AC00064491868837A0278007D009004A82DF0AC
:100AD00013FB2068026804ABD2F814B00AF01F01BF
:100AE000CAF34412D847B5F868A41AF4006F19D0B5
:100AF00033689B0302D599F800309BB9544B564993
:100B00001868C37A4278407D009004A82DF0F4FA6A
:100B10002068026804ABD2F814B00AF01F01CAF3CF
:100B20004412D847B5F86AA41AF4006F19D0336894
:100B30005F0302D599F800309BB9454B47491868C7
:100B4000037B8278807D009004A82DF0D5FA206880
:100B5000026804ABD2F814B00AF01F01CAF34412C1
:100B6000D847B5F86CA41AF4006F1FD03368180387
:100B700002D599F80030CBB9394AD8F8003010883E
:100B8000384A394903FB00F382FB0302DB17C3EB4E
:100B9000A21204A82DF0B0FA2068026804ABD2F8C3
:100BA00014800AF01F01CAF34412C047B5F86E84DE
:100BB00018F4006F1CD03368D90202D599F80030C0
:100BC000B3B995F8E0252949742303FB025304A81F
:100BD00093F8D034013201332DF08EFA2068026888
:100BE00004ABD2F814A008F01F01C8F34412D04798
:100BF000B5F870542A057FF5CBAC33689B0204D559
:100C000099F80030002B7FF4C3AC194B1A88144BB1
:100C10001B889A427FF7BCAC04A816492DF06CFAE9
:100C20002068026804AB566905F01F01C5F3441241
:100C3000B047ADE4104B82E6104B1148D3F800E00A
:100C4000104B1EF4800F08BF03466AE60E4B76E693
:100C500048390020947A0308A47A0308B47A030878
:100C6000941A0020D34D6210C47A0308C87A03088E
:100C7000082D0020D07A0308C4790308504F0020C3
:100C8000B8790308C0790308C87903082DE9F04F43
:100C9000BA4C2DED028B94F85C318FB00546002BD9
:100CA00040F0808194F81832002B00F0CA80D4F80C
:100CB0001C32B34AEB1A934200F22A8494F856721B
:100CC000002F4CD0D4F86022002A00F0BA80D4F86B
:100CD000683240F6B731EB1A8B4240F2B28094F89A
:100CE0006432002B40F05684D4F86C22C4F8603291
:100CF000927884F85632022A01F26B82A14AD4F823
:100D000058125068814201F053841369994202F0ED
:100D1000CF84D369994202F0C884936A994202F061
:100D2000C184536B994202F0BA84136C994202F069
:100D3000B384D36C994202F0D584936D994201F04B
:100D40003684012391F90400009300224FF4964366
:100D500008212BF0ADFBC4F8580201F04ABAD4F8D0
:100D6000580203685B689847C0B2012840F2B98016
:100D7000022840F0AC80844E3378002B42F06D8224
:100D8000D4F85C32EB1AB3F57A6FC0F0AA80D4F8CD
:100D9000580203680122DB68327098470646D4F88F
:100DA00058020368DB689847760640F09A808E28E0
:100DB00040F0978094F85632002B83D1734BC4F8DF
:100DC00060322D2384F86432D4F86C329A7801238F
:100DD000022A84F8563200F21C856A4AD4F8581266
:100DE0005068814202F075831069814201F0A5804C
:100DF000D369994202F06A83936A994202F063834D
:100E0000536B994202F07283136C994202F06B8328
:100E1000D36C994202F06483936D994201F08C8007
:100E2000022391F90400009300224FF49643082115
:100E30002BF03EFBC4F85802002384F87032C4F84B
:100E4000685209F0A9F994F872325BB1504E3068DB
:100E500040B1D4F86081D4F87432A8EB0303632B5B
:100E600000F2BF8194F8A332022B00F04782464E75
:100E700096F87430032B00F0A58494F8BE326BB161
:100E8000D4F8C03253B113F0FDFBD4F8C43244F6A9
:100E90001F62C31A9342824600F2508294F82034B3
:100EA000002B40F0778194F85E3433B1D4F860348D
:100EB00003F5C333A0339D421DD20FB0BDEC028BAE
:100EC000BDE8F08FD4F858020368DB689847D4F87F
:100ED000580203685B6898470028F3D12A4E012323
:100EE0003370D4F86022002AABD094F85632002B2D
:100EF0003FF46AAFEBE694F86434264AC4F86054D1
:100F000002EB8302526A4AB3234E0EADF31C45F83E
:100F1000203D06F1150100230791A4F866348021D5
:100F20001523A52784F86A34284684F8691484F8C0
:100F3000687490472846B4F866142CF0C7FF069DE5
:100F4000AD1B152DA8BF15252A46314606F1180000
:100F500031F07AF894F8643484F895540F4A0133E8
:100F600082FB0312A2EBE37202EB42029B1A84F8AB
:100F700064340FB0BDEC028BBDE8F08F8C180020FC
:100F80003F0D03002088002004000020AC1A002040
:100F900030910020B84E0308F41C002056555555DA
:100FA00000007A44D4F86021D4F86431D31A7C2B41
:100FB0007FF678AE94F868311FED078AC4F8642193
:100FC00001330F4684F8683104F5CE784FF02409D8
:100FD000D4F8AC0103685E211B689847D4F8AC01D3
:100FE000036849461B689847B4F87431F8EC016A05
:100FF00007EE103AF8EEE66AB8EEC77A09F1010991
:10100000C6EE877A5FFA89F967EE887AFDEEE77AAD
:10101000CDED027ABDF90860F0B209F0FDFCC6F32F
:10102000072009F0F9FCB9F1270FD1D1D4F8AC01B0
:1010300003685E211B689847D4F8AC01036830212F
:101040001B689847D4F8B061F0B209F0E5FCC6F32C
:10105000072009F0E1FCD4F8AC0103685E211B68AD
:10106000984794F8683113F0030642D1D4F864210C
:1010700041F288339A4202F20B81D4F8AC01036842
:101080005E211B689847D4F8AC01036814211B68E3
:101090009847A44AB4F9D831DE1782FB0323C6EB84
:1010A000A30636B2F0B209F0B7FCC6F3072009F088
:1010B000B3FCD4F8AC0103685E211B689847D4F8F0
:1010C000AC0103681C211B689847D4F8AC01036885
:1010D00000211B689847D4F8AC01036800211B6805
:1010E0009847D4F8AC0103685E211B68984794F8D0
:1010F00068315E0701F06682282B7FF4D3ADD4F807
:10110000AC01D4F860610368874F1B684FF000089A
:101110005E2184F868819847D4F8AC0103681721F0
:101120001B689847D4F8AC01036841461B68984790
:101130007E4BA3FB06239B0BA7FB03125209C2EBBA
:101140000212A3EB8203D8B209F066FCD4F8AC011A
:1011500003685E211B689847D4F8AC010368182126
:101160001B689847724BA3FB06239B09A7FB03123E
:101170005209C2EB0212A3EB8203D8B209F04CFC75
:10118000404609F049FCD4F8AC0103685E211B68B5
:10119000984787E594F82124002A40F02983D4F861
:1011A000283403F5C333A0339D42FFF47CAE94F89A
:1011B0002C64C4F82854A31993F83074FA0701F189
:1011C000F985BB0701F1FC827F0700F1EC8694F8FA
:1011D0005D24013696FBF2F302FB136684F82C645F
:1011E00061E6544FDFF83C9100233B7003682421F3
:1011F0001B6898473068036854211B68984730681B
:10120000036841211B689847B4F9D631306889FBDF
:101210000312DB17C3EBA2030FFA83FA03685FFA2A
:101220008AFB59461B689847397830688BEA010178
:1012300039700368CAF3072A51461B6898473A7801
:10124000B4F9D431306889FB03E18AEA0202DB1782
:101250003A70C3EBA10302680FFA83FA5FFA8AFBC4
:10126000136859469847397830688BEA010139701C
:101270000368CAF3072A51461B6898473A78B4F9BD
:10128000D83130688AEA020289FB0319DB173A7009
:10129000C3EBA90301680FFA83F95FFA89FA0B68B7
:1012A000514698473A7830688AEA02023A700368F1
:1012B000C9F307291B68494698473978306889EA95
:1012C0000101397003681B68984794F8783213F06D
:1012D000010200F05987184AC4F874820133DBB266
:1012E000A2FB0312D20802EB8202A3EB420384F8B2
:1012F000783294F8A332022B7FF4B9AD13F0C2F91F
:10130000D4F8A42240F6B833801A984200F25787E6
:1013100094F8B0323A2B00F06381002384F8A332B2
:10132000ABE500BF676666668988888873B2E74563
:10133000D34D621034910020CDCCCCCC94F8CA327D
:10134000002B40F06E82D4F8D43203F00802002A59
:1013500048F603414AF60B404BF60F4249F6074662
:1013600004BF02460E4613F0040F4FF0190118BFD8
:1013700016469B0684F8CA1203D546F4804646F00A
:101380002006924B1F6817F00207C6F3090841F0C8
:10139000FF804FF0FF3964204FF0000E069607964D
:1013A000ADF82670CDF82080ADF828908DF8360085
:1013B000ADF824E0CDF82AE0CDF82EE0CDF832E00B
:1013C00006AF0FCF824E84F82DE00FC697E80F00CE
:1013D00007C626F8023B314601271B0CFE261F20BC
:1013E000C82201F81E3984F82B0084F82E2084F8D6
:1013F0002F7084F82A6094F8DE6284F82C6086F0FE
:10140000F10383EA0313DAB2130983F0E70343EA33
:10141000022383EAC2031BB283EA0312D2B2C3F3EC
:10142000072383EA121343EA022383EAC2031BB2AF
:1014300083F0C80282EA0212D2B2C3F3072383EA1E
:10144000121343EA022383EAC2031BB283EA0700B2
:1014500080EA0010C0B2C3F3072282EA101242EA07
:1014600000223E4482EAC00084F8DE62208501F159
:101470001F0611F8013B434083EA0313DBB21A094C
:1014800082EA102242EA032282EAC3031BB298B224
:10149000B1422085EDD183F07C0181EA0111C9B20E
:1014A0000B0983EA102383EA012383EAC1031BB2F9
:1014B0009AB24FEA122C5FFA83FEDFF82081228570
:1014C00084F850C084F84FE004F12A0704F14A0977
:1014D00038687968BA68FB6846460FC610374F45CA
:1014E000B046F5D1386830603A4E3B7988F8043020
:1014F00006F1270784F82DE384F82EC3D4F8C00240
:1015000016F8011F03681B689847B742F6D18BE1B4
:10151000B4F80832D4F85062D4F84C12D4F86021F0
:10152000D8B21B0A84F83F3284F8353284F83E0280
:1015300084F83402307C4FF47A73521A03FB00F3C0
:1015400000219A4284F8221284F8241280F0FF8449
:10155000D4F81422D4F810121F4894F85672C4F824
:101560001C5280FB013680FB0230C917D317C3EB36
:10157000A003C1EBA6021012191284F83C2284F8D1
:101580003D0284F8403284F84112002F7FF49AAB78
:10159000FFF7E5BB013BDBB284F86432D4F85802B4
:1015A000002B01F04B8612F8011B94F8706294F83E
:1015B00071320768C4F8602201338A193F6884F8E1
:1015C000702284F87132B84739E400BF504F0020D0
:1015D000BC180020931B002067666666941B0020E1
:1015E00094F8AE72C7B1013FFFB2AB4E013737443A
:1015F000002216F8013B534083EA0313DBB2120AC0
:10160000D90042EA0322B74281EA131382EA0302B5
:10161000EFD1002A7FF481AED4F8B8129F4E0B6B45
:10162000B4F80822D4F81072F066F261D4F8CC0154
:10163000D4F81422F762B4F8A872F063F264F76584
:10164000002B02F01C805B680A6C93423BBFCF68A2
:101650009B1A9F1AFF18002F7FF40AAC0B680846EC
:101660009B690221984794F8BC9294F8AF32029398
:10167000B9F1640F4FF0040386F8743041F05887D5
:1016800094F8BD32072B02F0378003F101095FFAAD
:1016900089F903F0F00203F00F0706EB0318059237
:1016A000D8F80410049108462EF03AFAD8F8083019
:1016B00003935FFA80F818462EF032FA059ADFF8A5
:1016C000ECA1A2725FFA80FB08EB0B0208320BEB75
:1016D000C8000499E271A07342460AF109006773D9
:1016E00030F0B2FC039B08F1090019465A465044F9
:1016F00030F0AAFCE37903F1010EC3B1581EC0B269
:101700000830674F20440AF10101002311F8012B32
:101710005A4093004FEAD20C83EA42030CF0180CB3
:10172000534047FA0CF253408842DBB2EED10AF83C
:101730000E30E3799DF80820E27003F03F039A1C15
:1017400003F10A0E627184F802E0564C0833E01887
:101750002746002217F8013B534083EA0313DBB20C
:10176000120AD90042EA032281EA131353401BB242
:10177000B8429AB2EED1A644120A0EF8023CA378FF
:1017800084F8BD9223444FF0000903F8012C84F83B
:10179000BC92A3786BB10027D4F8B802E15D03686E
:1017A0001B6898470137A378FFB2BB42F4D894F87E
:1017B000BC92032309F1010984F8BC9286F87430C5
:1017C00084F8A332D4F8B80203685B69984700280C
:1017D0003FF453ABD4F8B802036801219B699847E2
:1017E0000222002386F8742084F8A332FFF745BB59
:1017F000D4F824643368D3F81C801746B8F1000F7E
:1018000000F0BF8330462849C047002384F82134C4
:10181000C5E4D4F85802036802219B699847FFF792
:101820000BBB013B84F8CA3294F8CB22002A41D189
:1018300094F81014D4F860310A2084F8CB020029FF
:1018400000F0F0840129B4F8E08141F25E870229BA
:10185000B4F8E2B101F07D850329B4F8E4E101F0C8
:101860006387B4F8E6010390042901F0578705293E
:10187000B4F8E80101F063870629B4F8EAC101F081
:101880005A870729B4F8EC7101F03C87B4F8EE21CF
:10189000029200F0CFBC00BF381B002004000020E3
:1018A0000007090E8C180020C4190020921800208F
:1018B00088C3E43A013A84F8CB2294F8D272002F1C
:1018C00040F0E280B4F9D43194F8DEE2B4F9D611F4
:1018D0001FED096AD4F86021069206EE903AB4F939
:1018E000D83184F82D7007EE103A8EF06A0383EA3F
:1018F0000313D8B2030983F0D50343EA002383EA34
:10190000C0031BB283EA03104942C0B207EE901A2B
:10191000C3F3072383EA101343EA0023F8EEE77AC0
:10192000F8EEE66AB8EEC77A83EAC0031BB267EE48
:10193000867A66EE866A27EE067A4FF0000883F014
:10194000C806CDF82880CDF82C80CDF83080CDEDBC
:10195000087ACDED076A8DED097A86EA061C0DF14D
:1019600018085FFA8CFCC3F30726B8E80F0086EA74
:101970001C1646EA0C2686EACC06DFF804C136B20D
:10198000ACE80F0086F01E0798E8070087EA071307
:10199000DBB2C6F3072787EA131747EA03278CE869
:1019A000070087EAC3071C21ACF110064FF00509B8
:1019B0004FF01E08FE20C8220EF1010384F82B1000
:1019C00084F8D29284F82F8084F82A0084F82E209C
:1019D000711884F82CE0278584F8DE3216F8013B74
:1019E0007B4083EA0313DBB21A0982EA172242EA38
:1019F000032282EAC3031BB29FB28E422785EDD138
:101A000083F0270282EA0212D2B2130983EA172373
:101A100083EA022383EAC2031BB29AB24FEA122C72
:101A20005FFA83FEDFF85480228584F84DC084F885
:101A30004CE004F12A0704F14A0938687968BA6869
:101A4000FB6846460FC610374F45B046F5D10A4EE3
:101A50003B88A8F8003006F1240784F82AE384F8CC
:101A60002BC3D4F8C00216F8011F03681B689847FF
:101A7000B742F6D10BE000BF931B0020941B00205F
:101A8000BC1800200AD7233C013F84F8D27294F896
:101A9000D392B9F1000F40F04A82D4F8D432052233
:101AA00013F0140F84F8D32200F0AA83D4F81C3466
:101AB0001FED0C7A07EE903AF8EEE77A67EE877A38
:101AC00094F8DE72B4F9E661B4F9D821724873492A
:101AD000CDED087A87F0220383EA03135FFA83FED1
:101AE0004FEA1E1383F05903B6F5FA6F43EA0E234B
:101AF00083EACE03A8BF4FF4FA661BB2B6F57A7F2D
:101B000083EA031EB8BF4FF47A764FF0640C5FFA95
:101B10008EFEA6F57A76C3F307230CFB06F683EA5E
:101B20001E1381FB02C180FB06C043EA0E28F61794
:101B3000D2174FF0000BC6EBA010C2EBA10388EA4E
:101B4000CE080FFA88F8ADF82A00ADF82830CDF8A5
:101B500018B0CDF81CB0CDF824B00DF1180EBEE8C9
:101B60000F0088F0C80C8CEA0C1C5FFA8CFCC8F3E0
:101B7000072686EA1C16DFF83481DEF800E084F8D8
:101B80002C7046EA0C26A8E80F0086EACC031BB2AC
:101B900083F04A0686EA0616F6B2C3F3072282EA03
:101BA000161248F810E942EA06224A2382EAC606DB
:101BB0004FF0140E01374FF0FE0C002284F82F3046
:101BC000C82384F8DE722685414608EB0E0084F8AF
:101BD0002AC084F82BE084F82D2084F82E3011F8E8
:101BE000013B734083EA0313DBB21A0982EA16222F
:101BF00042EA032282EAC3031BB29EB281422685D7
:101C0000EDD183F0140383EA0313DBB24FEA131E12
:101C10008EEA162E8EEA032E8EEAC30E26460FFAA1
:101C20008EFE1FFA8EFB56F82A0F1D4FA4F828B01F
:101C30004FEA1B2C5FFA8EFE84F844E084F845C01E
:101C40007168F368B2680FC730697169338B03C775
:101C500004F207363B8004F2233B374684F823C363
:101C600084F822E3D4F8C00217F8011F03681B6848
:101C70009847BB45F6D10B4B0B4A93F8B332127819
:101C8000013B12F00401DBB214BFC0224022172B2B
:101C900040F2AF830CE000BFD34D6210676666660A
:101CA000941B002074450020744F0020BC180020B5
:101CB000B4F87A0287071ABF002342F0100201230A
:101CC00010F4027F18BF022310F0100F18BF062374
:101CD00010F0200F18BF1023002941F018830321B2
:101CE00094F8DE72069387F0460383EA0313D8B2B2
:101CF000030983F0920343EA002383EAC0031BB283
:101D000083EA0310C0B2C3F3072383EA101343EA44
:101D1000002383EAC0031BB283F0C80E8EEA0E1EB6
:101D20005FFA8EFE4FF0000C0320C3F307238DF8FB
:101D30001C908DF81E208DF81DC08DF81F108DF899
:101D4000200083EA1E1306AA07CA43EA0E2383EA89
:101D5000CE031BB283EA031EA8E803005FFA8EFEDF
:101D6000C3F3072383EA1E1343EA0E2383EACE0359
:101D700094F830E088F800201BB28EEA030282EA71
:101D80000212D2B2C3F3072383EA121343EA0223F7
:101D900094F8310094F8321094F8338094F834E0D9
:101DA00084F82FC083EAC2031BB2584080EA0010B7
:101DB000C0B2C3F3072383EA101343EA002383EA84
:101DC000C0031BB2594081EA0111C9B2C3F3072312
:101DD00083EA111343EA012383EAC1031BB288EAB1
:101DE000030888EA08185FFA88F8C3F3072383EA30
:101DF000181343EA082383EAC8031BB28EEA030ED2
:101E00008EEA0E1E5FFA8EFEC3F3072383EA1E13CB
:101E100043EA0E2394F8350094F8361094F83720EE
:101E200094F8388084F82DC083EACE031BB2584062
:101E300080EA0010C0B2C3F3072383EA101343EA19
:101E4000002383EAC0031BB2594081EA0111C9B2E1
:101E5000C3F3072383EA111343EA012383EAC1038F
:101E60001BB25A4082EA0212D2B2C3F3072383EABA
:101E7000121343EA022383EAC2031BB288EA030275
:101E800082EA0212D2B2C3F3072383EA121343EAAF
:101E9000022383EAC2031BB283F0320282EA0212F7
:101EA000D2B2C3F3072383EA121343EA022383EA7D
:101EB000C2031BB2DFF860E384F82C709AB24FF0D3
:101EC000FE0C0920C8214FEA12290137DBB284F841
:101ED0002AC084F82E1084F82B0084F8DE72228544
:101EE00084F83A9084F83930DEF80000DEF8041007
:101EF000DEF80820BEF80CB00EF2DE2CACE80700CD
:101F00000EF2EE278CF80280ACF800B084F818933B
:101F100084F81733D4F8C00216F8011F03681B6851
:101F20009847B742F6D1C4F8C4A2FEF7B7BF09F18B
:101F3000FF3984F8D392F6E7072303EB430302EB60
:101F400083020023CB6213815360FEF769BF94F8CC
:101F50005422D4F86031C4F84C32032A3FF4F8AA72
:101F600094F85532934238BF1346013B012B3FF69C
:101F7000EFAA1022022384F8222284F82432FFF7E9
:101F8000E7BADFF8988200E033689B6830469847EC
:101F90000028F9D0336818F8011B1B6830469847B1
:101FA000013FF1D131E4D4F8DC212120002371215B
:101FB00084F83A04100184F8383484F8393484F809
:101FC0005C1440F1D78290484FF0030CB4F87A3299
:101FD000590501F14781DA0701F1B28103F00203EB
:101FE0008A4A002B1CBF4FF0030C1046DFF83082EA
:101FF00001384746712300216FF02A0E10F8012F97
:1020000007F8012B53405A0013F0800F82F0D509D6
:10201000D2B25FFA89F908BF91464FEA490282F0CD
:10202000D50319F0800F5FFA83F9D3B218BF4B467E
:102030004FEA430913F0800F89F0D5025FFA89F95E
:10204000D2B208BF4A464FEA420912F0800F89F027
:10205000D5035FFA89F9DBB208BF4B464FEA430963
:1020600013F0800F89F0D5025FFA89F9D2B208BF68
:102070004A464FEA420912F0800F89F0D5035FFA11
:1020800089F9DBB208BF4B464FEA430913F0800FD2
:1020900089F0D5025FFA89F9D2B208BF4A465300E7
:1020A00083F0D50912F0800F01F101015FFA89F286
:1020B000DBB218BF13468C45A0DC5A0082EA0E0141
:1020C00013F0800FC9B2D3B218BF0B46590081EA92
:1020D0000E0213F0800FC9B2D3B208BF0B465900ED
:1020E00081EA0E0213F0800FC9B2D2B208BF0A46CD
:1020F000530083EA0E0112F0800FCAB2DBB218BFA0
:102100001346590081EA0E0213F0800FC9B2D2B211
:1021100008BF0A46530083EA0E0112F0800FDBB2BB
:10212000CAB208BF1A46530083EA0E0112F0800FAC
:10213000DBB2CAB208EB0C0708BF1A46344950009C
:1021400007F10209A9EB010980EA0E0312F0800FE2
:10215000C0B2DBB208BF0346B9F1240FA8BF4FF0ED
:102160002409A7EB010E002208F80C20A1F540700D
:1021700084F839E44A467B7084F85C342FF064FFBD
:1021800084F82194FFF723B8B4F87A32D90500F126
:102190003581D80601F1D980990601F190815A065E
:1021A00001F19A81180701F17382D90701F19D822B
:1021B00013F0020F0CBF04230C2302931FE1B4F8A9
:1021C000A83200220133A4F8A83284F8A322FEF733
:1021D00054BED4F85802036801219B699847D4F88B
:1021E000580206E0D4F858020368DB689847D4F830
:1021F000580203685B6898470028F3D1FEF71FBEBA
:10220000DFED047A5CE400BFC0790308D0790308ED
:10221000C41C002000000000B6180020C4190020D3
:10222000C71C00200F468C46084603918E468B46FD
:102230008846029194F8DE62069386F0300383EAC2
:102240000313DBB24FEA1319B4F8A012C44A84F89E
:102250002C6089F07A09C1EB012149EA032989EA56
:10226000C30382FB01298944C917C1EB69214FF0DF
:10227000000968F30F09039A8DF82D104FF000083C
:102280006EF30F084FF0000E62F31F481BB260F3AD
:102290000F0E029ACDF82080002067F30F0083EA2A
:1022A0000317FFB26CF31F4E6BF31F4962F31F401D
:1022B0004FF0000CC3F3072383EA1713CDF81C90EB
:1022C000CDF824E00A908DF82CC00DF1180E43EAE9
:1022D0000728BEE80F0088EAC7073FB287F0C809A1
:1022E000DFF88C8284F82DC089EA0919A8E80F006C
:1022F0005FFA89F9C7F3072787EA19139EE80300F5
:1023000043EA092383EAC9031BB248F8040B83F0AC
:10231000230787EA0717FFB24046C3F3072282EA82
:10232000171242EA072220F8141982EAC707013679
:1023300016224FF023084FF0FE0EC82384F8DE6209
:102340002785811884F82F8084F82AE084F82B20D0
:1023500084F82E3010F8013B7B4083EA0313DBB294
:102360001A0982EA172242EA032282EAC3031BB255
:102370009FB288422785EDD183F0F40181EA0111F3
:10238000C9B20E0986EA172686EA012686EAC10640
:10239000A64636B21FFA86F85EF82A0F714FA4F8E7
:1023A00028804FEA182CF6B284F8466084F847C0BB
:1023B000DEF80410DEF80820DEF80C300FC7DEF877
:1023C0001000DEF81410DEF8182004F2073807C7F2
:1023D00004F2253784F825C384F82463D4F8C002B6
:1023E00018F8011F03681B6898474745F6D1FFF7A7
:1023F00064BA5D48034493F80C9059E402925B4A36
:1024000094F87F3292F800A0CAF3800A0BB14AF028
:10241000020A4FF0000B306887F800B003682421EF
:102420001B6898473068036854211B6898473068D8
:10243000036853211B689847B4F80832306803EBEF
:10244000830303EB83034FEA830902681FFA89F9C8
:102450005FFA89F319461268039390473A78039B11
:10246000306853403B7003684FEA192949461B689E
:1024700098473B78306889EA03033B700368594604
:102480001B6898473068036859461B689847B4F83A
:10249000A032334A3068C3EBC3135B0082FB0312E4
:1024A0001A444FEAE379C9EB622903685FFA89F9B4
:1024B00049461B6898473B78306889EA030987F8E2
:1024C0000090036859461B6898473068029A036871
:1024D00042EA0A0A51461B689847397830688AEA06
:1024E000010A5FFA8AF1397003681B68984794F80B
:1024F0007832002B7EF4EFAE30683B700368242105
:102500001B6898473068036854211B6898473068F7
:1025100003684F211B6898472AF06CFB2AF06AFB7E
:102520002AF068FB3068036801211B6898473B78F4
:10253000306894F8A29283F001033B70036809F0BD
:1025400001091B68494698473978306889EA0101D2
:10255000397003681B68984794F87832FEF7BBBE61
:1025600003082080941B0020B84E0308744F0020FD
:10257000BC180020894B8A4A1B688A4803F48003F0
:10258000002B0ABF10464FF0030C4FF0040C1DE562
:10259000B4F80832B4F9109203EB830303EB83031E
:1025A0009F0018F021FABFB240B2FEF7F5BE072334
:1025B00003EB430302EB83030022CA621A815A60D1
:1025C000FEF7BFBBD4F8AC01774E03685E211B68F1
:1025D0009847D4F8AC01036802211B689847D4F8E7
:1025E000D031323386FB0326DB17C3EB6616F0B21D
:1025F00008F012FAC6F3072008F00EFAD4F8AC017E
:1026000003685E211B689847D4F8AC010368032176
:102610001B689847654B1B78580740F12886DFF800
:102620007C81D8F80030D90440F17986D4F8DC21D7
:10263000D20000F174865E4AB4F9E611B2F86A225B
:10264000D01B814203DD3A449142C0F27086B4F956
:102650009E34584ADE1782FB0323C6EB630636B26C
:10266000F0B2C6F3072608F0D7F9304608F0D4F9DF
:10267000D8F80030504A1A4204D0504F3B78002B13
:1026800040F06F86D4F80C32D4F8AC011A7B0368A2
:10269000002A1B684FF05E0114BF3C266426984751
:1026A000D4F8AC01036813211B689847304608F042
:1026B000B3F9002008F0B0F9D4F8AC0103685E214A
:1026C0001B689847D4F8AC0103681B211B68984726
:1026D000002008F0A1F9002008F09EF9D4F8AC0120
:1026E00003685E211B689847D4F8AC010368232176
:1026F0001B6898474E2008F08FF9D4F8AC010368A6
:1027000000211B689847D4F80C32D4F8AC011A7B2E
:102710000368002A1B684FF05E0114BF3C26642644
:102720009847D4F8AC01036812211B6898473046DB
:1027300008F072F9002008F06FF9D4F8AC010368D2
:102740005E211B689847D4F8AC0103681A211B6806
:102750009847002008F060F9002008F05DF9D4F8EF
:10276000AC0103685E211B689847D4F8AC0103688C
:1027700022211B689847452008F04EF9D4F8AC0197
:10278000036800211B689847D4F8AC0103685E21F8
:102790001B68984794F86831FEF7AEBC504F002094
:1027A000B8790308C07903081F85EB51744F0020E6
:1027B000744500206766666602000008544F0020DA
:1027C000B4F80812D4F81022DFF8E0E5080A80F027
:1027D000290C4FEA4C031CF0800F83F0D50CDBB2C0
:1027E0005FFA8CFC08BF9C464FEA4C031CF0800F3C
:1027F00083F0D50CDBB25FFA8CFC08BF9C464FEA35
:102800004C031CF0800F83F0D50CDBB25FFA8CFC1C
:1028100008BF9C464FEA4C031CF0800F83F0D50C98
:10282000DBB25FFA8CFC08BF9C464FEA4C031CF0FD
:10283000800F83F0D50CDBB25FFA8CFC08BF9C469E
:102840004FEA4C031CF0800F83F0D50CDBB25FFA2B
:102850008CFC08BF9C464FEA4C031CF0800F83F0B1
:10286000D50C5FFA8CFCDBB218BF63464FEA430C11
:1028700013F0800F8CF0D5035FFA8CFCC9B2DBB289
:1028800008BF63464B404FEA430C13F0800F8CF0B7
:10289000D503DBB25FFA8CFC18BF9C464FEA4C03B1
:1028A0001CF0800F83F0D50CDBB25FFA8CFC08BF04
:1028B0009C464FEA4C031CF0800F83F0D50CDBB232
:1028C0005FFA8CFC08BF9C464FEA4C031CF0800F5B
:1028D00083F0D50CDBB25FFA8CFC08BF9C464FEA54
:1028E0004C031CF0800F83F0D50CDBB25FFA8CFC3C
:1028F00008BF9C464FEA4C031CF0800F83F0D50CB8
:10290000DBB25FFA8CFC08BF9C464FEA4C031CF01C
:10291000800F83F0D50C5FFA8CFCDBB218BF6346E6
:1029200013F0800F8EFB02CE4FEA43034FEAE272B0
:10293000C2EBAE0283F0D50E5FFA8EFEDBB218BF9B
:102940007346C2F3072E8EEA03034FEA430C13F0DB
:10295000800F8CF0D503DBB25FFA8CFC18BF9C466D
:102960004FEA4C031CF0800F83F0D50CDBB25FFA0A
:102970008CFC08BF9C464FEA4C031CF0800F83F090
:10298000D50CDBB25FFA8CFC08BF9C464FEA4C03C7
:102990001CF0800F83F0D50CDBB25FFA8CFC08BF13
:1029A0009C464FEA4C031CF0800F83F0D50CDBB241
:1029B0005FFA8CFC08BF9C464FEA4C031CF0800F6A
:1029C00083F0D50CDBB25FFA8CFC08BF9C464FEA63
:1029D0004C031CF0800F83F0D50C5FFA8CFCDBB24B
:1029E00018BF63464FEA430C13F0800F8CF0D503F9
:1029F0005FFA8CFCD2B2DBB208BF634653404FEAA9
:102A0000430C13F0800F8CF0D503DBB25FFA8CFC23
:102A100018BF9C464FEA4C031CF0800F83F0D50C86
:102A2000DBB25FFA8CFC08BF9C464FEA4C031CF0FB
:102A3000800F83F0D50CDBB25FFA8CFC08BF9C469C
:102A40004FEA4C031CF0800F83F0D50CDBB25FFA29
:102A50008CFC08BF9C464FEA4C031CF0800F83F0AF
:102A6000D50CDBB25FFA8CFC08BF9C464FEA4C03E6
:102A70001CF0800F83F0D50CDBB25FFA8CFC08BF32
:102A80009C464FEA4C031CF0800F83F0D50C5FFA94
:102A90008CFCDBB218BF63464FEA430C13F0800F87
:102AA0008CF0D50AD4F8043284F83C145FFA8CFC1C
:102AB0005FFA8AFA4FF00A0108BFE2464FF00008B9
:102AC00084F83E240822B3F80E9084F83DE484F89C
:102AD000391484F83A2484F83B0484F85CA484F81C
:102AE000388417F081FF4FEA4A031AF0800F83F011
:102AF000D502DBB2D2B208BF1A46530012F0800FE3
:102B000083F0D502DBB2D2B208BF1A46530012F0EE
:102B1000800F83F0D502DBB2D2B208BF1A46530051
:102B200012F0800F83F0D502DBB2D2B208BF1A4692
:102B3000530012F0800F83F0D502DBB2D2B208BF8F
:102B40001A46530012F0800F83F0D502DBB2D2B2E6
:102B500008BF1A46530012F0800F83F0D502D2B29C
:102B6000DBB218BF13465A0013F0800F82F0D50372
:102B7000D2B24FEA1921DBB208BF13464B405A00CC
:102B800013F0800F82F0D503DBB2D2B218BF1A4621
:102B9000530012F0800F83F0D502DBB2D2B208BF2F
:102BA0001A46530012F0800F83F0D502DBB2D2B286
:102BB00008BF1A46530012F0800F83F0D502DBB233
:102BC000D2B208BF1A46530012F0800F83F0D5022C
:102BD000DBB2D2B208BF1A46530012F0800F83F066
:102BE000D502DBB2D2B208BF1A46530012F0800FF2
:102BF00083F0D502D2B2DBB218BF13465A0013F0ED
:102C0000800F5FFA82FE82F0D503DBB25FFA89F2B1
:102C100008BF734653404FEA430E13F0800F8EF007
:102C2000D503DBB25FFA8EFE18BF9E464FEA4E0315
:102C30001EF0800F83F0D50EDBB25FFA8EFE08BF68
:102C40009E464FEA4E031EF0800F83F0D50EDBB296
:102C50005FFA8EFE08BF9E464FEA4E031EF0800FBD
:102C600083F0D50EDBB25FFA8EFE08BF9E464FEAB8
:102C70004E031EF0800F83F0D50EDBB25FFA8EFE9E
:102C800008BF9E464FEA4E031EF0800F83F0D50E1C
:102C9000DBB25FFA8EFE08BF9E464FEA4E031EF07F
:102CA000800F83F0D50E5FFA8EFEDBB218BF73463D
:102CB0004FEA430E13F0800F8EF0D5035FFA8EFEBD
:102CC000DBB208BF734643404FEA430E13F0800F58
:102CD0008EF0D503DBB25FFA8EFE18BF9E464FEA38
:102CE0004E031EF0800F83F0D50EDBB25FFA8EFE2E
:102CF00008BF9E464FEA4E031EF0800F83F0D50EAC
:102D0000DBB25FFA8EFE08BF9E464FEA4E031EF00E
:102D1000800F83F0D50EDBB25FFA8EFE08BF9E46B1
:102D20004FEA4E031EF0800F83F0D50EDBB25FFA40
:102D30008EFE08BF9E464FEA4E031EF0800F83F0C2
:102D4000D50EDBB25FFA8EFE08BF9E464FEA4E03F9
:102D50001EF0800F83F0D50E5FFA8EFEDBB218BF37
:102D600073464FEA430E13F0800F8EF0D503DBB2AB
:102D70005FFA8EFE18BF9E460B4B84F8412484F800
:102D80003F8403F5407284F8420484F8401484F8C8
:102D900043E407CA83E807000C2384F85CE484F862
:102DA0002134FEF711BA00BFC419002067666666B9
:102DB00058A08B41B4F9D6311FED036A06EE903A64
:102DC000F8EEE66AB4F9D43166EE866A07EE103A98
:102DD000FDEEE66AB4F9D831CDED026ABDF908001E
:102DE000C0F3072888F0FA0207EE903A530012F079
:102DF000800F83F0D502DBB2D2B208BF1A4653006F
:102E000012F0800F83F0D502DBB2D2B208BF1A46AF
:102E1000530012F0800F83F0D502DBB2D2B208BFAC
:102E20001A46530012F0800F83F0D502DBB2D2B203
:102E300008BF1A46530012F0800F83F0D502DBB2B0
:102E4000D2B208BF1A46530012F0800F83F0D502A9
:102E5000DBB2D2B208BF1A46530012F0800F83F0E3
:102E6000D502D2B2DBB218BF13465A0013F0800F5E
:102E700082F0D503D2B2C0B2DBB208BF13464340E2
:102E80005A0013F0800F82F0D503DBB2D2B218BF24
:102E90001A46530012F0800F83F0D502DBB2D2B293
:102EA00008BF1A46530012F0800F83F0D502DBB240
:102EB000D2B208BF1A46530012F0800F83F0D50239
:102EC000DBB2D2B208BF1A46530012F0800F83F073
:102ED000D502DBB2D2B208BF1A465300B8EEC77AA9
:102EE00012F0800F83F0D502DBB2D2B227EE067A61
:102EF00008BF1A46530012F0800FBDEEC77A83F068
:102F0000D502D2B2DBB28DED037A18BF13465A0058
:102F1000BDF90C1084F83B8413F0800F82F0D503C8
:102F2000D2B2C1F3072CDBB208BF13468CEA03030D
:102F300013F0800F4FEA430383F0D502D2B2DBB225
:102F400018BF134613F0800F4FEA430383F0D502F6
:102F5000D2B2DBB218BF134613F0800F4FEA43031F
:102F600083F0D502D2B2DBB218BF134613F0800F44
:102F70004FEA430383F0D502D2B2DBB218BF134647
:102F800013F0800F4FEA430383F0D502D2B2DBB2D5
:102F900018BF134613F0800F4FEA430383F0D502A6
:102FA000D2B2DBB218BF134613F0800F4FEA4303CF
:102FB00083F0D502D2B2DBB218BF134613F0800FF4
:102FC0004FEA430383F0D502D2B2C9B2DBB218BFD5
:102FD00013464B4013F0800F4FEA430383F0D502B2
:102FE000D2B2DBB218BF134613F0800F4FEA43038F
:102FF00083F0D502D2B2DBB218BF134613F0800FB4
:103000004FEA430383F0D502D2B2DBB218BF1346B6
:1030100013F0800F4FEA430383F0D502D2B2DBB244
:1030200018BF134613F0800F4FEA430383F0D50215
:10303000D2B2DBB218BF134613F0800F4FEA43033E
:1030400083F0D502D2B2DBB2F8EEE77A18BF1346AE
:103050005A0013F0800F67EE867A82F0D5035FFA8C
:1030600083FEFDEEE77AD3B218BF73465A0013F021
:10307000800FCDED027A82F0D503D2B2DBB208BF69
:103080001346BDF9082084F83C04C2F3072E8EEAEB
:10309000030313F0800F4FEA430383F0D5095FFA6F
:1030A00089F9DBB218BF4B4613F0800F4FEA430398
:1030B00083F0D5095FFA89F9DBB218BF4B4613F0EC
:1030C000800F4FEA430383F0D5095FFA89F9DBB239
:1030D00018BF4B4613F0800F4FEA430383F0D50926
:1030E0005FFA89F9DBB218BF4B4613F0800F4FEA45
:1030F000430383F0D5095FFA89F9DBB218BF4B4669
:1031000013F0800F4FEA430383F0D5095FFA89F982
:10311000DBB218BF4B4613F0800F4FEA430383F036
:10312000D5095FFA89FA5FFA83F918BFD14619F019
:10313000800F4FEA490989F0D5035FFA89F9D2B2C5
:10314000DBB208BF4B46534013F0800F4FEA4303F6
:1031500083F0D5095FFA89F9DBB218BF4B4613F04B
:10316000800F4FEA430383F0D5095FFA89F9DBB298
:1031700018BF4B4613F0800F4FEA430383F0D50985
:103180005FFA89F9DBB218BF4B4613F0800F4FEAA4
:10319000430383F0D5095FFA89F9DBB218BF4B46C8
:1031A00013F0800F4FEA430383F0D5095FFA89F9E2
:1031B000DBB218BF4B4613F0800F4FEA430383F096
:1031C000D5095FFA89F9DBB218BF4B4613F0800FBF
:1031D0004FEA430383F0D5095FFA89F9DBB218BFE0
:1031E0004B4613F0800F4FEA430383F0D508DBB260
:1031F0005FFA88F884F83DC408BF984684F83E1406
:1032000008201E21C14B84F83FE44FF0000C84F8E5
:10321000402484F8418484F838C484F8390484F85C
:103220003A1493E80700A3F5407303C30A2184F816
:103230005C841A8084F82114FDF7C3BF94F87012DF
:1032400094F8713202684E1C0133126884F870627F
:1032500084F871329047FDF7F2BDC4F85C523770C4
:10326000FDF73FBE4FF0030CA948FEF7BFBED4F8F0
:103270000422A84BD689DFF8B482A3FB0636B60831
:10328000F0B207F0C9FB300A07F0C6FBFFF7F0B950
:10329000D4F8AC01DFF88C9203685E211B68984774
:1032A000D4F8AC01036810211B689847D4F8CC31DE
:1032B00089FB0328DB17C3EB68185FFA88F007F077
:1032C000ABFBC8F3072007F0A7FBD4F8AC010368F9
:1032D0005E211B689847D4F8AC01036821211B6864
:1032E0009847D4F8CC2189FB0213D017C0EB6310A8
:1032F000642303FB102383EAE370A0EBE370C0B206
:1033000007F08AFB304607F087FBFDF7B6BE94F85E
:103310007F1200290CBF04210521FEF7E1BC7E4A83
:10332000B4F9E611B2F86C229142BFF690A9DB061F
:10333000B4F99E2440F1DD8000263046FFF793B9B2
:103340004FF0040C7548FEF751BE34230293FFF78B
:1033500056B8174694461046039296460292FEF7D8
:1033600069BFB4F80A62D4F8AC01B4F80812642258
:10337000360102FB0131B6B202685B00B1FBF3F328
:1033800046EA03261268C3F303235E21B6B21E4346
:103390009047D4F8AC01036806211B689847F0B247
:1033A00007F03AFB300A07F037FBB4F80A32D4F8DA
:1033B0000C023A78867B01339BB2012E93FBF2F12B
:1033C00002FB1133A4F80A3200F07581B4F80862E8
:1033D0005349C07B6E2303FB06F381FB0361DB17BC
:1033E000C3EBA10310B19BB293FBF2F34D4E9FB21E
:1033F000A6FB073676093A201FFA86F807F034FB59
:103400005FFA88F007F008FB4FEA182007F004FB8A
:10341000D4F8AC0103685E211B689847D4F8AC016E
:1034200003683B211B689847642303FB16739BB218
:103430003D48053380FB0320DB17C3EBA000C0B27F
:1034400007F0EAFA002007F0E7FAD4F8AC010368C5
:103450005E211B689847D4F8AC01036828211B68DB
:103460009847314AD4F81032DE1782FB0323C6EBAB
:10347000A306F0B207F0D0FAC6F3072007F0CCFAA3
:10348000D4F8AC0103685E211B689847D4F8AC01FE
:10349000036804211B689847D4F80432DB89002BA9
:1034A00040F01581D4F8146286F31006F0B207F0EC
:1034B000B3FAC6F3072007F0AFFAFFF7E3B8242307
:1034C0000293FEF79CBF0323FEF737BD0223FEF7EE
:1034D00034BD0023FEF731BD10230293FEF78FBFEA
:1034E0000623FEF72ABD0523FEF727BD0423FEF7BA
:1034F00024BD0D4BD61783FB0232C6EB620636B2F3
:10350000F0B2C6F30726FFF7AEB800BFC41C002018
:10351000C4790308CDCCCCCC74450020C87903080D
:10352000310CC3301F85EB5167666666504F002033
:1035300096F87500DFF818B2DFF818A2020704BF8A
:103540000130C0B2062888BF012006EB00134FEA05
:10355000001E1F7C00231BF80710A37252465FFA5F
:103560008EF806EB0E0348EA070701291770DB689F
:1035700002F1010C0CD90239CFB2B91C11446246D8
:1035800002F8013B8A424FEA1323F9D10137BC44C8
:10359000B64401309EF8112023F06003C0B21343FB
:1035A00008288CF800300CF1010200F0A2804FEAEC
:1035B000001E06EB0E01A2EB0A030F7C1BF807109E
:1035C00001EB030C08F11008BCF1130F5FFA88F847
:1035D000C7DDDBB29A1DD2B242F04001E17102F1C7
:1035E000010C594FE2B10533DBB20833DFF868E173
:1035F0002344791C002211F8018B88EA02084FEA63
:1036000088024FEAD80A82EA48020AF0180A82EAD7
:1036100008024EFA0AF882EA08029942D2B2EAD1C6
:1036200007F80C20E3799DF80820E27003F03F03CF
:103630009A1C03F10A076271A770444C86F8750062
:103640000833E018A64600221EF8013B534083EAE7
:103650000313DBB2120AD90042EA032281EA1313F0
:1036600053401BB270459AB2EED12744120A07F8B4
:10367000023CA378234403F8012CFEF78AB8CB69F7
:103680000F6ABB423CBFCA689B18DF1BFDF7E3BF54
:1036900020230293FEF7B3BE0523FEF789BF042360
:1036A000FEF786BF0323FEF783BF0223FEF780BF2A
:1036B0000123FEF77DBF392007F0D6F9B4F8086280
:1036C000F0B207F0A9F9300A07F0A6F9BDE617F045
:1036D0008BF907F0A1F90021D4F8AC0113F098FDA3
:1036E000FEF7D0BF0623FEF763BF08230293FEF761
:1036F00086BEA2EB0A036CE73A463B464FF001094F
:10370000FDF7CBBF0292FEF795BD174694461046D3
:103710000392964693460292FEF78CBD1746944656
:1037200010460292FEF786BD174694461046039255
:103730000292FEF77FBD17460292FEF77BBD174649
:1037400094460292FEF776BD921800208C18002055
:10375000B84E0308991800200007090E2DE9F04F14
:103760000F46B0F908102DED028B3981C9B24B1EFE
:1037700091B01546FD2B00F20081DFE813F04A05F9
:103780003F0517050805E704FE00FE00FE00FE00E9
:10379000D604FE00FE00FE00FE00FE00FE00FE005D
:1037A000FE00FE00FE00FE00FE00FE00FE00FE0029
:1037B000FE00FE00FE00FE00FE00FE00FE00FE0019
:1037C000B004FE00A804FE009504FE007C04FE0088
:1037D0007704FE002B04FE001304FE000804FE0024
:1037E0000304FE002E0AFE00A102FE002203FE00DA
:1037F0009C02D102FE001203FE00FE000603FE0042
:10380000D902FE00FB038D02E703FE00FE00DE038B
:10381000FE00BD03FE009D03FE0059033F03FE00B2
:103820005B05FE009B07FE00FE00FE00FE00FE00A2
:103830006907FE003507FE00DC06FE00CB06FE0031
:10384000FE00FE00880650061C060C06F405E30583
:10385000FE00FE00CB05BE05FB0185056B05FE00E5
:10386000C108B7087B086F08FE003908FF07FE0093
:10387000FE00FE00EB07CF07AE096F09FE00FE0059
:10388000FE00FE00FE00FE00FE00FE00FE00FE0048
:10389000FE00FE00FE00FE00FE00FE00FE00FE0038
:1038A000FE00FE00FE00FE002E09FE00FE00FE00EF
:1038B000FE00FE00FE00FE00FE00FE001B09FE00F2
:1038C000FE00FE00FE00FE00FE00FE00FE00FE0008
:1038D000FE00FE00FE00FE00FE00FE00FE00FE00F8
:1038E000FE00FE00FE00FE00FE00FE00FE00FE00E8
:1038F000FE00FE00FE00FE00FE00FE00FE00FE00D8
:10390000FE00FE00FE00FE00FE00FE00FE00FE00C7
:10391000FE00FE00FE00FE00FE00FE00FE00FE00B7
:10392000FE00FE00FE00FE00FE00FE00FE00FE00A7
:10393000FE00FE00FE00FE00FE00FE00FE00FE0097
:10394000FE00FE00FE00FE00FE00FE00FE00FE0087
:10395000FE00FE00FE00FE00FE00FE00130AC0098D
:10396000FE00FE00FE00FE00FE00FE00FE00FE0067
:10397000FE00FE00FE00FE00220AF529044600F0CB
:10398000318194E828000B39ED1AEF2901F28D817D
:10399000DFE811F093098B098B098B098B098B09DF
:1039A0008B098B098B098B098B098B098B098B0977
:1039B0008B098B098B098B098B098B098B098B0967
:1039C0008B098B09AE098B09E3098B09EF098B0978
:1039D000030A8B091D0A8B09270A8B09830A8B09A5
:1039E000AA0A8B09BF0A8B09C90A8B094F098B09DF
:1039F000F90A8B098B091F018B091B0B8B098B099A
:103A00002B0B8B09C50C8B098B098B098B098B0937
:103A10008B09F50C8B09FC0C8B09220D8B098B098A
:103A20004B0D8B09650D8B097E0D8B09A40D8B0940
:103A30008B098B09100E8B09430E8B09670E8B09BE
:103A4000D80E8B098B098B098B098B098B098B0984
:103A50008B098B098B098B098B098B098B098B09C6
:103A60008B098B098B098B098B098B098B098B09B6
:103A70008B098B098B098B098B098B098B098B09A6
:103A80008B098B098B098B098B098B098B098B0996
:103A90008B098B098B098B098B098B098B098B0986
:103AA0008B098B098B098B098B098B098B098B0976
:103AB0008B098B098B098B098B098B098B098B0966
:103AC0008B098B098B098B098B098B098B098B0956
:103AD0008B098B098B098B098B098B098B098B0946
:103AE0008B098B098B098B098B098B098B098B0936
:103AF0008B098B098B098B098B098B098B098B0926
:103B00008B098B098B098B098B098B098B09B90EE2
:103B10008B093B0F8B09ED0E2E0FCF0BDD0B310CFC
:103B20008B094A0C5E0C890C8B09670C8B098B097D
:103B3000750C880BA20BAA0BBF0B8B098B098B0989
:103B40008B098B098B098B098B098B098B098B09D5
:103B50008B098B098B098B098B098B09450B8B0909
:103B60008B09540B8B098B098B098B098B098B09EA
:103B70008B09380BC24B3A681B88C249FF2BA8BF80
:103B8000FF23501C3860137009684FF6FF74A14280
:103B9000A8BF214621EAE17189B238462AF096F998
:103BA000B94B384619882AF091F9B84B93F8453249
:103BB000002B01F0A086B64B1B6803EB8303590072
:103BC000A142A8BF214621EAE17189B238462AF014
:103BD0007DF901231A4618467A8111B0BDEC028B9B
:103BE000BDE8F08F94E80C00934241F04686A94B63
:103BF000FF2283F822204FF00009A74C13F00CFBA2
:103C000049463022A54884F8009030F056FD8DF8E2
:103C100000909DF800300B2B01F24C80DFF894826D
:103C20009E4E4A469DF8003003EB830308EB830366
:103C30001B7BE3B19DF8003003EB830308EB8303A8
:103C400020211B699BB19DF8003003EB830308EB37
:103C50008303186946F8220009F074FF237856F8A8
:103C600023000AF031F922780132D2B222709DF895
:103C700000300133DBB28DF800309DF800300B2BA3
:103C8000D0D93B68591C39601A70002DA1D0844BE3
:103C90002B6001231A469EE7824B03F10B043A681E
:103CA00013F8011B501C9C4238601170F7D10021A1
:103CB00038462AF0F3F8002138462AF0EFF888E772
:103CC000724C04F1400502E00834A54281D094F919
:103CD000DA62304618F04EFC0028F5D03B685A1CDA
:103CE0003A601E70B4F8D81238462AF0EFF83B68F4
:103CF00094F8DB22591C39601A703B6894F8DC2276
:103D0000591C39601A703B6894F8DE22591C3960DE
:103D10001A703B6894F8DD22591C39601A70D3E799
:103D2000396801200A183A6003460246087052E7D3
:103D3000564C3B6894F8B322591C39601A70A1683C
:103D400038462AF0ABF83B6894F85C22591C39607D
:103D50001A70B4F8E41138462AF0B8F8B4F8E8114B
:103D600038462AF0B3F8B4F8EC1138462AF0AEF829
:103D7000B4F8401238462AF0A9F8B4F8421238468E
:103D80002AF0A4F801231A4625E7474B03F108015E
:103D90003A6813F8010B541C8B423C601070F7D149
:103DA00017E73A68394B501C93F8B212386011701B
:103DB000396893F8B1024A1C01233A601A46087028
:103DC00009E73A68314B501C93F83812386011708B
:103DD0003A6893F83C12501C386011703A6893F8B6
:103DE0003B12501C386011703A6893F83D12501C19
:103DF00038601170396893F83F02DCE73968234A6C
:103E00000123481C38600B70396892F8C406CC183E
:103E10003C600870396892F8C206CC183C600870A3
:103E2000396892F8C306CA183A601A460870D2E692
:103E30003B6801241A193A601C7022F043F80028EC
:103E400041F05185194D1A4A03463968481C3860BB
:103E50000B703B6841F2B410591C105C396041F2A0
:103E60007811187051583846890A2AF017F8E96B0A
:103E7000384649082AF012F801231A46ABE600BF7B
:103E8000941A0020A01A00202C1B0020744500204A
:103E90009C1A00202C1D0020234400208C69002047
:103EA00075CD0108447B0308C84700205C7F0020D3
:103EB000784F002000780020C54E3378002B3FF467
:103EC00088AEC44C00253B6894F87C22591C3960AC
:103ED0001A7094F87D3203EB830303EB830303F240
:103EE000EE2189B2384629F0F1FF337801359D4241
:103EF00004F10204E7DB6CE63B68B64C591C94F80D
:103F0000B62239601A703B6894F8B722591C3960A0
:103F10001A70B4F8B812384629F0D8FF3B6894F804
:103F2000BA22591C39601A70B4F8BC12384629F00C
:103F3000CDFF396894F8BE023DE7A74B3846B3F889
:103F4000481029F0C3FF01231A4644E63B680024C9
:103F50005A1C3A6021461C70384629F09FFF2146C2
:103F6000384629F09BFF2146384629F097FF012368
:103F70001A4630E6002D3FF42CAE984B2B600123FF
:103F80001A4628E6934B396893F8670213E7944C76
:103F900004F1800554F8041F384629F07FFFA5423C
:103FA000F8D116E68B4C04F14005B4F8CC13384632
:103FB00029F08CFF3B6894F8CE23591C39601A70A5
:103FC0003B6894F8CF230434591CAC4239601A7012
:103FD000EBD1FEE57F4C3B6894F85C22591C3960BC
:103FE0001A70B4F86E12384629F070FFB4F86A12ED
:103FF000384629F06BFFB4F86C12384629F066FF9A
:104000003B6894F86522591C39601A70B4F878122C
:10401000384629F05BFFB4F87A12384629F056FF8B
:104020003B6894F87022591C39601A703B6894F808
:104030007222591C39601A70B4F87612384629F089
:1040400045FF3B6894F85F22591C39601A70D4F818
:104050006012384629F022FF3B6894F86422591C0C
:1040600039601A70396894F87302A4E6594B3968BC
:1040700093F8B3029FE6574C3846B4F8401229F043
:1040800025FFB4F84212384629F020FF3B6894F827
:104090004422591C39601A70B4F84612384629F087
:1040A00015FF01231A4696E54A4C3846B4F8E41148
:1040B00029F00CFFB4F8E811384629F007FFB4F8EE
:1040C000EC11384629F002FF01231A4683E5414BE3
:1040D0003846996829F0E2FE01231A467BE53D4BFC
:1040E000404D03F1500493F8E125396802EB420298
:1040F00005EB8202481C92F8382038600A703A6852
:1041000093F8E215501C386011703A6893F8E31583
:10411000501C386011703A6893F8E4150433501C51
:10412000A34238601170DED153E52F482BF0F8FC24
:10413000011E7FF74EAD2C4B19443A6813F8010B62
:10414000541C8B423C601070F7D142E5274B03F1C1
:104150000B043A6813F8011B501C9C423860117024
:10416000F7D1234B03F108013A6813F8010F541CEF
:1041700099423C601070F7D11E4BD91D3A6813F874
:10418000010F541C99423C601070F7D121E51A4B85
:10419000191D3A6813F8010B541C99423C601070C9
:1041A000F7D10021384629F091FE12E53B68032241
:1041B000591C39601A703A680123D118396013709C
:1041C00039680620CA183A601A46087003E500BF2D
:1041D0009C1C00207445002070740020610F0108B1
:1041E000BC480020E84E0308444C0020447B0308F0
:1041F0004F7B03085B7B03083C7B0308B04B191D16
:104200003A6813F8010B541C99423C601070F7D1C6
:10421000DFE43B680022591C39601A703A680123B8
:10422000D1183960137039681F20CA183A601A46CD
:104230000870D0E43A68A34B501C01213860981DE7
:1042400011703A6813F8011F541C98423C601170B9
:10425000F7D1BEE49C4E00233A683168501CC95C1B
:1042600038601170326839681A44481C927A386094
:104270000A70326839681A440133127D481C0A2BCF
:1042800038600A70E8D1A4E4904C3B682268591C5D
:10429000127839601A7023683A689978531C3B6029
:1042A00000231170226839681A4401335279481C7E
:1042B000032B38600A70F5D13B682268591C127ACA
:1042C00039601A703B682268591CD27839601A70BC
:1042D0003B682268591C127939601A702368384685
:1042E000598929F0F3FD3B682268591C527A3960DC
:1042F0001A702368396858785DE5754B3846196837
:1043000029F0CCFD734B3846198829F0DFFD0123D5
:104310001A4660E4704C3846218829F0D7FD618840
:10432000384629F0D3FDB4F904306C49DA1781FB23
:104330000313C2EBA30399B2384629F0C7FD01234A
:104340001A4648E4664E3378002B3FF442AC654D84
:10435000002435F8021F384629F0B8FD33780134BF
:104360009C42F6DB35E4604C604D04F1A00607E0AA
:10437000143429F0ABFDB44205F102053FF429AC39
:10438000237B38461946002BF2D028881EF01EFFEA
:1043900001463846ECE7564A3B6814685068916815
:1043A000D268DA601C60586099603A680123103264
:1043B0003A601A460FE44F4C2289B2F5007F04F1AF
:1043C000300594BF012604263C3455F8041B91FBAC
:1043D000F6F1384689B229F079FDA542F5D1464C6F
:1043E00004F10C06A4F14C05B4EC010AD5ED067AF3
:1043F00080EE270A2EF054F881B2384629F066FD87
:10440000A642F1D13D4C04F10C0554F8041B38468A
:1044100089B229F05BFDA542F7D1FFF7DABB384B33
:104420003846B3F8581029F051FD364B19883846F4
:1044300089B229F04BFD344B1A68C2F3C003C2F3B2
:1044400080019B0043EA4103C2F340010B43C2F3E6
:10445000401143EAC10102F010021143384629F02D
:1044600035FD0DF0C3FC0146384629F017FD3B68C9
:10447000264A581C92F8E015254A386019701188B0
:1044800064293846A8BF642129F020FD89E63B68ED
:104490001E4A581CE721386019703B6892F8B32215
:1044A000591C39601A703B680022591C3960384623
:1044B0001A70042129F0F2FC01231A46FFF78BBB86
:1044C000347B0308B349002048390020E47F0020F2
:1044D000A81C00203C1A0020601A0020676666664F
:1044E0009C1C00206A1A002000780020046D002027
:1044F0003C7E0020F8190020BC740020FC3800200D
:10450000A01000201C450020601B002074450020E6
:10451000FC3900203A68CB4B501C93F819123860D4
:1045200011703A6893F82412501C38601170396881
:1045300093F80F023FE4C44C0021384629F0C6FC32
:104540000021384629F0C2FC23683846598D29F0ED
:10455000BDFC3A680023511C396013703A68216829
:10456000501C91F83110386011703A682168501C65
:1045700091F84010386011703A682168501C91F829
:104580004110386011703A68511C396013703A68F4
:10459000511C396013703A68511C396013702368DC
:1045A00093ED120AB2EE048A20EE080A2DF078FF8D
:1045B00081B2384629F08AFC236893ED110A20EE77
:1045C000080A2DF06DFF81B2384629F07FFC3B6868
:1045D0002268591C92F8332039601A7023683968B0
:1045E00093F83400FFF7E7BB964C3B6894F8012240
:1045F000954D591C39601A702B683846198C29F072
:1046000065FC2B683846598C29F060FCB4F804121C
:10461000384629F05BFCB4F80612384629F056FCFF
:104620002B683846998C29F051FC2B683846D98C78
:1046300029F04CFCB4F80812384629F047FCB4F8CD
:104640000A12384629F042FC01231A46FFF7C3BA82
:104650007C4E96F8FF31002B01F053813B68082215
:10466000591C39601A703B680122991839601A7018
:104670003B6896F8D520591C39601A703B6896F84B
:10468000D420591C39601A70B6F8D210384629F077
:104690001DFCDFED6E7A96ED360A20EE270A2DF02E
:1046A000FFFE81B2384629F011FC396896F8030202
:1046B000FFF781BB3B68634D591C012239601A70BA
:1046C0003B6895F87C24591C39601A703B6895F852
:1046D0007A24591C39601A703B6895F87224591C69
:1046E00039601A70B5F87414384629F0EFFBB5F844
:1046F0007614384629F0EAFBB5F87814384629F0E4
:10470000E5FB05F2444405F58E6534F8021F384692
:1047100029F0DCFBAC42F8D1FFF75BBA3A68494BB1
:10472000501C93F84C12386011703A6893F84D128F
:10473000501C386011703A6893F84E12501C386063
:104740001170B3F8EE10384629F0C0FB01231A4669
:10475000FFF741BA3B4C3846B4F8E81029F0B6FBF5
:10476000B4F8EA10384629F0B1FBB4F8EC1038463A
:1047700029F0ACFB01231A46FFF72DBA314E002574
:104780003446B4F87211384629F0A0FBB4F874111D
:10479000384629F09BFBB4F87611384629F096FB91
:1047A0003B6894F87821591C39601A703B6894F87A
:1047B0007921591C39601A703B6894F87A21591C88
:1047C00039601A703A6894F87B11C5EBC503501C28
:1047D00006EB430338601170D3F87C11013538467D
:1047E00029F05CFB082D04F10E04CAD1FFF7F1B9E2
:1047F000174C2378002B3FF4ECA9DFF85CE0E61CB3
:104800000025002316F8010F124A194604E001336F
:104810001F2B10D012F80C1C884202F10C02F6D1AA
:10482000DBB203EB43033A680EEB8303511C93F8AE
:10483000383039601370237801359D42E1DBFFF792
:10484000C8B900BF74450020483900200000C842A4
:104850002C1D0020244F0308E84E0308C1495223B1
:104860003A68501C3860137011F8013F002BF7D1E3
:10487000FFF7AFB9BC4C2378002B3FF4AAA9B94E7F
:104880000125DFF818934FF00108002319F8010FF4
:10489000B64A194605E001331F2B00F0E18712F8F4
:1048A0000C1C814202F10C02F5D1DBB203EB430395
:1048B00006EB8303D3F834A050462BF031F9002DDA
:1048C00040F0CE8700280ADD53460AEB000E3A6816
:1048D00013F8011B501C734538601170F7D1237811
:1048E00043457FF776A908F10108CEE701233A682E
:1048F000511C396013700133092BF8D1FFF769B9E6
:104900009B4C3846B4F86A1229F0E0FAB4F8CC109F
:10491000384629F0DBFAB4F8CE10384629F0D6FA3A
:10492000B4F8D010384629F0D1FAB4F8B8123846A5
:1049300029F0CCFA3A688F490023501C3860137074
:104940003A68501C386013703A68501C3860137015
:104950003A6894F84502551C3D6010703A6894F826
:104960006702551C3D6010703A68501C3860137027
:10497000B4F90C3281FB0321DB17C3EBA10189B22F
:10498000384629F0A3FA3B6894F83822591C39605C
:104990001A703B6894F83C22591C39601A703B68C5
:1049A00094F83B22591C39601A70396894F83D021A
:1049B000FFF701BA704B3846196829F06FFA6F4B50
:1049C0003846196829F06AFA6D4B3846196829F09B
:1049D00065FA01231A46FFF7FEB86A4B3846B3F86A
:1049E000581029F073FA684B1988384689B229F0B3
:1049F0006DFA664B1A68C2F3C003C2F380019B00D4
:104A000043EA4103C2F340010B43C2F3401143EABE
:104A1000C10102F010021143384629F057FA0DF097
:104A2000E5F90146384629F039FA3B68504A581CE6
:104A300092F8E015564A3860197011886429384692
:104A4000A8BF642129F042FA3B68524A581C03214E
:104A50003860197039681078FFF7ADB9DFF840E1B8
:104A60000025EEB2714600233A68501C386016707B
:104A70003A68501C386013703A6811F8010F01331E
:104A8000541C062B3C601070EED10135062D0EF142
:104A9000060EE6D1404900233A68501C3860157074
:104AA0003A68501C386013703A6811F8010F0133EE
:104AB000541C0B2B3C601070EED13B682C4A581CE8
:104AC0000721386019703B680021581C3860197044
:104AD000396892F83C04FFF76EB93A68244B501CD1
:104AE00093F8FC11386011703A6893F81812501C52
:104AF00038601170396893F80E02FFF75CB91C4BEF
:104B000003F170043A6893F80211501C3860117078
:104B10003A6893F80311501C386011703A6893F8A2
:104B20000411501C386011703A6893F80511501C3C
:104B3000386011703A6893F80611501C3860117093
:104B40003A6893F80711501C386011703A6893F86E
:104B500008110733501C9C4238601170D2D1FFF706
:104B600038B800BFE84E03082C1D0020244F03086E
:104B70007445002067666666ACF7FF1FB0F7FF1F3D
:104B8000B4F7FF1FA01000201C450020601B002070
:104B9000FC390020E17F0020A34900202F1D0020C8
:104BA0007F490020C94C3846B4F8221229F08EF90A
:104BB000B4F82012384629F089F901231A46FFF784
:104BC0000AB8C34C04F1080534F8021B384629F032
:104BD0007DF9A542F8D1FEF7FCBFBC4B03F15A04A6
:104BE0003A6893F83616501C386011703A6893F89A
:104BF0003116501C386011703A6893F83216501C08
:104C0000386011703A6893F83316501C3860117090
:104C10003A6893F83416501C386011703A6893F86B
:104C200035160633501C9C4238601170D8D1FEF7FF
:104C3000D0BFA84AA2FB0512A91A02EB51029208A2
:104C4000C2EBC2016D1A30D1D2B202F1FF385FFA65
:104C500088F8002A3EF4BDAF08F101081AE080F898
:104C60000290204629F008F9226830801346511C32
:104C7000216013F8021BF170236053783371D31C49
:104C800023609378B371131D2360D2787271A845A5
:104C90003EF49FAF5A1C226093F90090484617F0EB
:104CA000B3FD013506460028D9D14FF0FF331A462F
:104CB000FEF791BF4A46FEF7E4BF8749102D4FF03B
:104CC00000022B4628BF10230A604A608A60CA602F
:104CD0000A74002B3EF47DAF226813440132226037
:104CE00012F8010C01F8010B9342F7D1FEF771BFE6
:104CF0005A1C226018781328D7D89A1C22600022E8
:104D00005E787649154604E001321F2ACDD011F8AD
:104D10000C5CB54201F10C01F6D1D2B2704D6B4979
:104D2000704E02EB420205EB820500F5BC7001EB10
:104D3000800295F830105170D91C216099789170DB
:104D4000191D2160D978D170591D21601B793068F7
:104D5000137119F0E1F9FEF73CBF5C4B00229A6039
:104D6000204629F071F809F071FB01231A46FEF77D
:104D700032BF204629F080F8544DC5F8E4012046A2
:104D800029F07AF8C5F8E801204629F075F80123E2
:104D9000C5F8EC011A46FEF71EBF204629F06CF854
:104DA0004A4DA5F84002204629F066F82368A5F888
:104DB00042025A1C22601B7885F84432204629F0B2
:104DC0005BF80123A5F846021A46FEF704BF5A1CF9
:104DD00022603E4A1B7882F8B33201231A46FEF75E
:104DE000FABE5A1C2260394E1B7886F85C32204687
:104DF00029F042F8A6F86E02204629F03DF8A6F800
:104E00006A02204629F038F82368A6F86C025A1C7A
:104E100022601B7886F86532082D7EF6DAAE2046D1
:104E200029F02AF8A6F87802204629F025F80C2D5A
:104E3000A6F87A027EF6CDAE23681A46591C216088
:104E400012F8021B86F8701222605B7886F87232C4
:104E5000204629F011F8102DA6F876027EF6B9AE9C
:104E600023685A1C22601B7886F85F32204628F09F
:104E7000EBFF2368C6F860025A1C22601A7886F895
:104E80006422162D7EF6A5AE9A1C22605B7886F809
:104E9000733201231A46FEF79EBE0C4D05F1400603
:104EA000204628F0E9FF2368A5F8CC03591C1A46D0
:104EB000216012F8021B85F8CE1322605B7885F81A
:104EC000CF330435AE42EBD1FEF783BE74450020EC
:104ED0003C7F002025499224444C00202C4F03089D
:104EE000E84E0308483900205A1C22601E781F2E05
:104EF0003FF6DBAE052D7FF4D8AE204628F0A4FFA8
:104F0000C44B03EB8603C3F84C031AF047FBFEF7D0
:104F100060BE5A1C2260BF4A1B7882F867320123A8
:104F20001A46FEF758BE5A1C22601A780E2A3FF61F
:104F3000BCAE991C2160597803293FF6B6AEB5483E
:104F400002EB420200EB4202D81C82F836162060C7
:104F5000997882F83116191D2160D97882F83216B5
:104F6000591D2160197982F83316991D21605979EC
:104F700082F83416D91D21609B7982F835360123D9
:104F80001A46FEF728BE19465A1C2260A14A11F89B
:104F9000020B82F838022160597882F83C12D91C41
:104FA0002160997882F83B12191D2160D97882F826
:104FB0003D12042D7EF60DAE591D21601B7982F83D
:104FC0003F3201231A46FEF706BE1A46591C2160DD
:104FD000904912F8020B81F8B20222605B7881F8E6
:104FE000B13201231A46FEF7F6BD8B4A03F10801E0
:104FF0000133236013F8010C02F8010B9942F7D139
:10500000FEF7E7BD854B1B785B073FF54EAE09F019
:10501000C3FB09F053FA01231A46FEF7DCBD204614
:1050200028F02AFF7B4DA5F82202204628F024FF15
:105030000123A5F820021A46FEF7CDBD5A1C2260B6
:1050400019780F293FF631AE724A981CC1EBC101A5
:1050500020600A44597882F80211D91C216099789D
:1050600082F80311191D2160D97882F80411591DA5
:105070002160197982F80511991D2160597982F80A
:105080000611D91D2160997982F8071103F10801F1
:105090002160DB7982F808311DF008FC01231A46F3
:1050A000FEF799BD1A46591C21605A4D12F8021B91
:1050B00085F84C1222605A7885F84D22DA1C22605D
:1050C0009B7885F84E32204628F0D6FE0123A5F8BD
:1050D000EE001A46FEF77FBD514B186809F0BAFE84
:1050E00001231A46FEF777BD19465A1C2260494A29
:1050F00011F8020B82F8FC012160597882F818122D
:10510000D91C21609B7882F80E3201231A46FEF7E3
:1051100062BD1A46591C216012F8020B2260DA1C8B
:10512000597822609A7806F0C5FB00287EF451ADCC
:10513000BBE53A4B1B785A073EF54BAD39490A7827
:10514000012342F004020A701A46FEF744BD2046CD
:1051500028F092FE2F4DA5F86A02204628F08CFE1A
:10516000A5F8CC00204628F087FEA5F8CE00204602
:1051700028F082FEA5F8D000204628F07DFEA5F894
:10518000B802204628F084FE204628F081FE204602
:1051900028F07EFE23681A46591C216012F8021B73
:1051A00085F8451222605B7885F86732204628F042
:1051B0006FFE204628F060FE236800EB80001A4650
:1051C0004100581CA5F80C12206012F8021B85F84B
:1051D000381222605A7885F83C22DA1C22609A78CC
:1051E00085F83B221A1D2260DB7885F83D320123C9
:1051F0001A46FEF7F0BC094B1B7858073EF5E9ACA0
:105200000AF02EFA09F0C8FA09F058F901231A46F3
:10521000FEF7E1BC74450020C8470020744F002011
:10522000483900202E1B00205A1C226018780506E1
:1052300000F18D83A14B1B785C073EF5CAAC0328B7
:1052400028BF002009F022FD01231A46FEF7C3BC47
:10525000204628F011FE9A4A012310801A46FEF7D4
:10526000BABC984D05F11006204628F005FE1DF049
:10527000DBFF25F8020FAE42F6D1FEF7AABC2046AE
:1052800028F0FAFD904DA5F8E800204628F0F4FD3E
:10529000A5F8EA00204628F0EFFD0123A5F8EC0070
:1052A0001A46FEF798BC0F2D7FF4FFAC5A1C226003
:1052B0001E78072E3FF6F9AC2046834D28F0DCFD22
:1052C000C6EBC60605EB4605A5F87201204628F098
:1052D000D3FDA5F87401204628F0CEFD2368A5F87B
:1052E00076011A46591C216012F8021B85F87811C4
:1052F00022605A7885F87921DA1C22609A7885F83C
:105300007A211A1D2260DB7885F87B31204628F04F
:105310009BFD0123C5F87C011A46FEF75CBC5A1CB4
:10532000694D22601B7885F8B3320023AB602046BC
:1053300028F08AFD09F08AF823685A1C22601B783D
:1053400085F85C32204628F097FDC5F8E401204638
:1053500028F092FDC5F8E801204628F08DFDC5F83B
:10536000EC01204628F088FDA5F84002204628F0F0
:1053700083FD0123A5F842021A46FEF72CBC204605
:1053800028F07AFD01231A46FEF725BC1A46591C5F
:1053900021604D4D12F8021B85F8B61222605B7831
:1053A00085F8B732204628F067FD2368A5F8B802D3
:1053B0005A1C22601B7885F8BA32204628F05CFD22
:1053C0002368A5F8BC025A1C22601B7885F8BE32FF
:1053D00001231A46FEF7FFBB5A1C22601A78112AD5
:1053E0003FF663AC384D02F59E72991C05EB420501
:1053F00021605B782B71204628F03EFD40F6CA0301
:105400009842A8BF184640F2EE239842B8BF18460B
:105410002E4AA0F2EE2082FB0032C017C0EBE2025F
:1054200001236A711A46FEF7D6BB294A1278012A6F
:105430003EF6CFAB19465A1C2260234A11F8020BE4
:1054400082F8C4062160597882F8C216D91C2160FE
:105450009B7882F8C33601231A46FEF7BCBB062DA3
:105460007FF423AC1B4A991D0133236013F8010C10
:1054700002F8010F9942F7D1174B93F82430002B13
:105480003EF4A7AB18F070FC01231A46FEF7A3BB4D
:105490005A1C22601D78FF2D00F0A082204628F0C3
:1054A000EBFC152D3EF695AB074A02EB45020123B6
:1054B000A2F846041A46FEF78EBB00BF744F0020C8
:1054C000DA2C002022730020744500201F85EB5148
:1054D00048680020B34900202C1D00205A1C22607F
:1054E00013F8376B0DF1FF310132226012F8010C15
:1054F00001F8010F9342F7D1D04C94F82530002BDE
:10550000FBD194F82650002DFDD1DFF848A3DFF839
:105510004893DAF800004FF0010884F8268008F07C
:10552000CDFC284684F8278018F0DCFB284618F0CC
:10553000D9FB092018F0D6FB304618F0D3FB6E4695
:105540006D460DF13608A5EB060B5FFA8BFB0A20C2
:1055500018F0C8FB584618F0C5FB15F801BB0B2026
:1055600018F0C0FB584618F0BDFBD9F8003033B135
:105570001A689B88918A0B4218BF1B049361A84547
:10558000E1D1082018F0AEFBA02018F0ABFBA02062
:1055900018F0A8FB002018F0A5FB10F02005F6D1AC
:1055A000DAF8000008F090FC012384F826501A462F
:1055B000FEF711BB1A46591C2160A14E12F8021BBE
:1055C00086F8FE1122605A7886F8F821DA1C2260EB
:1055D0009A7886F8D5201A1D2260DB78082BA8BFA0
:1055E0000823204686F8D43028F046FC072DA6F87C
:1055F000D20000F2E581236862689A4207D05A1C03
:1056000022601B78003318BF012386F8033209F0AB
:105610005BFB01231A46FEF7DEBA5A1C2260894E54
:10562000DFF81C821B78D6F8009088F801322046FB
:1056300028F022FCA9F820002046D6F8009028F097
:105640001BFC052DA9F8220000F2948109F03CFB17
:1056500014F05CFC30681DF025FC01231A46FEF7AF
:10566000BABA204628F008FC764E9FED778A20468D
:1056700028F002FC2046D6F8008028F0FDFBA8F8B0
:105680002A00204628F004FC236832681946581C7A
:10569000206011F8020B82F831002160597882F8FD
:1056A0004010D91C21609B7882F84130204628F0B8
:1056B000EFFB204628F0ECFB204628F0E9FB2046D3
:1056C000D6F8009028F0D8FB07EE900AF8EEE77ABB
:1056D000204667EE887AD6F80080C9ED127A28F065
:1056E000CBFB07EE900AF8EEE77A112D67EE887A89
:1056F000C8ED117A00F2E98030681DF0EFFA01235D
:105700001A46FEF768BAC5F34705122D3FF6CDAA33
:10571000002D00F02D8105F10043013BE9460DEB22
:105720004308ADF10206204628F0A6FB26F8020F3A
:105730004645F8D1294648461CF0B8F801231A46D8
:10574000FEF749BA19465A1C22603D4A11F8020B6D
:1057500082F819022160597882F82412D91C21603C
:105760009B7882F80F3201231A46FEF734BA092DCE
:105770007FF69BAADFF8E4801A46591CD8F800602F
:10578000216012F8021B317022605A78B270DA1C64
:1057900022609A78642A03F10401A8BF642272711E
:1057A0002160DA78642A03F10501A8BF6422B2718E
:1057B00021601A79F2719A1D22605A79642A28BFF1
:1057C0006422D91D327221609A79F27003F10802C5
:1057D0002260DB793371204628F04EFB0A2D708160
:1057E00040F0A6800CF090FB01231A46FEF7F3B9B7
:1057F000164B1B7859073EF5ECA9154A4FF4C871B2
:10580000012311801A46FEF7E6B90E4A1068DA1C29
:10581000411E2133951E256012F8035C01F8015FDB
:10582000551E256012F8025C8D72226012F8015C30
:105830000D7503329342EDD15FE700BF2C1D0020B0
:105840007445002048390020CDCCCC3D744F002059
:10585000F47F00201C91002020450020E47F0020E0
:1058600023789845FFF63FA8002D3EF4B2A9002505
:10587000002B7FF406A8FEF7ACB9531C1146236039
:10588000684811F8023B80F822302160527880F895
:105890002320042B06D9FF2B3EF4ADA93968002044
:1058A000FEF789BA0B2A03D9022BF7D1FF2AF5D1CB
:1058B0003A680123D11839601370002D3EF489A98C
:1058C000594A2A601A46FEF786B923683068591C7F
:1058D0001A46216012F8021B80F8331022605B78B0
:1058E00080F8343009E7514D514A95F82430B3B966
:1058F0002346FEF7AABA4F4B196801F30F01FEF7D2
:1059000064B93B6896F8FE21591C39601A703B68EF
:1059100096F8F821591C39601A70FEF7A9BE517823
:1059200002291FD003290CBF04232346FEF78DBA9A
:105930002368D8F80020591C2160197851720B2D6A
:105940003FF450AF991C21605B7853704AE700F038
:105950007F00032828BF002009F076F901231A46AA
:10596000FEF739B9042B34BF02230323FEF76DBAC7
:10597000E946DFE6204628F07FFAA8F80402204630
:1059800028F07AFAA8F806022046D6F8009028F007
:1059900073FAA9F824002046D6F8009028F06CFA93
:1059A0000D2DA9F826007FF651AE204628F064FAA6
:1059B000A8F80802204628F05FFAA8F80A0245E68F
:1059C000204628F059FA07EE900A9FED1B7AF8EE70
:1059D000E77A67EE877AC6ED367A0CE69A1C226083
:1059E000164D5A7885F87C24DA1C22609A7885F85E
:1059F0007A241A1D2260DB7885F87234204628F05C
:105A00003BFAA5F87404204628F036FAA5F8760487
:105A1000204628F031FA0123A5F878041A46FEF74B
:105A2000DAB800BF2C1D0020790F01085C7F002030
:105A3000784F00209C1A00200AD7233C7445002090
:105A400010B51A4B93F8C436022B82B006D0184B0F
:105A5000186803681B68984702B010BD154B8DF895
:105A6000071018680A4690F91A104B1C0FD04368AB
:105A700040F2FF14C3F30803A34208D003EB412311
:105A80000D495A5443680133436002B010BD037E90
:105A900013F0060FE0D090F82830002BDCD1012263
:105AA0000DF1070115F0F4FDD6E700BF74450020A5
:105AB0002C87002014870020904F002010B51A4B2F
:105AC00093F8C436022B82B0014606D0174B1868F3
:105AD00003681B68984702B010BD154B8DF807008E
:105AE000186890F91A20531C0FD0436840F2FF1435
:105AF000C3F30803A34208D003EB42230D4A995491
:105B000043680133436002B010BD037E13F0060FFB
:105B1000E1D090F82830002BDDD101220DF10701F2
:105B200015F0B6FDD7E700BF744500202C87002094
:105B300014870020904F00202DE9F04FBA4F3B888A
:105B400093B00546002B00F0BF80B84AD7F88831E3
:105B50001468A34207D0B64BC7F888411B78093BAD
:105B6000012B40F21684B34BD7F88C611C68B44209
:105B700007D0AF4BC7F88C411B78093B012B40F293
:105B8000FA83AD4C3B8894F8C21694F8C3060B44D4
:105B9000013BB3FBF0F200FB1233994202D813B081
:105BA000BDE8F08F012026F011FA284625F096FB7B
:105BB000A24B0293194694F8C4360A680392022B4A
:105BC0004A68019200F0BD839D4B1868036850211C
:105BD0001B689847029A136852680299126888688D
:105BE00019680368DFF86092954D964E0B44A3EB5D
:105BF0004203D81780EA430006F0D0FE03990198CB
:105C00004B6842689B1A0A9382688B689B1A0B93B5
:105C1000CB68C2680DF1280A9B1A0C93D04658F83D
:105C2000043B4FEAE37B8BEA430BBBF17F0F94F815
:105C3000C4360CD8C4E3286803681B68984794F8F6
:105C4000C4364FEADB1BBBF17F0F40F2B9836BF028
:105C50007F01022BC9B2EED1306840F2FF1E90F9ED
:105C60001A308DF81F105A1C1AD04268C2F308026D
:105C7000724502EB432313D003F8091043684FEA3F
:105C8000DB1B0133BBF17F0F43606BF07F0140F200
:105C9000418590F91A30C9B25A1C8DF81F10E4D111
:105CA000037E13F0060F04D090F82830002B00F08C
:105CB00028854FEADB1BBBF17F0F6BF07F0140F2C1
:105CC0002985C9B23068CAE75B4C5C4BB4F8C206A0
:105CD00002931E4642F20103C01AB0FA80F0400956
:105CE00026F074F9284625F0F9FA94F8C436D6F867
:105CF0000080022B00F07786514B18680368492119
:105D00001B6898477868DFF840B14D4D4D4E06F05E
:105D100045FED8F8000006F041FE08F10C038DE8BE
:105D2000080194F8C426C24699465AF8043FD91788
:105D300081EA4308B8F17F0F0BD851E02868036867
:105D40004FEAD8181B689847B8F17F0F94F8C4261B
:105D500046D968F07F01022AC9B2EFD1306840F21B
:105D6000FF1E90F91A308DF817105A1C1AD042688D
:105D7000C2F30802724502EB432313D003F80B1061
:105D800043684FEAD8180133B8F17F0F436068F0D9
:105D90007F0140F25E8190F91A30C9B25A1C8DF829
:105DA0001710E4D1037E13F0060F02D090F82830CC
:105DB00053B14FEAD818B8F17F0F68F07F0140F275
:105DC0004881C9B23068CCE701220DF117014FEAD2
:105DD000D81815F05DFCB8F17F0F94F8C426B8D838
:105DE000022A5FFA88F100F03681286803681B6890
:105DF000984794F8C426CA4597D1DDF80480DFF8A7
:105E000048A00F4D0F4EDDF80090CDF8008008F14E
:105E100018039B4659F8041FCB1783EA4108B8F1D1
:105E20007F0F1ED856E000BF541D002024440020E0
:105E300048680020681A0020744500200887002068
:105E40002C87002014870020904F002028680368CA
:105E50001B68984794F8C4264FEAD818B8F17F0F0A
:105E600038D968F07F01022AC9B2EFD1306840F218
:105E7000FF1E90F91A308DF819105A1C19D042687B
:105E8000C2F30802724502EB432312D003F80A1052
:105E900043684FEAD8180133B8F17F0F436068F0C8
:105EA0007F012CD990F91A30C9B25A1C8DF81910FB
:105EB000E5D1037E13F0060F02D090F82830B3B17D
:105EC0004FEAD818B8F17F0F68F07F0117D9C9B22F
:105ED0003068CEE7022A5FFA88F112D0286803689A
:105EE0001B689847CB4526D094F8C42692E7012238
:105EF0000DF1190115F0CCFB94F8C426ACE75FFA5C
:105F000088F130688DF81A1090F91A20531C00F0AF
:105F1000E780436840F2FF1EC3F30803734500F0B7
:105F2000DF8003EB4223CB4503F80A10436803F1FB
:105F300001034360D8D1BB68DDF80080DD0300F1C8
:105F4000B985980300F1A285590300F1AA8508F1EB
:105F5000280026F087F9B4F8CC30B8F92E00C01A22
:105F600006F01CFDBB68DA0400F1BC859E0400F15C
:105F7000B2855D0500F1A885180500F1808519043A
:105F800000F1778508F1300026F06CF908F1360051
:105F900026F068F9DFF82CA3C34DC44ECDF800807D
:105FA00008F1420308F13A099B4639F9021F94F8B7
:105FB000C426CB1783EA4108B8F17F0F0CD89FE0C5
:105FC000286803681B68984794F8C4264FEAD818D5
:105FD000B8F17F0F40F2948068F07F01022AC9B2C5
:105FE000EED1306840F2FF1E90F91A308DF81B1088
:105FF0005A1C1AD04268C2F30802724502EB4323CE
:1060000013D003F80A1043684FEAD8180133B8F1E7
:106010007F0F436068F07F0140F2568190F91A309B
:10602000C9B25A1C8DF81B10E4D1037E13F0060F81
:1060300004D090F82830002B00F015814FEAD818D2
:10604000B8F17F0F68F07F0140F23E81C9B230683D
:10605000CAE75FFA88F1306840F2FF1E90F91A2013
:106060008DF81810531C21D04368C3F308037345FF
:106070001CD003EB4223CA4503F80B10436803F11D
:106080000103436000F0CA845AF8043F590081EAD2
:10609000E3717F2988464FF002023FF65AAE90F92D
:1060A0001A20C9B2531C8DF81810DDD1037E13F0ED
:1060B000060F04D090F82830002B00F03B81CA4531
:1060C00000F0AC845AF8043F590081EAE3717F295B
:1060D00088464FF002023FF63CAEC9B23068BDE7D9
:1060E000037E13F0060F3FF4FDAE90F82830002B2E
:1060F0007FF4F8AE01220DF11A0115F0C9FAF1E6AC
:10610000022A5FFA88F100F0E180286803681B68C2
:106110009847CB457FF449AFDDF80080644BB8F970
:1061200044001B88C01A06F039FC624B1B78012B17
:1061300067DD213308EB4303DFF888A15A4D5B4E3E
:10614000009308F1440939F9023FB8F9441094F872
:10615000C426591ACB1783EA410BBBF17F0F0BD82A
:1061600044E0286803681B68984794F8C4264FEAFF
:10617000DB1BBBF17F0F39D96BF07F01022AC9B25B
:10618000EFD1306840F2FF1E90F91A308DF81D10E3
:106190005A1C19D04268C2F30802724502EB43232D
:1061A00012D003F80A1043684FEADB1B0133BBF13E
:1061B0007F0F43606BF07F015DD990F91A30C9B24F
:1061C0005A1C8DF81D10E5D1037E13F0060F03D085
:1061D00090F82830002B3ED04FEADB1BBBF17F0F3D
:1061E0006BF07F0147D9C9B23068CDE7022A5FFA68
:1061F0008BF142D0286803681B689847009B99453B
:10620000A1D1BB68990508D5B8F96630A3F2DC5373
:10621000D81780EA430006F0C1FB029D2649286892
:10622000264B274A6860441AA41003FB04F3013389
:1062300082FB0342A2EBE37202EB42029B1AC3EB26
:10624000431301EB83030122A8602B6087F88421AC
:1062500013B0BDE8F08F01220DF11D0115F018FA01
:1062600094F8C42683E701220DF11B0115F010FA02
:1062700094F8C426AAE65FFA8BF130688DF82810EE
:1062800090F91A20531C37D0436840F2FF1EC3F325
:106290000803734530D003EB422303F80A10436828
:1062A00001334360AAE700BF2C8700201487002039
:1062B0004672002058720020641D0020DF7BEFBD75
:1062C00056555555904F00205FFA88F130688DF88B
:1062D0001C1090F91A20531C1DD0436840F2FF1E79
:1062E000C3F30803734516D003EB422303F80A10E7
:1062F0004368013343600CE7037E13F0060F3FF45D
:106300007DAF90F82830002B7FF478AF01220AA9E6
:1063100015F0BEF972E7037E13F0060F3FF4F9AEF5
:1063200090F82830002B7FF4F4AE012207A915F075
:10633000AFF9EEE6012206A915F0AAF994F8C426F1
:1063400059E5AD4B186890F91A1050224D1C8DF884
:106350001E2029D0436840F2FF15C3F30803AB4267
:1063600022D003EB4123A5495A544368019A0133D3
:106370004360039B31E44520FFF7A0FB1E20FFF79D
:106380009DFB204606F00AFB304606F007FBFFF7B0
:10639000F8BB4520FFF792FB0020FFF78FFB20465C
:1063A00006F0FCFAFFF7DFBB037E13F0060F04D004
:1063B00090F82830002B00F07284019A039B0CE4C3
:1063C000022B5FFA8BF100F0A781286803681B6835
:1063D00098470DAB43457FF422AC0399019D0B69AF
:1063E0002A699B1A0A936A694B699B1A0B938B69FA
:1063F000AA690AA89B1A0C9306F05EF9BB68DE0333
:1064000000F1BF839D0300F1B083580300F1E683E0
:106410000398019EB0F92820B6F92830D21A0A92C2
:10642000B0F92A10B6F92A30C91A0B91B6F92C30F6
:106430000546B0F92C00C01A0C90B5F92E30B6F90B
:106440002E505B1B0D9353B103F108050F2D40F245
:10645000D0838033B3F5807F34BF022303239B00B6
:1064600058B100F108050F2D40F2C5838030FF2898
:106470008CBF43F0030343F002039B00DBB259B12E
:1064800001F108000F2840F2B9838031FF298CBF49
:1064900043F0030343F002039B00DDB232B102F18B
:1064A00008030F2B00F2AD8345F0010594F8C436C4
:1064B000022B00F02283524B1868036829461B68A0
:1064C00098474FF0000BD8460DF138090AAE05F099
:1064D0000303022B00F05A81032B00F04C81012BA7
:1064E00000F03F810436B1454FEA9505EFD1B8F190
:1064F000000F40F0A583BB6813F4805500F0AB8219
:10650000039A0199B2F86C20B1F86C10521A0A92F1
:106510000221012598040CD50198039AB0F86E6009
:10652000B2F86E2012A800EB8500921B0D4640F8D1
:10653000202C590521D5039E0199B6F97420B1F993
:1065400074000DF1480E0EEB8501121A41F8202C53
:106550000199B6F97620B1F976000EEB8501121A91
:1065600041F81C2C0199B6F97820B1F978000EEBAE
:106570008501121A41F8182C03351A0540F164827E
:10658000039A0199126F096F12A800EB8500521A45
:106590001B0440F8202C05F101050CD5019A039B42
:1065A000B2F87A10B3F87A3012AA02EB85025B1ABD
:1065B00042F8203C0135012D00F06A830AAB03EB61
:1065C000850200216B1E52F8040D49000028C9B253
:1065D00003F1FF3318BF41F00101581CF3D194F8C7
:1065E000C436022B00F0D982054B186803681B687B
:1065F0009847002608E000BF14870020904F002035
:106600002C870020AE420BDA5AF8043B0136002BEF
:10661000F8D0D81780EA430006F0C0F9AE42F3DBA9
:10662000302025F07BFD362025F078FD0298BF4D07
:10663000436881680268BE4E03F13A084233009312
:1066400001F13A0A02F13A0938F9022F3AF9021F28
:1066500039F9023F0A4402EBD272A3EB6202D3176C
:1066600083EA420BBBF17F0F94F8C4260CD89DE05F
:10667000286803681B68984794F8C4264FEADB1B18
:10668000BBF17F0F40F292806BF07F01022AC9B20A
:10669000EED1306840F2FF1E90F91A308DF82410C8
:1066A0005A1C1AD04268C2F30802724502EB432317
:1066B00013D0A04A995443684FEADB1B0133BBF166
:1066C0007F0F43606BF07F0140F23E8190F91A30FA
:1066D000C9B25A1C8DF82410E4D1037E13F0060FC2
:1066E00004D090F82830002B00F019814FEADB1B12
:1066F000BBF17F0F6BF07F0140F22681C9B2306899
:10670000CAE701220DF11F0114F0C2FF94F8C4364C
:10671000FFF797BA5FFA8BF130688DF8201090F987
:106720001A20531C0ED0436840F2FF1EC3F3080327
:10673000734507D003EB422303F809104368013384
:10674000436046E6037E13F0060F3FF442AE90F836
:106750002830002B7FF43DAE012208A914F098FFE9
:1067600037E6B8F1000F40F02F82326812019846E8
:106770005FFA82FBB6E6B8F1000F40F05481707802
:10678000FFF79CF93078FFF799F9ABE6B8F1000F05
:1067900040F0638194F8C4363178022B00F03982DE
:1067A000624B186803681B6898479BE6022A5FFAE9
:1067B0008BF100F0CB80286803681B689847009B2A
:1067C00043457FF441AF5C4B029D1B7829686A68A2
:1067D000A868002B70D0213302EB4303534D544E75
:1067E000009302F1420800F1420A01F1420938F92E
:1067F000022F3AF9021F39F9023F0A4402EBD27222
:10680000A3EB6202D31783EA420BBBF17F0F94F82C
:10681000C4260BD845E0286803681B68984794F89D
:10682000C4264FEADB1BBBF17F0F3AD96BF07F0127
:10683000022AC9B2EFD1306840F2FF1E90F91A3037
:106840008DF826105A1C1AD04268C2F3080272450D
:1068500002EB432313D0374A995443684FEADB1BBA
:106860000133BBF17F0F43606BF07F0140F2848006
:1068700090F91A30C9B25A1C8DF82610E4D1037E63
:1068800013F0060F03D090F82830002B3FD04FEACA
:10689000DB1BBBF17F0F6BF07F016DD9C9B2306894
:1068A000CCE7022A5FFA8BF168D0286803681B687E
:1068B0009847009B98459AD1BB68990508D5039BDA
:1068C000B3F96600019BB3F96630C01A05F0D0FF3A
:1068D000029E1A4930687468B460194B194A706096
:1068E000441AA41003FB04F3013382FB0342A2EB1E
:1068F000E37202EB42029B1AC3EB431301EB8303E7
:106900000122336087F8842113B0BDE8F08F0122A3
:106910000DF1260114F0BCFE94F8C42681E7012293
:1069200009A914F0B5FE94F8C426A7E62C87002028
:1069300014870020904F002058720020641D002012
:10694000DF7BEFBD565555555FFA8BF130688DF8FA
:10695000251090F91A20531C35D0436840F2FF1ED1
:10696000C3F3080373452ED003EB4223BE4A995468
:1069700043680133436022E75FFA8BF130688DF89A
:10698000271090F91A20531C0ED0436840F2FF1EC6
:10699000C3F30803734507D003EB4223B24A99546B
:1069A00043680133436084E7037E13F0060F80D011
:1069B00090F82830002B7FF47CAF01220DF12701E5
:1069C00014F066FE75E7037E13F0060F3FF4F7AE92
:1069D00090F82830002B7FF4F2AE01220DF1250152
:1069E00014F056FEEBE6A14B186890F91A104922F4
:1069F0004D1C8DF8162000F0A780436840F2FF156B
:106A0000C3F30803AB4200F09F8003EB4123964998
:106A10005A54436801334360FFF774B9DDF80480CA
:106A20000222FFF7ECB93368C3F3033343EA0B00E8
:106A3000FFF744F83068C0F30710FFF73FF83368FA
:106A40001B015FFA83FB4DE51E043FF5A7AD002D4A
:106A50003FF4E6ADAFE501215CE53368C3F3031312
:106A600043EA0B00FFF72AF833681B015FFA83FB48
:106A700038E5B8F87A0005F091FFFFF783BAD8F847
:106A8000700005F0F5FEBB68FFF779BAD8F8203042
:106A9000580080EAE37005F081FFBB6859037FF579
:106AA00056AAD8F82430D81780EA430005F076FFBC
:106AB000FFF74DBAD8F81C30580080EAE37005F0B3
:106AC0006DFFBB68FFF73DBA08F1740025F0CAFB03
:106AD000BB68FFF751BAB8F86E0005F05FFFBB68FE
:106AE000FFF747BAB8F86C30B889C01AC0F30D0088
:106AF00005F054FFBB68FFF739BA5C4B8DF82150A5
:106B0000186890F91A20511C0ED0436840F2FF110A
:106B1000C3F308038B4207D003EB4223524A9D5430
:106B2000436801334360CCE4037E13F0060F3FF467
:106B3000C8AC90F82830002B7FF4C3AC01220DF1D3
:106B4000210114F0A5FDBCE4037E13F0060F3FF411
:106B5000D9A890F82830002B7FF4D4A801220DF199
:106B6000160114F095FDFFF7CDB8039B019A1B6A3F
:106B7000126A9B1A580080EAE37005F00FFFBB68A9
:106B800043E4039B019ADB69D2699B1A580080EAAF
:106B9000E37005F003FFBB6834E4344B8DF8231039
:106BA000186890F91A20561C4ED0436840F2FF1620
:106BB000C3F30803B34247D003EB42232A4A995454
:106BC00043680133436014E5336803F00F0343EA7D
:106BD0000B00FEF773FF4FF0000883E4039B019A5C
:106BE0005B6A526A9B1AD81780EA430005F0D6FE0A
:106BF0000EE4012333E443F001033EE443F00103D8
:106C00004AE48032FF2A94BF45F0020545F00305AF
:106C10004CE4164B8DF82210186890F91A20531C7A
:106C200026D0436840F2FF1EC3F3080373451FD00C
:106C300003EB42230C4A995443680133436051E407
:106C40005846FEF73BFF56E4037E13F0060F3FF471
:106C5000D0AC90F82830002B7FF4CBAC01220DF1A2
:106C6000230114F015FDC4E4904F00201487002088
:106C7000037E13F0060F3FF435AC90F82830002B5C
:106C80007FF430AC01220DF1220114F001FD29E462
:106C90000A9BD81780EA430005F080FEC0E4012279
:106CA0000DF11E0114F0F4FC029A13685268FEF70D
:106CB00094BF00BF2DE9F04FAE4DAF4C2B78DA1EDC
:106CC000052A8DB0064640F2B880023B092B25D834
:106CD000DFE813F01901C301F801240024001502B4
:106CE0002B0236022B016201A44F7B78032B15D1B6
:106CF00041F2A4020123BA5C3375002A01F001813C
:106D000041F2E802BA5C002A01F0FC8041F22C1347
:106D1000FB5C002B01F0A6810023337594F8C42698
:106D2000022A11D1954A41F2B513D35C5BB1944F5D
:106D300097F8A13101222A7013B1002387F8A131FD
:106D40000DB0BDE8F08F022294F8C536002BF7D0C5
:106D50008C4B196811F4805100F0F982B4F8EC10F2
:106D60008948B0F90430B0F90270B0F906608F427A
:106D700008BF8B4214BF01230023B0F908708E4274
:106D800018BF43F00103B0F90A608F4218BF43F007
:106D90000103B0F90C708E4218BF43F00103B0F943
:106DA0000E608F4218BF43F00103B0F910708E429D
:106DB00018BF43F00103B0F912608F4218BF43F0CF
:106DC0000103B0F914708E4218BF43F00103B0F90B
:106DD00016608F4218BF43F001038E4218BF43F084
:106DE0000103002B40F0E881B0F900308B4240F005
:106DF000E381664E624F3368D7F8A411994200F2DE
:106E0000E3812B78012B9BD097F8A121002A97D002
:106E10000B2B0CD801229A4040F603010A428CD178
:106E200012F4C06F03D0093B012B41F2B3803368E9
:106E3000C7F898310B232B707FE794F8C426002AFB
:106E400000F0A181022A40F00C824C4F41F227024F
:106E5000BA5CD00740F18582002241F23701795CAB
:106E6000C90706D441F23601795C012998BF02F5C1
:106E7000007241F24701795CC80706D441F246012D
:106E8000795C012998BF02F5007241F25701795CE3
:106E9000C90706D441F25601795C012998BF02F571
:106EA000007241F26701795CC80706D441F26601BD
:106EB000795C012998BF02F5007241F27701795C93
:106EC000C90706D441F27601795C012998BF02F521
:106ED000007241F28701795CC80706D441F286014D
:106EE000795C012998BF02F5007241F29701795C43
:106EF000C90706D441F29601795C012998BF02F5D1
:106F00000072104645E194F8C426022A00F050862B
:106F10001E4B1B491B681E4EC1F8983103200023ED
:106F2000C1F8943133602870FAE6154F97F8A03114
:106F300023B1184B1B689B0140F11C823046FEF7C1
:106F4000FBFD3B88B7F89C117A6801339BB2013195
:106F50000132202B3B80A7F89C117A607FF4DEAED3
:106F6000B7F89E3194F8C42601330021A7F89E316A
:106F70003980D5E64868002074450020784F00200D
:106F8000541D0020504F002024730020EC190020D5
:106F900018260020681A002094F8C426B24F022A4E
:106FA00041D197F88431B14E002B40F0EB81D6F8F7
:106FB0000080B8F1000F32D098F800307BB398F819
:106FC0002820002A7FF4AEAE98F81830D8F82410A4
:106FD000C8F8382088F83C2013F008034FF004026A
:106FE00088F82820C8F82C10C8F8301003D0A04A20
:106FF00041F29413D358C8F834304FF00009C8F860
:107000002490C8F80890C8F80C90404625F00EFC73
:107010000523C8F8409088F8283094F8C426002149
:107020000423316033759349D7F898310968C83320
:107030008B420CD3002A00F05287022A7FF484AEE0
:107040001FF0D8F894F8C42600283FF469AE002A4F
:1070500000F0078701232B7062E6834F854AD7F83B
:107060009831126864339342BFF458AEDFF814923B
:10707000D9F800303F2B5DDDD7F894317E4E4FF0CC
:1070800040080FE0FEF71AFDD9F80020D7F8943138
:10709000013A0133B8F10108C9F80020C7F894316A
:1070A00000F02987F35C1846002BEBD14FF0FF323C
:1070B00000210423C7F89821C7F894112B7094F885
:1070C000C4262DE66D4A0292A2F10C0329210193F8
:1070D0000091A2F10A035021163A492023F0CEFF75
:1070E00000287FF41BAE604B94F8C426C3F89401CB
:1070F00007214FF0FF30C3F89801297010E6604B6C
:10710000002105208DE80300A3F10802029153201D
:1071100023F0B4FF00287FF401AE534B94F8C4264B
:10712000C3F8940108232B70FAE5564B1B683F2BDC
:1071300000F3B48094F8C426002A7FF4F1AD03E68E
:10714000514B494F1B6813F0007F3B883FF4FAAE68
:10715000002B7FF4F7AED7F804804520FEF7AEFC95
:107160000E20FEF7ABFC404605F018FC304605F05B
:1071700015FC4FF480520A233046A7F89C212B704F
:10718000FEF7DAFCDDE6414B186803689B68984718
:107190002B78DFF8F0E0344FDEF8002097F89011FC
:1071A0000A44B2F5807FA8BF4FF480728242A8BF24
:1071B0000246CEF8002088E52E4B2B4F1B6803F5C6
:1071C0009C530833C7F8A4312B78012B7FF4B8AD5A
:1071D00097F8A131002B7FF4B3AD002A3BD12C49A5
:1071E0002C4B2D4891F9008091F90CC091F918E0D1
:1071F00091F9246091F9305091F93C4091F948900F
:1072000091F954A01B6802700132D2B2F3B119880F
:1072100001F08101812919D193F90210414500F053
:107220000F878C4500F00987714500F00387B14254
:1072300000F0FD868D4200F0F786A14200F0F18655
:10724000894500F0EB86514500F0E086082A03F1FD
:107250000803D9D1027024F0ABF9012387F8A131DA
:107260006EE5002095E700BF541D00201487002024
:10727000784F0020EC1900208C50030802510308BD
:10728000E052030818260020681A00202C870020EE
:1072900020880020848800208088002094F8E02541
:1072A000B24F742303FB0243D7F8941193F8D03400
:1072B000492900F2BB85DFE811F0A8019C01930188
:1072C0008B014E0145013C0133016D0264025E02F7
:1072D0005102490242023902300227021602050217
:1072E000F401E301D201C101B0016A04550445046F
:1072F0003504250415040504F503E503D503C90386
:10730000B903AD03A103950389037D0314030803A7
:10731000FC02F002E402D802CC02C002B402A802CD
:107320009C0293028A028102780219010E01030174
:10733000F900F000E700DE00D500CC00C300BA0081
:10734000B100A8009F00960081002A012201884B0D
:107350001B681B7A053B032B7FF602ADB4F8D010F7
:10736000FEE441F22602BA5C022A34BF4FF40072F6
:10737000002272E597F8A131002B7FF4DFAD0923DD
:107380002B70DEE5306800283FF449AE0378002B0F
:107390003FF445AE90F82830002B7FF4C3AC8268F0
:1073A0004168C3628A4238BF0A460323826080F87C
:1073B000283022F0F7FF94F8C42630E6D4ED367A70
:1073C0009FED6C7A6C4867EE877AFDEEE77A17EEF0
:1073D000901A05F077FBD7F894310133C7F8943150
:1073E00094F8C4269CE4B4F8D210644805F06AFB13
:1073F000D7F894310133F1E794F8D410604805F0E0
:1074000061FBD7F894310133E8E794F8D5105D4873
:1074100005F058FBD7F894310133DFE794F85C129C
:10742000594805F04FFBD7F894310133D6E7B4F84B
:107430007612564805F046FBD7F894310133CDE774
:1074400094F87212524805F03DFBD7F8943101339D
:10745000C4E794F870124F4805F034FBD7F8943124
:107460000133BBE794F8B0124B4805F02BFBD7F87B
:1074700094310133B2E794F80F12484805F022FB2B
:10748000D7F894310133A9E794F82412444805F061
:1074900019FBD7F894310133A0E794F81912414849
:1074A00005F010FBD7F89431013397E7B4F81632A2
:1074B0009FED307A3C4807EE903AF8EEE77A82E7A3
:1074C000B4F80A22B4F80612384805F0FBFAD7F8E7
:1074D0009431013382E7B4F80822B4F80412344836
:1074E00005F0F0FAD7F89431013377E794F80112F8
:1074F000304805F0E7FAD7F8943101336EE7A16818
:107500002D4805F0DFFAD7F89431013366E794F897
:10751000F9112A4805F0D6FAD7F8943101335DE71E
:107520004FF07E51264805F0CDFAD7F8943101335B
:1075300054E7B4F8CE10234805F0C4FAD7F89431D4
:1075400001334BE7B4F8CC101F4805F0BBFAD7F86D
:107550009431013342E794F8C32694F8C2161B48CD
:1075600005F0B0FAD7F89431013337E7541D002005
:10757000387200200000C8424882030834820308A1
:107580001C82030804820308EC810308CC810308F1
:10759000AC810308988103087C8103086C8103088F
:1075A00058810308488103083881030820810308B3
:1075B0000C810308F88003087082030860820308C6
:1075C000787D0308687D0308587D0308447D03081F
:1075D000CA49CB4805F076FAD7F894310133FDE675
:1075E000C84AC949C94805F06DFAD7F89431013342
:1075F000F4E6C74B0093C74AC74BC849C84805F0D3
:1076000061FAD7F894310133E8E6C649C64805F077
:1076100059FAD7F894310133E0E6742101FB02F204
:1076200003EB430302EB83032344C04893F8DA14CB
:1076300005F048FAD7F894310133CFE6742101FB05
:1076400002F203EB430302EB83032344B84893F8AD
:10765000D61405F037FAD7F894310133BEE6742119
:1076600001FB02F203EB430302EB83032344B14823
:1076700093F8D51405F026FAD7F894310133ADE626
:10768000742101FB02F203EB430302EB8303234467
:10769000A94893F8DB1405F015FAD7F894310133B3
:1076A0009CE6742101FB02F203EB430302EB83032C
:1076B0002344A24893F8D31405F004FAD7F8943180
:1076C00001338BE6742101FB02F203EB430302EB6F
:1076D000830323449A4893F8D41405F0F3F9D7F8B8
:1076E000943101337AE6742101FB02F203EB430388
:1076F00002EB83032344934893F8D21405F0E2F994
:10770000D7F89431013369E694F8F8118E4805F002
:10771000D9F9D7F89431013360E694F8FE118B481B
:1077200005F0D0F9D7F89431013357E6884B8948F2
:10773000996C05F0C7F9D7F8943101334EE6864BC2
:107740001B681A0500F152840E2347E6B989834865
:1077500005F0B8F9D7F8943101333FE694F83B329D
:1077600094F83D2294F83C127D4805F0ABF9D7F827
:107770009431013332E6BB68D90400F127840D232C
:107780002CE6784B7848198905F09CF9D7F89431A4
:10779000013323E6754B764A19881288754805F03F
:1077A00091F9D7F89431013318E694F80012724831
:1077B00005F088F9D7F8943101330FE694F8FF11FA
:1077C0006E4805F07FF9D7F89431013306E694F856
:1077D0004D126B4805F076F9D7F894310133FDE589
:1077E00094F84C12674805F06DF9D7F894310133DD
:1077F000F4E5742303FB02426348D2F8CC1405F08D
:1078000061F9D7F894310133E8E5742303FB0242B0
:107810005E48D2F8C81405F055F9D7F89431013311
:10782000DCE5742303FB0242594892F8C51405F0C5
:1078300049F9D7F894310133D0E5742303FB0242B0
:10784000544892F8C41405F03DF9D7F89431013347
:10785000C4E5742303FB02424F48D2F8C01405F07C
:1078600031F9D7F894310133B8E5742303FB0242B0
:107870004A48B2F8BC1405F025F9D7F89431013321
:10788000ACE5742303FB0242454892F8B61405F0B8
:1078900019F9D7F894310133A0E5742303FB0242B0
:1078A000404892F8B51405F00DF9D7F8943101333A
:1078B00094E5742303FB02423B4892F8B41405F0AC
:1078C00001F9D7F89431013388E5742303FB0242B0
:1078D0003648B2F8AE1405F0F5F8D7F89431013314
:1078E0007CE5742303FB0242314892F8AC1405F0A6
:1078F000E9F8D7F89431013370E500BF444C00201B
:10790000347D0308507B0308447B0308207D030873
:10791000107D0308DC7C03085C7B0308E47C03081F
:10792000F07C0308BC7C0308C87C03087C7E030849
:10793000707E0308647E0308547E0308447E0308B7
:10794000387E03082C7E0308147E0308007E03089B
:1079500070740020F47D0308504F0020D47D03088C
:10796000B87D0308F81900209C7D030846720020AA
:107970004C720020887D0308E4800308D880030847
:10798000C8800308CC800308B48003089C800308E7
:10799000848003086C80030854800308388003083F
:1079A0002480030808800308F07F0308E07F0308B1
:1079B000C47F0308742303FB02428748B2F8AA1469
:1079C00005F080F8D7F89431013307E5742303FB01
:1079D00002428248B2F8A81405F074F8D7F894313E
:1079E0000133FBE4742303FB02427D48B2F8A61482
:1079F00005F068F8D7F894310133EFE4742303FB02
:107A000002427848B2F8A41405F05CF8D7F8943133
:107A10000133E3E4742303FB0242734892F8A21497
:107A200005F050F8D7F894310133D7E4742101FB05
:107A300002416E4891F8A13491F8972491F88D1481
:107A400005F040F8D7F894310133C7E4742303FB01
:107A50000242674892F88C1405F034F8D7F8943154
:107A60000133BBE4742101FB0241624891F89F3469
:107A700091F8952491F88B1405F024F8D7F89431F7
:107A80000133ABE4742101FB02415B4891F89E3461
:107A900091F8942491F88A1405F014F8D7F89431E9
:107AA00001339BE4742101FB0241544891F89D3459
:107AB00091F8932491F8891405F004F8D7F89431DB
:107AC00001338BE4742101FB02414D4891F89C3451
:107AD00091F8922491F8881404F0F4FFD7F89431C7
:107AE00001337BE4742101FB0241464891F89B3449
:107AF00091F8912491F8871404F0E4FFD7F89431B9
:107B000001336BE4742101FB02413F4891F89A3440
:107B100091F8902491F8861404F0D4FFD7F89431AA
:107B200001335BE4742101FB0241384891F8993438
:107B300091F88F2491F8851404F0C4FFD7F894319C
:107B400001334BE4742101FB0241314891F8983430
:107B500091F88E2491F8841404F0B4FFD7F894318E
:107B600001333BE4742103EB430301FB02F101EB1E
:107B700083012144274891F8D93491F8D82491F809
:107B8000D71404F09FFFD7F89431013326E4742111
:107B900001FB02F203EB430302EB830323441E4881
:107BA000B3F8DC1404F08EFFD7F89431013315E4F8
:107BB0001A4E337D052B3FF6B1A801A252F823F0EF
:107BC000E96C00081D6D0008B77D0008797C00088D
:107BD000C77C0008257E0008AC7F0308987F030857
:107BE000887F0308787F0308607F0308507F0308BD
:107BF000447F0308307F03081C7F0308087F0308C5
:107C0000F87E0308E87E0308D87E0308C47E0308D4
:107C1000B07E0308A07E03088C7E03081487002032
:107C2000716891F91A305F1C0AD0C64A03F5817356
:107C300002EB0313FF20DA796FF30002DA71887622
:107C400091F91B30581C15D0BE4F03F5817307EB1B
:107C5000031207EB0317D279FB79C2F34502012A1D
:107C6000C6BF02F1FF32D2B20022FF2062F3460308
:107C7000FB71C87603233375B3480378002B7FF478
:107C80004DA87768002F00F07B8197F82830002BF3
:107C90007FF444A82838442239462AF0D5F93B78A5
:107CA0007BB197F8283063B9BA687968FB628A4279
:107CB00038BF0A460323BA6087F82830384622F0D6
:107CC00071FB002373603769DFF898E2DFF898B240
:107CD0009E4BDFF89892DFF8988201370597AEFB4C
:107CE000077C059FABFB077B059F0FCBA9FB0779A3
:107CF000059F4FEADC0CA8FB0778AEFB0C7A4FEA35
:107D0000DA0A0AEB8A070DF1200AAAE807004FEA0F
:107D10005B1B4FEA58384FEA9919AEFB0B21AEFBBB
:107D20000902AEFB080EACEB4700059F8AF8003055
:107D30000CEB8C0CA7EB4C0C41F2A403C908D20845
:107D40004FEADE0E7F4F01EB810102EB82020EEB68
:107D50008E0EABEB4101A9EB4202A8EB4E0E17F8D9
:107D6000038001F1300B303002F130010CF1300CA6
:107D70000EF1300201238DF826008DF827C08DF812
:107D800025B08DF824108DF823203375B8F1000F3D
:107D900000F0D68041F2E802BA5C002A00F08E8042
:107DA00041F22C130220FB5C002B00F0888004239E
:107DB0003375FEF7B3BFDFF8BC91DFF8BC81DFF8A5
:107DC000BCA1706807AA494622F02EFA0128414654
:107DD0004FF003027EF4A2AF079F3846002F3FF416
:107DE0001FAF3B78002B3FF41BAF2CF00DFD03229F
:107DF00051460028E5D107F108002CF005FD0346A7
:107E00000028DED157F8030F08903A798DF8242026
:107E100008A88DF825302AF0EFF83369984265D824
:107E20003361CEE794F8C426FFF772B894F8C426FD
:107E30008AB1022A7EF488AF1EF0DCF900283EF4F5
:107E40006DAF4FF480520A23A7F89C212B7094F851
:107E5000C426FEF765BF3E4B186803685B69984708
:107E6000ECE73B4B3B4918684E68B04266D00E6960
:107E7000B04261D0CE69B04254D08E6AB04200F0B8
:107E8000AF804E6BB04200F0AF800E6CB04200F09D
:107E9000A980CE6CB04200F0B7808E6DB04200F089
:107EA000B18097F8A2110020022918607FF4D2A8AF
:107EB00019F079FD94F8C426FFF7CCB8184600EB0A
:107EC000001007EB8000244B009300F5855008A9B3
:107ED0003C232022043022F00DFEFEF71FBF1C4B76
:107EE000186803685B699847FFF7ACB808A82AF0E0
:107EF00083F8034694E7F35C002B7EF40FAFFFF7A3
:107F0000D5B8134603EB031307EB830000F5855048
:107F1000124B0093102213231149043022F0EAFD82
:107F2000FEF7FCBE022606EB460601EB86010026A4
:107F3000C6620E814E60B4E70126F4E71646F2E70A
:107F40004046BCE7784F0020586100207C8203083F
:107F50002C8700202088002067BB000871C600081D
:107F6000AC7C0308CDCCCCCC1F85EB51D34D62103B
:107F70005917B7D11C870020B47C0308B87C0308CC
:107F800029F07CFF00283EF4C9AE7768002F7FF40B
:107F900086AE96E64520FDF791FDFF20FDF78EFDAC
:107FA00094F8C436022B4ED02F4B304C45219846C6
:107FB000D8F8000002681268904714F8011F0029E1
:107FC000F6D10020FDF77AFDFEF731BF94F83812A4
:107FD000274804F077FDD7F894310133FFF7FEB955
:107FE0000326A0E705269EE704269CE7B4F9402275
:107FF000B4F942121F4804F065FDD7F894310133FB
:10800000FFF7ECB907268EE706268CE71A4B0270BD
:108010005B68002B7EF494AEFFF71DB90270174B1E
:10802000F6E70270164BF3E70270164BF0E70270AA
:10803000154BEDE70270154BEAE70270144BE7E7CA
:10804000144B0270E4E7144B1868037E13F0060F1C
:10805000B7D090F82830002BB3D10A22034913F08F
:1080600017FBAEE702234DE72C870020A07C030816
:10807000A87D0308E07D030874880020688800203C
:108080005C88002050880020448800203888002028
:108090002C8800202088002014870020437913F0CA
:1080A000020308D00369426A806A013B101A184033
:1080B000C0B2181A704718467047426A806A131A8D
:1080C00058425841704741717047704743799B0748
:1080D0000AD5436A8269D154436A01690133B3FB0B
:1080E000F1F201FB123343627047437913F001034D
:1080F0001FBFC369026AC0689B1A1ABF00F1FF3034
:1081000018401846704710B5437913F00103014633
:108110000ED0FFF7EAFF60B10B6A4A69CC68D05C09
:108120000133B3FBF4F204FB1233C0B20B6210BD97
:10813000184610BD90F8433830B53BB990F8411857
:1081400090F842380124DAB2914200D830BDB0F83C
:108150004A5804FA03F22A43A0F84A280133F2E706
:10816000054B064A19785B7882F88B16013B82F83A
:108170008C360020704700BFFC1E00207445002094
:10818000094B9A7832B9094AD27802F00102DA70C2
:1081900001229A70064A92F88B1692F88C26197072
:1081A00001325A7000207047FC1E0020504F002002
:1081B0007445002030B1007910F1FF3018BF4FF046
:1081C000FF3070474FF0FF307047064B1A7932B9D5
:1081D000054A528802F001025A7101221A710020E8
:1081E000704700BFFC1E0020504F00200B4A0C4976
:1081F0009379742000FB03131189A3F8A414518907
:10820000A3F8A8149189A3F8AA14D189128AA3F813
:10821000A614A3F8AE240020704700BFFC1E002067
:10822000744500200B4A0C499379742000FB03131A
:108230000020B3F8A4141181B3F8A8145181B3F845
:10824000AA149181B3F8A614B3F8AE34D181138285
:10825000704700BFFC1E0020744500200D4B0E49E6
:108260009A7C30324A709A790C49742000FB0212D1
:10827000002092F8C514D97492F8C414197592F8B4
:108280008B14597592F8951492F89F249975DA75A4
:10829000704700BFFC1E00207A00002074450020BB
:1082A0000E4A0F49937C907930330B71137E303333
:1082B0008B7192F82630742141430C2000FB03138C
:1082C00008490B4400201968C2F81A105968C2F80E
:1082D0001E109968C2F82210704700BFFC1E0020D3
:1082E0007A000020464A00200B4B987993F826101C
:1082F000742242430C2000FB01220849114453F828
:108300001A2FC1F8D2245A68C1F8D6249A68C1F845
:10831000DA240020704700BFFC1E002074450020B6
:1083200008B5A0F15002D2B280213C2015F0A4F98A
:10833000002280213C2015F09FF9102280213C2052
:10834000BDE8084015F098B964292DE9F84328BF25
:1083500064212F4B11FB00F983FB09235B090746BE
:108360005FFA83F89BB12B4D00262B4C14F8012BA0
:1083700040213C2015F080F9AC42F7D101360022B3
:1083800040213C2015F078F9F3B29845EDD84745E7
:108390001ED808F10103DBB29F4217D9023FA7EBB9
:1083A0000807FFB21D4D013700261D4C14F8012BA4
:1083B00040213C2015F060F9A542F7D1013600229A
:1083C00040213C2015F058F9BE42EED1BDE8F883BB
:1083D000144C154A84FB0934E408C8EB8813663C46
:1083E000C8EB83031C44E4B2203C04EB8404651D09
:1083F0001544144414F8012B40213C2015F03CF99D
:10840000AC42F7D1002240213C2015F035F9C0E7FD
:108410001F85EB516C6F0308676F0308536F0308E8
:108420004E6F030867666666EC6C030810B50C4671
:1084300005F0F2F8032282710022C2712146BDE8E4
:10844000104005F07FBB10B50446007910B1222121
:10845000FFF7ECFF63792268990802238B40D94328
:1084600089B21161D1689BB20B43D36010BD10B5C6
:108470000446007910B10121FFF7D8FF6379216824
:108480009A0802239340C868DB439BB20340CB6049
:1084900010BD73B590F85338032B04460D462DD10B
:1084A00000231D4E8DF807309DF8073094F85428AE
:1084B0009A4201D802B070BD9DF8073006EBC303A5
:1084C00093F82C3083B185F001037BB19DF8073020
:1084D00006EBC303986A05F0F7FC9DF807300133FB
:1084E000DBB28DF80730DFE72B46EEE79DF807306B
:1084F00006EBC303986A05F0E1FCEEE7836B406B83
:10850000DB799B0748BF81F0010515B105F0DCFC64
:10851000D0E705F0D3FCCDE7FC1E002008B5074BE3
:108520009A782AB1DB784FF080701BB105F08EFF8E
:10853000002008BD05F082FFFAE700BFFC1E002006
:1085400008B5074B1A792AB15B794FF480301BB11B
:1085500005F07CFF002008BD05F070FFFAE700BFC2
:10856000FC1E002070B50F4C0F4DA279E37C7426E1
:1085700006FB025282F8C534237D82F8C4340B4BCB
:1085800018681AF0ABFBA379627D06FB0353002049
:1085900083F88B24A27D83F89524E27D83F89F24C1
:1085A00070BD00BFFC1E002074450020483900202B
:1085B00010B50C490C4A8879742300FB03238831D9
:1085C0000022505C03F8010F881803324478807849
:1085D0009C72092A1875F4D1044B18681AF07EFBB6
:1085E000002010BDFC1E0020F74900204839002063
:1085F0001FB50123ADF80830ADF80410002301A920
:10860000ADF80A30ADF80C30ADF806201DF044FF8F
:1086100005B05DF804FB70B5A0F6580494F8453831
:10862000C3B1B4F84C3801339BB2082BA4F84C38D2
:1086300040F29180002384F84538A4F84C38A36BAD
:10864000022259791868FFF7D3FF94F84538002BB8
:1086500040F08180404D95F891301BB901212046B2
:10866000FFF717FF94F8443853BBA36A626A9A4233
:1086700003D1002385F8913070BD95F89120022A2E
:1086800012D802F1010214BFFF237F2385F8912045
:10869000A4F84838082384F84638012384F844387D
:1086A000A06BBDE87040E2E65A1CA169A262CB5CF7
:1086B00021698A4228BF0022DBB228BFA262E7E715
:1086C00094F94638002B3CD094F8481811F0010179
:1086D00027D095F89260012E03D801212046FFF79C
:1086E000D8FE023E012E03D800212046FFF7D1FE1E
:1086F00095F892300133DBB2032B85F892302AD9FA
:10870000B4F848385B08A4F8483894F84638013B78
:108710005BB2002284F8463885F89220002BA4D062
:1087200070BD95F8923013F0FD0304D1012120466D
:10873000FFF7AFFEDCE7012BDAD12046FFF7A9FEF9
:10874000D6E7616AA26A914205D184F84438A06BE9
:10875000BDE8704077E670BDFC1E00202DE9F04FAB
:10876000074685B0002016460C4615F04BF9002050
:1087700015F02EF90EF050FD022E09D0042E0AD06D
:10878000022E4FF4964508D1FF2C06D1032629E08E
:108790004FF41645F8E744F6C0150023C8498DF894
:1087A0000D3014209DF80D300B2B01D900230AE069
:1087B0009DF80D3000FB0313DB79DA0740F1B08040
:1087C0009DF80D30DBB2611E1944C9B20B2900F2CD
:1087D0001282032E06D0BA4B01EB810103EB81011B
:1087E000B84B9963B74CB84BB54A236004F13C00D1
:1087F00003234FF4806163716061002304F5886096
:108800004FF00108032E84F85368C4F83C24A56097
:10881000A371E362E1602362E361A0612161A3626D
:10882000636284F8443884F8408884F84138A4F8B6
:108830004E38A4F85038A4F84C3884F85238914691
:108840000DD0D4F838A09AF8040004F0E5FE606377
:108850005046FFF7F8FD41462046FFF71AFE32204A
:1088600007F0FEFC002E62D1D4F83C5428681DF0BD
:10887000F3FE28460122222107F03EF9934BC4F86B
:10888000583832469249284607F090F8A56B286878
:108890001DF0E2FE01224FF6FF71284607F02CF989
:1088A000022269792868FFF7A3FE8A4BC4F85C3876
:1088B00032468949284607F079F8884D4FF001097A
:1088C000C5F894404FF0060A022E10D0D5F8940057
:1088D0000EF09AFC58B1012015F094F8D5F89400E8
:1088E0000EF092FC002840F0C08015F08BF838465E
:1088F0000EF08AFC70B1012015F06AF84FF0050BFC
:108900004FF0000838460EF07FFC002840F0B6809B
:1089100015F05EF8042ED9D0052007F0A1FCD3E7AE
:108920009DF80D200132D2B28DF80D203AE7012ECC
:1089300008D1D4F83C04294623F0C5FFA06B23F0EE
:10894000EFFFBAE7022E08D1A06BFFF790FD294692
:10895000D4F83C0423F0B7FFAFE7032E7ED14FF0ED
:10896000000884F85488602241465D48DFF874A10D
:108970002BF0A3FE8DF80E809DF80E200B2A09D94E
:1089800001215048FFF785FD2946D4F83C0423F027
:108990009AFF92E79DF80E2002EB82020AEB820218
:1089A000127B002A4CD09DF80E2002EB82020AEBCB
:1089B00082021269002A43D000228DF80F204FF066
:1089C000140B9DF80F200B2A2AD89DF80E809DF8D5
:1089D0000F205FFA88F80BFB029208EB88081079E9
:1089E0000AEB880804F018FED8F8102082422ED135
:1089F0009DF80F0000EB800009EB8000FFF737FDCA
:108A00009DF80F200BFB029B9BF80720930707D5CF
:108A100094F85428314B03EBC202012182F82C1048
:108A20009DF80E2094F854182C4B02EB82020AEBAE
:108A3000820203EBC10012698262013184F854188A
:108A40009DF80E200132D2B28DF80E2094E79DF8E9
:108A50000F200132D2B28DF80F20B2E7042E7FF43E
:108A60002CAFA06BFFF703FD63E7D5F894000EF081
:108A7000C7FB014638460EF0CBFB2FE738460EF019
:108A8000BFFB95F8A62003468AB9242801D185F8B2
:108A9000A690012E05D11946384601930EF0B8FB79
:108AA000019BD5F8940019460EF0B2FB2AE7012A83
:108AB0001AD14D280CBF0222002285F8A620E8E733
:108AC000546A03088C8800200053030817860008A6
:108AD000E4900020FD8B0008E8900020FC1E0020A0
:108AE000241F002000780020022A06D13C280CBF59
:108AF0000322002285F8A620CBE7032A10D10A28FA
:108B000002D985F8A680C4E7042285F8990085F883
:108B1000988085F89B8085F89A0085F8A620B8E7AC
:108B2000042A09D195F89A2085F8A700424085F8D3
:108B30009A2085F8A6B0ACE7052AAAD195F8981036
:108B400095F8992095F89A00914209D24A1C294437
:108B5000584085F89A0085F8982081F89C3098E76D
:108B60009842CED195F8A71085F8A6A0F42990D107
:108B7000002A8ED12421384685F8A62001920EF0D5
:108B800047FB4D2138460EF043FB3E2138460EF0A0
:108B90003FFB019A384611460EF03AFBF421384665
:108BA0000EF036FBF42138460EF032FB032E18D0BF
:108BB000A26B53791168980802238340DB439BB270
:108BC0000B61C8680340CB60107910B12021FFF71A
:108BD0002DFCA06B002123F0D3FBA36B18681DF0C4
:108BE0003BFDD4F83C04002123F0CAFBD4F83C340C
:108BF00018681DF031FD05B0BDE8F08F38B5A0F65E
:108C00005C04A1F12905A36B18680022302D426293
:108C1000324D31D895F8A8300133DBB2012B89BF32
:108C2000B4F84A3885F8A8305B08A4F84A3881BF00
:108C300095F8A93085F8A820013385F8A93095F872
:108C4000A9200023082AA4F84C3814D185F8A930AB
:108C5000B5F8AA3001339BB2032BA5F8AA3007D987
:108C60006379DB0704D5E36A94F84A0853B398475D
:108C70000023A4F84A3838BD5B396C290ED8B4F803
:108C80004A3885F8A8205B0843F08003A4F84A38E6
:108C900095F8A930013385F8A930D0E794F8452834
:108CA000002ACCD1012184F8451885F8A91080212B
:108CB000A4F84A18597985F8A820A5F8AA20FFF742
:108CC00097FCBCE7E3696269D054E369E16801336A
:108CD000B3FBF1F201FB1233E361C9E7FC1E002094
:108CE00038B5A0F65C046379DB074AD5A57994F81A
:108CF000403805F0010503B3D4F83C341A68D36A50
:108D00005B08536294F8443823B1B4F84E38013309
:108D1000A4F84E38A36B6A0059791868FFF768FC0D
:108D2000012384F84338002384F8413884F842381A
:108D300084F84038A4F84A3838BD94F84338012BF9
:108D400004BF94F8413884F842382046FFF7F2F91E
:108D500094F84328A36B4AB9012284F8432859792F
:108D6000186805FA02F2BDE8384041E4002284F8B0
:108D7000432895425979186808BF0222BDE8384057
:108D800036E438BD10B5A0F6580494F845381BBB3E
:108D900094F844288ABBA36A616A99421CD0591C82
:108DA000A069A162C35C2069DBB25B0043F400737D
:108DB000A4F848380A2384F84638012384F8443854
:108DC00094F85338814228BFA262012B01D0042BB2
:108DD00002D1A06BFFF74BFB94F84038002B73D106
:108DE00094F841380133DBB2092B84F8413827D19C
:108DF0002046BDE81040FFF79DB994F946387BB195
:108E0000B4F848184B08A4F8483801F0010120468E
:108E1000FFF73FFB94F84638013B84F84638DBE720
:108E200084F84438626AA36A9A42D5D194F85338D8
:108E3000012B01D0042BCFD1A06BFFF704FBCBE7B4
:108E40000A2B41D194F843382BB9B4F84A3843F08F
:108E50000103A4F84A386379D9070AD5B4F84A0857
:108E6000820501D4C3071DD4B4F850380133A4F8E7
:108E70005038012284F8402894F843280023012A1E
:108E800084F8413820D1A27984F84338A36B12F0DA
:108E9000010F0CBF0222002259791868BDE810406A
:108EA000FFF7A6BBE36AC0F347000BB19847E0E7C2
:108EB000E3696269D054E369E1680133B3FBF1F21D
:108EC00001FB1233E361D4E710BD10B5D422802139
:108ED0003C2014F0D1FB802211463C2014F0CCFB46
:108EE000A82280213C2014F0C7FB3F2280213C2097
:108EF00014F0C2FBD32280213C2014F0BDFB0022E1
:108F000080213C2014F0B8FB402280213C2014F04A
:108F1000B3FB8D2280213C2014F0AEFB1422802173
:108F20003C2014F0A9FBA12280213C2014F0A4FBDA
:108F3000C82280213C2014F09FFBDA2280213C20B3
:108F400014F09AFB122280213C2014F095FB812220
:108F500080213C2014F090FBCF2280213C2014F093
:108F60008BFBD92280213C2014F086FBF12280214A
:108F70003C2014F081FBDB2280213C2014F07CFBA0
:108F8000402280213C2014F077FBA42280213C2049
:108F900014F072FBA62280213C2014F06DFBAF225E
:108FA00080213C2014F068FBA62280213C2014F094
:108FB00063FBAE2280213C2014F05EFB2022802146
:108FC0003C2014F059FB002280213C2014F054FB7B
:108FD000B02280213C2014F04FFB402280213C2015
:108FE00014F04AFB002280213C2014F045FB1022A3
:108FF00080213C2014F040FB4FF48064013C0022AF
:1090000040213C20A4B214F037FB002CF6D1812281
:1090100080213C2014F030FBC82280213C2014F039
:109020002BFBAF2280213C2014F026FB012010BD39
:109030009F4B1B6823B193F90830002B00DD70476C
:109040002DE9F04F9B4CD4F8C4302DED028BC31AA0
:10905000002B87B02CDB984B94F8C8101B7803F0DA
:109060000403002B059300F5433314BF01220022B3
:1090700003F5A07384F8C820C4F8C4301DD00129BA
:1090800016D08E4F01237A783B707B70FB78BA70D4
:109090008B4D23F002030544AE2280213C20FB705F
:1090A000BD6014F0E9FA002840F01E81854B18706D
:1090B00007B0BDEC028BBDE8F08F804FFB7821B18B
:1090C000BA787A7043F00203FB709D071BD4BA682C
:1090D000821A002A02DBD90700F162810023DFF83F
:1090E000E4813B7098F80030002BE1D07B78072BAF
:1090F0004FD8DFE813F058014E009E015704D90302
:1091000095022102CC0101223A70DA07C0D53A79E2
:109110006D496E4D0132D2B2A1FB0261890801EBAB
:109120004101A2EB4102D2B215443A7195F82820D0
:109130007A70ADE7034623440022284683F8AC202A
:10914000FFF7EEF894F8AC60CEB1614F614D203E70
:1091500006EB860606F10509A9442E4416F8012BF4
:1091600040213C2014F088FAB145F7D1002240217B
:109170003C2014F081FA17F8016F002EE7D111F0AE
:1091800033FC05464046FFF7CBF829461520FFF78C
:10919000DBF8059B002B8BD14F4B4E4D93F82030C5
:1091A000052B9CBF494A9B184FF0800198BF93F84C
:1091B0005C604FF0B0024FF03C0094BF203E1F2691
:1091C00014F05AFA0C2280213C2014F055FA162291
:1091D00080213C2006EB860614F04EFA771D2F44C2
:1091E0002E4416F8012B40213C2014F045FABE42D3
:1091F000F7D1002240213C2014F03EFAB022802119
:109200003C2014F039FA022280213C2014F034FA78
:10921000172280213C2014F02FFA304A304B12786C
:109220001B78002A14BF52260126002B18BF3226B5
:1092300006EB8606771D2F442E4416F8012B40219D
:109240003C2014F019FAB742F7D1002240213C200B
:1092500014F012FAB02280213C2014F00DFA0822FA
:1092600080213C2014F008FA172280213C2014F0C1
:1092700003FA94F8C9201B4BD35C203B03EB830318
:109280005E1D2E441D4415F8012B40213C2014F096
:10929000F3F9B542F7D1002240213C2014F0ECF95B
:1092A00094F8C930013303F0030384F8C930FFE6B2
:1092B000FC900020FC1E0020744F00200091002034
:1092C000404B4C00EC900020ABAAAAAA0053030824
:1092D000A81F0020EC6C0308081B0020AC7F0020B6
:1092E000946A00207C840308FFF7EFFDDFF82483F5
:1092F00088F8000000283FF4DBAEB02280213C203B
:1093000014F0BAF9402280213C2014F0B5F9002273
:1093100080213C2014F0B0F9102280213C2014F070
:10932000ABF94FF48065013D002240213C20ADB2F5
:1093300014F0A2F9002DF6D1B02280213C2014F0C7
:109340009BF92A4680213C2014F096F910228021B6
:109350003C2014F091F99E4B7A7803EB8203D3F80A
:10936000309099F80060002E3FF4BCAE994D203E3D
:1093700006EB860606F1050AAA442E4416F8012BD0
:1093800040213C2014F078F9B245F7D10022402169
:109390003C2014F071F919F8016F002EE7D1A1E615
:1093A00001223A70B3E68C4B8C4A8D498D4824F0EB
:1093B000A3FE0120FEF7B4FF94F8AC60002E00F08D
:1093C0007185884F834D203E06EB860606F1050821
:1093D000A8442E4416F8012B40213C2014F04CF9EF
:1093E000B045F7D1002240213C2014F045F917F890
:1093F000016F002EE7D10220FEF792FF7A4F53262D
:10940000203E06EB860606F10508A8442E4416F811
:10941000012B40213C2014F02FF9B045F7D1002258
:1094200040213C2014F028F917F8016F002EE7D1F5
:10943000AFE66E4F3B689A0700F1DE844FF00208FA
:1094400001251F057FF5A5AE694B6A481B686A4A6E
:109450000068009082FB0320DA17C2EB60126420E0
:1094600000FB123365495F4824F046FE5D4826F054
:1094700057FBC0B214283FF65DAE2021431CDBB27F
:109480002218152B184682F8AC10F7D153E6DFF8F6
:1094900088A1DFF850914FF000083AF9023B584993
:1094A0004246484624F028FE484626F039FBC0B222
:1094B000142800F2AB832021431CDBB22218152BA9
:1094C000184682F8AC10F7D12344A8F14F020025CA
:1094D000D2B280213C2083F8AC5014F0CDF82A465B
:1094E00080213C2014F0C8F8102280213C2014F088
:1094F000C3F894F8AC50CDB13A4F364E203D05EB51
:10950000850505F1050BB344354415F8012B4021C1
:109510003C2014F0B1F85D45F7D1002240213C20F9
:1095200014F0AAF817F8015F002DE7D108F101083F
:10953000B8F1040FB1D12CE60120FEF7F1FEDFF8FF
:10954000DC80244D5426203E06EB8606771D2F44F2
:109550002E4416F8012B40213C2014F08DF8B74220
:10956000F7D1002240213C2014F086F818F8016F52
:10957000002EE8D1234B9FED248A186837464FF020
:1095800001094FF0020AA846204BFAB234260028FF
:1095900006FB02360FDD1E4B1B68B34200F08082D3
:1095A0001B49002304E051F8045FAE4200F07482CE
:1095B00001338342F7D1B9F1110F3FF6EAAD114BF8
:1095C000186809F101095FFA89F90137DCE700BF82
:1095D00000530308EC6C03085C7B0308DC7C030885
:1095E000A8830308A81F0020107D0308504F002007
:1095F0009C1A0020A01A00201F85EB51CC83030881
:10960000708403087043002000247449A0100020D7
:1096100014430020EC9000203C7F0020908303083E
:10962000D14BD24993F8E025D14824F065FD0120C3
:10963000FEF776FE94F8AC60CEB1CD4FCD4D203E16
:1096400006EB860606F10508A8442E4416F8012B01
:1096500040213C2014F010F8B045F7D10022402101
:109660003C2014F009F817F8016F002EE7D1C24B27
:10967000DFF820B31B684FF0B20803F1FF3919F887
:10968000013F5BF8042B99F81410019199F80A1026
:109690000091B748B94924F02FFDB54826F040FAAB
:1096A000C0B2142800F2B4822021431CDBB222187D
:1096B000152B184682F8AC10F7D1234400254246FA
:1096C00080213C2083F8AC5013F0D6FF2A4680213D
:1096D0003C2013F0D1FF102280213C2013F0CCFF5E
:1096E00094F8AC50CDB1A24FA24E203D05EB8505BC
:1096F00005F1050AB244354415F8012B40213C2000
:1097000013F0BAFFAA45F7D1002240213C2013F004
:10971000B3FF17F8015F002DE7D108F101085FFAE8
:1097200088F8B8F1B50FAAD1954B964993F80090F7
:109730008F484A4624F0E0FC0520FEF7F1FD94F83E
:10974000AC60CEB18A4F8B4D203E06EB860606F10B
:109750000508A8442E4416F8012B40213C2013F0A4
:109760008BFFB045F7D1002240213C2013F084FF4D
:1097700017F8016F002EE7D174237B4A82497C4899
:1097800003FB09F31A4492F8D0844FEA480A0AEB23
:10979000080203EB8203744A1A4492F8D23492F816
:1097A000D42424F0A9FC724826F0BAF9C0B21428D7
:1097B00088BF034608D82021431CDBB22218152B92
:1097C000184682F8AC10F7D123440022062083F813
:1097D000AC20FEF7A5FD94F8AC30D3B1644F654DD5
:1097E0001E46203E06EB860606F1050BAB442E44D2
:1097F00016F8012B40213C2013F03EFFB345F7D172
:10980000002240213C2013F037FF17F8016F002E93
:10981000E7D17420544B5D49D04400FB09F000EBC4
:109820008800184490F8D83490F8D72490F8D904D8
:1098300000904F4824F060FC4D4826F071F9C0B20A
:10984000142888BF034608D82021431CDBB2221805
:10985000152B184682F8AC10F7D1234400220720BC
:1098600083F8AC20FEF75CFD94F8AC60002E3FF46A
:1098700090AC3F4F3F4D203E06EB860606F10508B3
:10988000A8442E4416F8012B40213C2013F0F4FE8E
:10989000B045F7D1002240213C2013F0EDFE17F82F
:1098A000016F002EE7D174E4DFF8ECA09AF80030E5
:1098B000002B3FF46EAC4FF0410BDFF8E090DFF887
:1098C000E0802C4D00265F4672084F3AD2B28021CC
:1098D0003C2013F0D1FE002280213C2013F0CCFE6E
:1098E000203F102280213C2007EB870713F0C4FEA5
:1098F00007F1050BAB442F4417F8012B40213C2006
:1099000013F0BAFEBB45F7D1002240213C2013F0F2
:10991000B3FE38F9023C1E49B3F5FA6FA8BF4FF405
:10992000FA63B3F57A7FB8BF4FF47A73A3F57A730D
:1099300081FB0321DB17C3EBA101C9B20920FEF7AC
:1099400003FD9AF80030B34200F21D810236F6B2F0
:109950009E42BFF41EAC0E2E08F104083FF419AC71
:1099600019F8027FB0E700BF7445002000840308A7
:10997000A81F0020EC6C0308483900200C84030861
:10998000E17F002024840308388403084C84030802
:1099900067666666505303089C1C0020986F030896
:1099A0006E1A00200120FEF7BBFCC24FC24D2026DC
:1099B000203E06EB860606F10508A8442E4416F85C
:1099C000012B40213C2013F057FEB045F7D1002277
:1099D00040213C2013F050FE17F8016F002EE7D114
:1099E000DFF80083D8F800309E0700F17D814FF04A
:1099F00003090227D80700F10D81190700F1B8818A
:109A0000AE48AF49B0F90420B0F90030B0F9020017
:109A1000009081FB0201D217C2EBA10212B20192A7
:109A2000A849A94AA94824F067FBA84826F078F875
:109A3000C0B2142800F239822021431CDBB2221864
:109A4000152B184682F8AC10F7D123440022384673
:109A500083F8AC20FEF764FC94F8AC60002E3FF471
:109A600098AB9A4F203E06EB860606F10508A844FF
:109A70002E4416F8012B40213C2013F0FDFDB0458B
:109A8000F7D1002240213C2013F0F6FD17F8016FBA
:109A9000002EE7D1FFF77DBB8D49342303FB021372
:109AA0009E6AD3F82CE093ED097A052A4FEA561600
:109AB0003FF487ADB8EE477A41F2883CC8EE077AAA
:109AC0007346009683498148FDEEE77A17EE905A77
:109AD00006FB05C60EFB05CE7F4DA5FB06567E4D4B
:109AE000A5FB0EE5760B6D0B0296019524F004FBA9
:109AF000764826F015F8C0B2142800F2858020219F
:109B0000431CDBB22218152B184682F8AC10F7D193
:109B10002344AAF150020025D2B280213C2083F8D0
:109B2000AC5013F0A9FD2A4680213C2013F0A4FD7F
:109B3000102280213C2013F09FFD94F8AC600AF1C4
:109B4000010A5FFA8AFAC6B1604D203E06EB86062E
:109B500006F1050BC344464416F8012B40213C2076
:109B600013F08AFDB345F7D1002240213C2013F0C9
:109B700083FD15F8016F002EE7D1BAF1080F7FF6CB
:109B80001AADFFF706BB4C4F07F1050B17F8012B79
:109B900040213C2013F070FDBB45F7D1002240214D
:109BA0003C2013F069FD99F80170203F07EB87070F
:109BB00007F1050BAB442F4417F8012B40213C2043
:109BC00013F05AFDBB45F7D1002240213C2013F091
:109BD00053FDB8F900303A49B3F5FA6FA8BF4FF416
:109BE000FA63B3F57A7FB8BF4FF47A73A3F57A734B
:109BF00081FB0321DB17C3EBA101C9B20920FEF7EA
:109C0000A3FB9AF80030A1E6034681E703465BE434
:109C1000034652E5314E96ED130A28F041FC96EDCD
:109C2000140A824628F03CFC96ED150A834628F07B
:109C300037FC534601902A4A2249CDF800B0234808
:109C400024F05AFA214825F06BFFC0B2142800F224
:109C500032812021431CDBB22218152B184682F8D2
:109C6000AC10F7D123440022384683F8AC20FEF72D
:109C700057FB94F8AC60C6B1144F203E06EB860645
:109C800006F1050AAA442E4416F8012B40213C2077
:109C900013F0F2FCB245F7D1002240213C2013F032
:109CA000EBFC17F8016F002EE7D1D8F800304F46D3
:109CB000A3E600BF78830308EC6C0308601A002059
:109CC00067666666E8830308FC830308A81F002014
:109CD000A0100020608403085917B7D170740020C9
:109CE000F8830308601B00207549764A0B6B886B6C
:109CF000496B009101907449744824F0FDF9734850
:109D000025F00EFFC0B2142800F2D1802021431CA0
:109D1000DBB22218152B184682F8AC10F7D1234479
:109D20000022022083F8AC20FEF7FAFA94F8AC6027
:109D3000C6B1664F203E06EB860606F10509A9442A
:109D40002E4416F8012B40213C2013F095FCB14520
:109D5000F7D1002240213C2013F08EFC17F8016F50
:109D6000002EE7D1D8F800304FF00409032741E670
:109D70005749584ACB68486909690091019052498E
:109D8000524824F0B9F9514825F0CAFEC0B214284F
:109D900000F293802021431CDBB22218152B1846B9
:109DA00082F8AC10F7D1234400217A1C384683F89E
:109DB000AC10D7B2FEF7B4FA94F8AC60002E3FF4C2
:109DC0001FAEDFF80881203E06EB860606F1050986
:109DD000A9442E4416F8012B40213C2013F04CFCE2
:109DE000B145F7D1002240213C2013F045FC18F882
:109DF000016F002EE7D103E6374B38481B88384AFD
:109E000000780090A2FB0302D20802EB8200A3EBD1
:109E1000400334492D489BB224F06EF92B4825F0BD
:109E20007FFEC0B2142844D82021431CDBB2221884
:109E3000152B184682F8AC10F7D1234400220120DC
:109E400083F8AC20FEF76CFA94F8AC60D6B1DFF87A
:109E50007C80254D203E06EB860606F10509A944C7
:109E60002E4416F8012B40213C2013F005FCB1458F
:109E7000F7D1002240213C2013F0FEFB18F8016FBF
:109E8000002EE7D110F0B0FD05460220FEF748FA9B
:109E900029461520FEF758FA4FF004083B680325C1
:109EA000FFF7CFBA104DFFF7A6BA0346CDE503463C
:109EB00035E70346C1E70346D4E6034673E700BF30
:109EC000F8190020E4830308E8830308A81F002092
:109ED000F0380020D8930308941A0020544F002033
:109EE000CDCCCCCCB4830308EC6C03082DE9F04155
:109EF000254FA0F17D0380463868012B03680D468D
:109F00001B682DD9414698471FFA88F8AE1D09E015
:109F1000444404EB1424984704F0FF04B5421FFAAC
:109F200084F811D015F8014B3868A4F17D03012B9A
:109F3000036821461B68EBD87D2198473868036881
:109F400084F020011B68E3E7E143C9B23868A1F15E
:109F50007D03012B03681B680BD9BDE8F04118474E
:109F60007D2198473868036888F020011B6898476E
:109F7000CAE77D2198473868036884F0DF011B68D1
:109F8000BDE8F041184700BFC81F0020036810B4A7
:109F90005A1C0A4C026019702388082283EA0121A6
:109FA00041F2210308044CBF83EA41014900013A10
:109FB00089B2F7D121805DF8044B7047F21C002074
:109FC00070B50A2104462A4EFFF7E0FF2046002123
:109FD000FFF7DCFF358805EB85056D00ADB2290A7A
:109FE0002046FFF7D3FF05F0FE012046FFF7CEFF26
:109FF000358805EB85056D00ADB2290A2046FFF7CF
:10A00000C5FF05F0FE012046FFF7C0FF194B1A4DB2
:10A010001B6885FB0325DB17C3EBA505C5F30721EB
:10A020002046FFF7B3FFE9B22046FFF7AFFF204617
:10A03000FF21FFF7ABFF2046FF21FFF7A7FF2046D8
:10A04000FF21FFF7A3FF2046FF21FFF79FFF2046D8
:10A05000FF21FFF79BFF2046FF21FFF797FF2046D8
:10A06000FF21FFF793FF20460021BDE870408DE7F8
:10A07000941A00209C1A00206766666638B57E2117
:10A080000446FFF783FF20460021FFF77FFF2046AD
:10A09000FF21FFF77BFF2046FF21FFF777FF1C4BD7
:10A0A0001D8805EB85056D00ADB2290A2046FFF736
:10A0B0006DFF05F0FE012046FFF768FF20467F2177
:10A0C000FFF764FF2046FF21FFF760FF2046FF21D6
:10A0D000FFF75CFF2046FF21FFF758FF2046FF21D6
:10A0E000FFF754FF2046FF21FFF750FF2046FF21D6
:10A0F000FFF74CFF2046FF21FFF748FF2046FF21D6
:10A10000FFF744FF2046FF21BDE838403EE700BF8F
:10A11000941A002010B57F210446FFF737FF204630
:10A120000021FFF733FF2046FF21FFF72FFF2046D6
:10A13000FF21FFF72BFF2046FF21FFF727FF2046D7
:10A14000FF21FFF723FF2046FF21FFF71FFF2046D7
:10A15000FF21FFF71BFF2046FF21FFF717FF2046D7
:10A16000FF21FFF713FF2046FF21FFF70FFF2046D7
:10A17000FF21FFF70BFF2046FF21FFF707FF2046D7
:10A18000FF21FFF703FF2046FF21FFF7FFFE2046D8
:10A19000FF21BDE81040F9E62DE9F043BF4CC04D6A
:10A1A00094F850302E6883B033B1206820B194F811
:10A1B0005130013B012B02D903B0BDE8F083B94F08
:10A1C0004FF001094FF0000808E01B2B00F06E82F1
:10A1D0000D2B00F0528287F80090206803685B68BE
:10A1E0009847002837D020680368DB68984783B217
:10A1F0007E2B2A6828D039780029EED194F8522095
:10A20000002AE2D07D2B00F04E8294F856E0BEF199
:10A21000000F04D080F02003DBB284F85610511CEC
:10A22000C9B22244092984F85210137100F0318216
:10A230000829D2D8B4F85420134403EB132303F0B5
:10A24000FF03A4F85430C8E784F8528084F85380A0
:10A2500087F80080C1E794F857302BB1637984F810
:10A260005700302B00F0F38294F853E08E4A8F4968
:10A27000DFF850C28E4F94F8688194F87A31BEF1BD
:10A28000000F99D0B8F1000F40F01A822868801BA7
:10A29000012846D832F8130000283CD00133B0F52D
:10A2A000826FDBB200F0CF8143D9B0F5E26F00F0EE
:10A2B0000B816BD9B0F5046F00F02281B0F5116FFE
:10A2C00000F0A681B0F5E46FE0D17A4A84F87A31E3
:10A2D000916B1289642303FB01F3202593FBF2F3B6
:10A2E00007224FEA132E1F0C1E0E694610208DF810
:10A2F00002308DF803E08DF804708DF805608DF85C
:10A3000000508DF80120FFF7F1FD002384F8533051
:10A3100003B0BDE8F0832868801B01284FF00103DB
:10A32000B8D9002284F87A3184F8532003B0BDE80C
:10A33000F083B0F5007F00F0448152D8B0F5807F03
:10A3400000F0ED80B0F5887FA0D1386884F87A31CC
:10A35000430790D5584B1B688DF8023010221F0A16
:10A3600023FA02F61B0E1046012569468DF803708C
:10A370008DF804608DF805308DF800208DF80150BF
:10A38000FFF7B4FD002384F8533015E7B0F5C06F34
:10A3900000F02D81B0F5E06F7FF478AF454A84F886
:10A3A0007A31116B1289642303FB01F3002593FBBF
:10A3B000F2F307224FEA132E1F0C1E0E69461020DF
:10A3C0008DF802308DF803E08DF804708DF805608B
:10A3D0008DF800508DF80120FFF788FD84F8535068
:10A3E000EAE6B0F5047F00F0BA80B0F5806F7FF444
:10A3F0004DAF94F8842184F87A31531CDAB2032AE1
:10A4000000F2418142F2107384F8842103FB02F3CD
:10A410002A4A1278D70748BF0133960748BF02334C
:10A420005507274A128848BF0433D00748BF0A336C
:10A43000910748BF1433170648BF2833D60548BFD5
:10A440002833550748BF6433100748BFC833910508
:10A4500048BF03F5C873970648BF03F57A73D6065D
:10A4600048BF03F5FA63550648BF03F57A63002534
:10A470001E0A0422694610208DF802308DF8036010
:10A480008DF800508DF804508DF805508DF801209E
:10A49000FFF72CFD84F853508EE600BFC81F002044
:10A4A000EC1900208200002064530308504F002064
:10A4B000601B0020F81900203C1A0020744F002077
:10A4C000061B0020544F0020CC4A84F87A31506B90
:10A4D00011896423102203FB00F393FBF1F34FEA8D
:10A4E000132E23FA02F71E0E104607258DF80230B0
:10A4F00069468DF803E08DF804708DF805603BE740
:10A50000BF4A84F87A31B2F9043003EB83035B006D
:10A510004FEA132E1F0C1E0E40250822E5E6386870
:10A5200084F87A3140077FF5A6AEB64B9B698DF86B
:10A5300002301F0A1E0C00251B0E01226946102046
:10A540008DF803708DF804608DF805308DF800509B
:10A550008DF80120FFF7CAFC84F853502CE60868F8
:10A5600084F87A3183077FF586AE9CF800000028D6
:10A570003FF481AED4F88031DB7B002B00F0EB8020
:10A58000A14B1B8893FBF0F303EB83035B001022CA
:10A590004FEA132E23FA02F71046022600256946D9
:10A5A0008DF802308DF803E08DF804708DF80020EE
:10A5B0008DF801608DF80550FFF798FC84F8535032
:10A5C000FAE5086884F87A3110F0082F3FF453AEAA
:10A5D0008E4A8F49126881FB0231D317C3EBA10366
:10A5E0004FEA132E1F0C1E0E00250222E6E6086815
:10A5F00084F87A3110F0082F3FF43DAE854B1B688C
:10A600008DF802301F0A1E0C00251B0E062295E74E
:10A61000086884F87A3183077FF52DAE9CF80080B6
:10A62000B8F1000F3FF427AE774B1B88102203EBE5
:10A6300083035B00104693FBF8F309264FEA132EC1
:10A6400023FA02F7AAE7386884F87A3110F0200874
:10A650007FF411AE0B68180600F1E480D4F8803165
:10A660005B7C002B3FF407AE94F88531032B00F29E
:10A670007781DFE803F0B8AE9F7684F852902371BB
:10A68000A4F85420A9E5012384F8843142F2107320
:10A69000BEE6B4F85420C2F1FF0293427FF49BADB2
:10A6A00084F8579097E584F8569096E520680368FB
:10A6B0005B68984700287FF48EAD84F853908CE552
:10A6C0002A68961B012E3FF62CAED4F85C31DFF8D9
:10A6D000509194F87B214B4500F01281511C94F865
:10A6E0007C51D4F8607184F87B1102F00F028DF870
:10A6F00000200DF10102F91A00296E460DF1060E37
:10A7000002DC12E0002829DD0133C4F85C3113F8C3
:10A71000011C02F8011B7245A7EB030085EA010545
:10A72000F0D384F87C5100F03481501C70451570D2
:10A7300005D202AB9A1A033A002129F0BEFF314636
:10A740003220FFF7D3FB4FF00008002384F8688124
:10A7500084F8533030E52C4B1B8815E784F87C5186
:10A76000E3E72D4B1A6853799179D27903F140735D
:10A7700003EB012303EB0243002284F8852110221E
:10A780001F0A23FA02F61D0E4FF0040E104669460A
:10A790008DF802308DF800208DF801E08DF80370FF
:10A7A0008DF804608DF80550FFF7A0FB002384F8B6
:10A7B000533001E5194A11688A7D487D097D1204EC
:10A7C00002EB00220A44591C84F8851102EB036352
:10A7D000D5E7124A11680A7BC87A897A120402EB1B
:10A7E00000220A44EFE70D4A11688A784878097810
:10A7F000120402EB00220A44E5E700BFF81900202A
:10A80000601A0020401A0020941A00209C1A002090
:10A8100067666666A01A0020E47F002048390020A1
:10A820002420002010230422184669468DF8028057
:10A830008DF803808DF804808DF805808DF8003048
:10A840008DF80120FFF752FB84F85380B4E4A3791C
:10A850005A09012A73D103F00F0C13F0100300F012
:10A860008980684FE37994F808E0A4F87601F91834
:10A870008EEA030084F858203B46C4F86C71C4F893
:10A880007011FA1F84F87801A4F874E194F8780143
:10A89000DFF880E103E0D4F87011D4F86C3199420C
:10A8A00003F1010708D012F8011BC4F86C7172455E
:10A8B00080EA01001970EED3724584F8780108BF70
:10A8C00084F879C13FF4D0AC127894F878319A4288
:10A8D00064D04D4BB4F87401C4F85C3101220133EB
:10A8E00000274FF6F671C4F8603184F85870A4F868
:10A8F000640184F85C2084F86821A4F86611B3E44C
:10A90000D4F86071B4F9661194F86451501CA7EB47
:10A91000090902F00F0242F01002002989EA050538
:10A92000B8BF42F02002EDB28DF8002084F87B0120
:10A930008DF8019084F87C510DF10202DBE6324B78
:10A94000324984F858005F1C012284F85C00C4F886
:10A950005C31C4F86071C4F8641184F8682183E440
:10A960005A1CD2B2042A84F885214FEA03637FF48B
:10A9700006AF01E794F85820002A3FF475AC94F82C
:10A980007921013202F00F0262452DD084F858304F
:10A990006AE431463220FFF7A9FAD6E6194BD4F81B
:10A9A0006C21C4F87021002703F5A672114603F14B
:10A9B0004C09C4F8602103F5AE703A46C4F85C91C6
:10A9C000C4F86C3184F85870C4F86471F8F7C6FEA6
:10A9D00001300FD0D4F85C31C4F860310123C4F8E1
:10A9E0005C9184F868313FE4D4F87011D4F86C318C
:10A9F000074A4BE7D4F85C310222591CC4F85C11B9
:10AA00001A70E7E7D81F0020242000200000F6FF7E
:10AA1000CF1F0020D41F00205E2810B515D05D2860
:10AA2000014606D00F4B18680368BDE810401B684C
:10AA300018470C4C206803681B6898472068036817
:10AA40003D211B68BDE810401847064C206803688C
:10AA50005D211B689847206803683E211B68BDE89C
:10AA600010401847381A002070B5074C23681A6840
:10AA700005465E21184612689047206803682946FB
:10AA80001B68BDE870401847381A00202DE9F84FC0
:10AA9000754C764F764994F9005094F90C0094F96E
:10AAA00018E094F9246094F9308094F93CC094F94A
:10AAB00048A094F954903A6800230B700133DBB23C
:10AAC000FAB1118811F0010F1BD011F03C0F18D012
:10AAD00092F90210A9421CD0814200F0B280714567
:10AAE00000F0A380B14200F0A880414500F0A180B1
:10AAF000614500F0B280514500F0AB80494500F05F
:10AB0000A480082B02F10802D8D1594A1370BDE87D
:10AB1000F88F5749544A0B705668002E00F0A180F8
:10AB2000544D2B68B34253D0D5F8CC30B34246D005
:10AB3000D5F89831B34239D04D4B3A681B7894F927
:10AB4000001094F90C0094F9186094F924E094F939
:10AB500030C094F93C8094F9489094F954A002EBE9
:10AB6000C3021DE00133DBB2CAB1B2F800B01BF082
:10AB7000010F14D01BF03C0F11D092F902B05945CF
:10AB80002FD0834535D0B34537D0F34539D0E34591
:10AB90003BD0C3453DD0CB453FD0D34541D0083213
:10ABA000072BDFD9324A1370BDE8F88F304611F019
:10ABB00009FDCC220021304829F07FFDBCE730465A
:10ABC00011F000FDCC2200212C4829F076FDAFE7E2
:10ABD000304611F0F7FCCC220021264829F06DFD0B
:10ABE000A2E72349204A0B705668002E99D1BDE890
:10ABF000F88F1F4A1370224AF6E71D4A1370214A44
:10AC0000F2E71B4A1370204AEEE7194A13701F4AF5
:10AC1000EAE7174A13701E4AE6E7154A13701D4A01
:10AC2000E2E7134A13701C4ADEE7114A1370154A13
:10AC300072E70F4A1370154A6EE70D4A1370124AF5
:10AC40006AE70B4A13700E4A66E7094A1370124A04
:10AC500062E7074A13700F4A5EE7054A13700C4A11
:10AC60005AE7BDE8F88F00BF2088002084880020C4
:10AC700080880020986A0020306C0020646B0020DF
:10AC80002C8800203888002044880020508800202C
:10AC90005C880020688800207488002070B5BA4C59
:10ACA000D4F8883182B033B11A88550603D512F42E
:10ACB000057F40F0368194F88C21022A00F026812D
:10ACC000A2F10102B2FA82F25209B04D2978914202
:10ACD00028D0002A40F04C82AD48AE4B01685E6837
:10ACE000B14200F0D3811A69914200F08782DA699B
:10ACF000914200F08B829A6A914200F08B825A6BEB
:10AD0000914200F08D821A6C914200F08D82DA6CD3
:10AD1000914200F091829A6D914200F0B681002339
:10AD200003602B7094F88D21022A00F00D81A2F1AE
:10AD30000102B2FA82F25209974D2B78934228D041
:10AD4000002A40F08C819548924B01685E688E42E3
:10AD500000F006811A69914200F03682DA69914268
:10AD600000F036829A6A914200F036825A6B914224
:10AD700000F038821A6C914200F03682DA6C91420F
:10AD800000F036829A6D914200F0E9800023036062
:10AD90002B7094F88E21022A00F02D81A2F101027D
:10ADA000B2FA82F2520994F8503093422AD0002A23
:10ADB00040F02C81774B21685868814200F0DA809E
:10ADC0001A69914200F00282DA69914200F002822F
:10ADD0009A6A8A4200F002825A6B8A4200F000822C
:10ADE0001A6C8A4200F00282DA6C8A4200F0028217
:10ADF0009A6D914200F0BD800023236084F85130A9
:10AE000084F85030D4F8941131B10B88580603D52A
:10AE100013F4057F40F0D28094F89821022A00F0C4
:10AE20005281A2F10102B2FA82F252095C4D2B78F2
:10AE3000934228D0002A40F082815A48554B01683D
:10AE40005E68B14200F02C811A69914200F0D48111
:10AE5000DA69914200F0D6819A6A914200F0DC8171
:10AE60005A6B914200F0DE811A6C914200F0DE8153
:10AE7000DA6C914200F0DE819A6D914200F00F8110
:10AE8000002303602B70D4F89C1131B10B885A0653
:10AE900003D513F4057F40F0A08094F8A021022A86
:10AEA00000F01A81A2F10102B2FA82F252093E4C7C
:10AEB0002378934228D0002A40F026813B48354B26
:10AEC00001685D68A94200F0F5801A69914200F0BE
:10AED0009781DA69914200F097819A6A914200F075
:10AEE00097815A6B914200F099811A6C914200F05F
:10AEF0009F81DA6C914200F0A1819A6D914200F03D
:10AF0000D88000230360237002B070BD284A126805
:10AF10001278002A40F0E980264A1278C2F38002B3
:10AF2000D3E61A4B1A78002A7FF4FCAE224A126844
:10AF3000002A3FF4F7AE1648026094F88D210121F3
:10AF4000022A19707FF4F3AE194B1B681B78002B93
:10AF500040F02A81174B1A78C2F38002ECE60722F0
:10AF600002EB420203EB82030022CA621A815A609A
:10AF70000CE7072202EB420203EB82030022CA62C3
:10AF80001A815A6038E700BFC81F0020E819002066
:10AF9000381A002020880020A41A0020E41A00207B
:10AFA000FE1A0020309100204A1B00204C1B00207C
:10AFB0001C260020744F0020D4730020A04B1A7868
:10AFC000002A7FF460AF9F4A1268002A3FF45BAF0B
:10AFD0009D4801210260197055E79C4B1A78002AA0
:10AFE00092D1984A1268002A8ED0994801210260B5
:10AFF000197002B070BD974B1B681B78002B40F096
:10B00000D880954B1A78C2F38002CCE6D4F8903100
:10B01000002B3FF4F7AED4F8802193F90200937827
:10B020005178002B15BF0822002209230123002993
:10B0300008BF134603228DE80C0020214FF4614322
:10B04000002211F0F3FA206000283FF4DBAE834ABF
:10B050000123126884F8513084F85030D2E6804BD6
:10B060001B68002B3FF495AE012693F90200009671
:10B070004FF496430022082121F01AFA794B186008
:10B0800000283FF486AE2E7083E6072202EB4202D0
:10B0900003EB82030022CA621A815A603FE607224C
:10B0A00002EB420203EB82030022CA621A815A6059
:10B0B000E6E6072202EB420203EB82030022CA62A9
:10B0C0001A815A601DE7634B1B681B78BBB9624B42
:10B0D0001A78C2F38002A9E65E4B1B681B784BB955
:10B0E0005D4B1A78C2F38002E1E65F4A1268C2F350
:10B0F000C042EAE55C4B1A68C2F3C042D7E65A4B3D
:10B100001A68C2F3C04291E600293FF4FDAE8B7984
:10B11000002B56D0554A52F8233091F902000222F2
:10B1200000924FF40071002221F0C2F9484B1860E0
:10B1300000283FF4E9AE0123237002B070BD00295E
:10B140003FF4A1AE8B79002B38D0484A52F8233017
:10B1500091F90200022200921021002221F0A8F9A8
:10B16000394B186000283FF48EAE01232B708AE61D
:10B17000002B3FF4D7AD3E4A93F9020013685B7889
:10B18000003318BF012302228DE80C0004214FF484
:10B190001653002211F04AFA364B186000283FF48B
:10B1A000C1AD01232B70BDE52F4B1A68C2F3C0421D
:10B1B000C2E52D4B1A68C2F3C042F4E54FF4964342
:10B1C000C6E74FF46143A8E70122C9E60122D1E6B0
:10B1D0000222C5E60222CDE60322C1E60322C9E629
:10B1E0000422C7E60422BBE60522B9E60522C1E631
:10B1F0000622B5E60622BDE6012251E7012245E717
:10B20000012257E702224BE7022253E702223DE7E1
:10B2100003224FE7032239E7032241E7042249E7EB
:10B22000042233E704223BE705222FE7052237E714
:10B2300005223FE7062233E7062227E7062239E701
:10B24000FE1A0020D4730020309100204A1B0020F9
:10B250004C1B00201C260020744F0020EC190020FD
:10B26000F81A0020E41A0020681A00204477030826
:10B27000981A0020381A0020038813F0400004D0E8
:10B2800013F4057F14BF012000207047F8B5414E2C
:10B29000414B32681A60042011F0F8FA3F4C404DDF
:10B2A000C4F88801042111F0E7FA3E4B326884F8B3
:10B2B0008C0108201A6011F0E9FA3B4B0821186054
:10B2C00011F0DAFA2C2284F88D010021284629F0A9
:10B2D000F4F93368C4F88031E0227D238E217C2686
:10B2E0002020EA7085F82B302E70697011F0CEFAAC
:10B2F0002021C4F8900111F0BFFA84F88E011020CB
:10B3000011F0C4FA1021C4F8940111F0B5FA274BDA
:10B3100084F898013B221A70A42100223A209F272A
:10B320001E2618719F711E7259729A72DA721A7300
:10B3300001254FF400705D7011F0A8FA4FF4007110
:10B34000C4F89C0111F098FA194B1A491B680E6851
:10B35000194F1A4A84F8A001191C18BF012139702D
:10B3600031064FF0040348BF08214FF0020048BFE8
:10B37000D170507093701570114A124912681248BA
:10B3800058BF03230B70003218BF0122BDE8F840FC
:10B39000027083E41C260020981A0020C81F002099
:10B3A000AC1A0020DC1A0020F81A00208C180020AB
:10B3B000B01C0020504F0020AC1C0020BC1C002002
:10B3C0006C740020E91C0020EA1C00202DE9F04FDD
:10B3D000C04BDFF804B31B6889B01A460293002300
:10B3E00042F820300C4601251F461E469846019320
:10B3F0009A462378039005F1FF3EA9462C225FFA76
:10B400008EFE002B00F08C809A4200F037818DF880
:10B4100014306378611C002B00F038819A4200F0F0
:10B4200037818DF81530A378A11C002B00F03281F4
:10B430009A4200F031818DF81630E378E11C002B40
:10B4400000F02C819A4200F02B818DF8173023797F
:10B45000211D002B00F026819A4200F027818DF8F3
:10B4600018306379611D002B00F022819A4200F0B0
:10B470001B818DF81930A379A11D002B00F01A81D2
:10B480009A4200F019818DF81A30E379E11D002B02
:10B4900000F014819A4200F013818DF81B30237A5A
:10B4A00004F10801002B00F00D819A4200F00C819C
:10B4B0008DF81C30637A04F10901002B00F006813D
:10B4C0009A4200F005818DF81D3004F10A01A37A3B
:10B4D0000A2408A804449A424FF0000004F80C0C17
:10B4E00040F091800EF1FF3E4C1CBEF1030F03D8DB
:10B4F000DFE80EF0694C196E05A826F07DFD042DDD
:10B5000082466AD80BEB0503013593F82420237893
:10B51000EDB205F1FF3E5FFA8EFE002B7FF474AFB3
:10B5200021461C46D5E79DF8143005AA1BBBE9E768
:10B53000462B72D0412B78D04C2B00F08E80532BB1
:10B5400000F09880472B00F09780522B08BF06260A
:10B55000542B16D04F2B5BD0422B68D04E2B71D082
:10B56000492B00F08280572B08BF05230AD012F820
:10B57000013F002BC6D0432BDAD1542B4FF00006ED
:10B58000E8D1002309FA03F31F43F0E79DF81430D4
:10B5900005AA83B9B6E7452B41D0532B4CD0572B86
:10B5A00055D0552B5BD0442B08BF052306D012F88D
:10B5B000013F002BA6D04E2BEDD1002309FA03F357
:10B5C00048EA0308F3E705A826F016FD019099E77D
:10B5D00005A826F011FD0F2818DD0022019B039914
:10B5E00003F00F0343EA8853134343EA06234FEA69
:10B5F0000A12D2B243EA07331343029A42F82130C7
:10B6000013F0CCFF012009B0BDE8F08F8204E5E71C
:10B61000012309FA03F31F43A9E7012698E7012351
:10B6200009FA03F348EA0308C1E7022690E7022378
:10B6300009FA03F31F439AE7022309FA03F348EADE
:10B640000308B4E7032309FA03F31F438FE7032337
:10B6500009FA03F348EA0308A9E7032678E7042375
:10B6600009FA03F348EA0308A1E7042309FA03F3FC
:10B670001F437CE704266BE7052669E72146002384
:10B6800008AA1344002203F80C2C2BE7012420E71E
:10B690000123F5E702241CE70223F1E7032418E75E
:10B6A0000323EDE7042414E70523E9E70423E7E790
:10B6B00005240EE706240CE70623E1E7072408E744
:10B6C0000723DDE7082404E70823D9E7092400E776
:10B6D0000923D5E778250020645303082DE9F041BC
:10B6E000614C236894B0F3B113F058FF23685F4CAA
:10B6F00093F8F1505E4B012704F5D27040F22A32E4
:10B7000000211F7028F0D9FF9DB95A4B002003F18A
:10B710008001FF2218809A70DA7004339942F9D1BF
:10B7200094F8603513B114B0BDE8F08122F02EFF1B
:10B73000F9E7284612F022F9C3680268C4F8D02459
:10B740000646002BE1D0284601F066FF00254FF0A9
:10B75000280880F80680C571327AC4F8D4042E21F6
:10B7600002F01EF82A464146307C24F067F8602239
:10B770004149307C12F08CF8D4F8D00404F08CFAF3
:10B7800011F000FF14A9022341F84C3DD4F8D00475
:10B7900003951D23029312F09FF8059506950795D2
:10B7A0000895F379602204925A0755D50422ADF822
:10B7B0001620002504A903F00203D4F8D004ADF844
:10B7C0001C3006951AF002FFD4F8D034F0689A695C
:10B7D000C4F8D80442F008029A615A6C42F400425C
:10B7E0005A641AF073FC09A81AF042FCD4F8D03459
:10B7F0007079224A0A923433034440F22A304FF4DB
:10B80000007209A94FF0100E0993ADF830004FF403
:10B8100000538027D4F8D8040F920D9510951195F8
:10B8200013951293CDF82CE00E971AF02FFC737934
:10B83000D4F8D0140C2B9CBF114A32F81350CB68AB
:10B84000D4F8D8242B43CB601368012143F00203C2
:10B85000136084F8DC1458E74FF48072ADF814706C
:10B86000ADF82020A5E700BF78250020C81F0020E4
:10B8700080250020A8240020F9F502086C21002072
:10B8800028700308F0B40A4E054606F13007344626
:10B890000FCCBC4228606960AA60EB60264605F1C7
:10B8A0001005F4D103CE28606960F0BC704700BF7A
:10B8B000905303080F2A05D8052805D9062818D063
:10B8C00007280ED0002070470529FBD80D4B1B68B8
:10B8D00000EB400003EB40000144012081F8C02050
:10B8E00070470029EED1074B1B68012083F8F02038
:10B8F00070470A29E6D8034B1B681944012081F8D8
:10B90000E4207047782500201F4B2DE9F041DFF837
:10B910007C801E680D4600F120070024284626F092
:10B920006BFB38F814209042034627DC012C11D021
:10B93000022C28464FF02C0104F1010418D026F8FF
:10B94000273028F024FF451CC0B1032CE6D101208C
:10B95000BDE8F08106EB8702284693702C2128F081
:10B9600016FF58B1013026F047FBFF28034605DCDF
:10B9700006EB87060120F370BDE8F081002046F851
:10B980002700BDE8F08100BF78250020C8530308D8
:10B9900010B50D4B0D4A1B780D48303353700D4BCD
:10B9A0000D4A1978742301FB0323002213F8014F79
:10B9B000145411189C7A4C7003321C7D8C70092A27
:10B9C000F4D1002010BD00BF0E1F00207A0000201F
:10B9D000841F0020021F0020F7490020034B044A67
:10B9E0001B78013B13700020704700BF141F00201C
:10B9F000221F0020034B044A1B78013B13700020D8
:10BA0000704700BF0E1F0020021F0020064B074A90
:10BA10001B7882F8E035742101FB0323044A127875
:10BA200083F8D02400207047021F002074450020B6
:10BA3000221F0020094A0A4992F8E0350B70094993
:10BA4000581C0870742101FB0323074A93F8D03473
:10BA50001370064A013313700020704774450020AC
:10BA6000021F00200E1F0020221F0020141F002094
:10BA700010B5084808490022135CA3F16104052CA5
:10BA80009CBF203BDBB28B540132072AF4D100204B
:10BA900010BD00BFC68403088425002070B5184B74
:10BAA0001B78012B17D8174BDD79174B93F8C2166B
:10BAB00083F8C45621B193F8C3260AB191420CD33E
:10BAC000012283F8C22683F8C32625B1022D1CBFAC
:10BAD000002283F8C426002070BD1446084634B105
:10BAE00090FBF4F604FB160620463446F7E791FB7C
:10BAF000F0F192FBF0F283F8C21683F8C326E4E774
:10BB000048680020842500207445002030B50B4B88
:10BB10009A68002115794C1C0E2DE4B20AD10278E6
:10BB20001973501E8842DCBF023A1A731A7B013A1D
:10BB30001A7330BD14322146ECE700BF8425002083
:10BB400070B54469054623790E2B04D12B694BB19E
:10BB5000BDE870401847032B02D1E068FFF7F0FF03
:10BB60001434F0E770BD064B30B11A691860013229
:10BB70001A6105221A75704704221A75704700BFB2
:10BB80001487002008B5074B5A7B2AB19B7B4FF4E2
:10BB900000201BB102F05AFC002008BD02F04EFC50
:10BBA000FAE700BF84250020F7B5324E96F8C43678
:10BBB000022B56D11AF086F9044620BB2E492F4895
:10BBC0002F4D28F0F2FD23462E4F2F4A00950821D5
:10BBD00007F1170028F07AFD234600952A4A08212C
:10BBE00007F11F0028F072FD96F8C436FB717B7BCD
:10BBF00033B9264B1B68C3F3C043BB7301237B736C
:10BC0000002003B0F0BD224D95F8244034B92149FD
:10BC10001A481B4D28F0C9FD2346D5E71E4C637812
:10BC2000022B14D0032B1AD11C49144828F0BDFD57
:10BC300041F278134FF4FA62E4584FF47A23B4FBDC
:10BC4000F3F4EB6B0E4DB3FBF2F31B1BBCE7144993
:10BC50000A480B4D002428F0A8FD2346B4E70D49FF
:10BC6000F6E710490548104D002428F09EFD2346B4
:10BC7000AAE700BF74450020D18403089325002063
:10BC8000CE84030884250020EE840308504F002052
:10BC90005C7F0020D9840308784F0020DF840308EC
:10BCA000E5840308EA840308CF840308234B9A6AD7
:10BCB000D2682DE9F04105461C4682BB94F82C3031
:10BCC00053B3284602F01AFA94F82C30013BDBB249
:10BCD00004EB830284F82C302344176B93F85860EC
:10BCE0007B69A36004354FFA86F82846A76284F87A
:10BCF0002D80FFF70BFF237B98450DDD7A69626687
:10BD0000142103FB0111DB430A4433442846A2609B
:10BD100084F82D30FFF7FAFE0020BDE8F08193F99A
:10BD20002D009B6800EB800003EB8000904700280B
:10BD3000C4DA4FF0FF30BDE8F08100BF8425002059
:10BD4000F8B5054649B3164CA06A81421AD094F85A
:10BD50002C20144FA16204EB8203A61818634069DB
:10BD6000A3681B1A94F82D009B1007FB030386F8A9
:10BD70005830002384F82D308B68013284F82C2051
:10BD800003B19847A36A5B69A360284600236366F2
:10BD900002F0B4F9281DFFF7B9FE0020F8BD00BF7E
:10BDA00084250020CDCCCCCC2DE9F04FB74A81467C
:10BDB0001068002889B04DDBB54DAA6E02F54342EC
:10BDC00050324A4546D895F86C80C5F868904FF4D3
:10BDD0007A72B9FBF2F20192AE4AB8F1000F3CD18F
:10BDE000D388A3F2E3439BB2B3F5F97F2FD8B2F91E
:10BDF000041040F2E143994229DCB2F9022040F2FA
:10BE0000D6639A4223DDA4490B7813F004041ED1B3
:10BE100040B1A24A10680028B8BF1460126805EB50
:10BE20008202106FC5F880009D4C68B1012223F09A
:10BE300001030B7085F86C20AC6202F051F9A96A1D
:10BE4000D5F88000FFF77CFF4FF4FA732383019B42
:10BE5000C5F8843009B0BDE8F08FD188904FA1F2C9
:10BE6000E34189B2B1F5F97F10D8B2F9040040F28C
:10BE7000E14188420ADCB2F9020040F2D661884210
:10BE800004DD85490978480740F17E83B2F9020054
:10BE900040F2D661884200F39D8340F2E144A04223
:10BEA00040F39A83B2F90000A04240F3978388429E
:10BEB00000F396839288A2F2E24292B2B2F5FA7F40
:10BEC00000F29083012200243A62C5F888405EE3C4
:10BED000002C00F068833A6AD5F88060029204F181
:10BEE000FF3B4FF0000A5FFA8BFB029A524524DCBD
:10BEF000033C012C3B8300F25683FA69142A40F379
:10BF00005283A2F1140193FBF1F31BB2322B3B835A
:10BF100000F34983D5F888300BB9C5F88820D5F8E7
:10BF20008830D21A5E4B186A052192FBF1F2024466
:10BF30008A42C8BF0A461A6235E3AB6A0BB9FA23D4
:10BF400084E0052C05D13046FFF7B0FE4FF4FA73BC
:10BF50007CE0022C42D195F92D302A7B93422DDAD8
:10BF6000013385F82D30BBF1010FE8D995F92D305B
:10BF7000AA6803EB830302EB83031A79013A0C2AC4
:10BF8000DDD801A151F822F047BF000873C00008B6
:10BF90003BC0000853C00008A5C0000879C10008D4
:10BFA000FBC00008A5C10008D5C100083FBF0008BC
:10BFB000FBC00008C7C0000841C100086B6E4BB150
:10BFC000304602F09BF86B6EAA686A66301DAB6063
:10BFD000FFF79CFD002385F82D30C4E7012CC2D16A
:10BFE00095F82D10AA684B1E5BB203EB830002EBA1
:10BFF000800085F82D30007920B9002BC4BF0239AC
:10C0000085F82D1095F92D30591C06D003EB8303CC
:10C0100002EB83031B79002B91D16B6E4BB1304641
:10C0200002F06CF86B6EAA686A66301DAB60FFF7B1
:10C030006DFD2B7B85F82D3095E7042C7FF47FAFC9
:10C04000D9683046FFF77CFE4FF4FA730AF1010A13
:10C050004BE79A68002A3FF472AF042C7FF46FAF6D
:10C06000D9683046904701303FF46DAF4FF4FA7312
:10C07000ECE79A68002A3FF462AF042C7FF45FAFCC
:10C08000D968304690474FF4FA73DFE73025002037
:10C09000842500206C1A0020744F002084000020AA
:10C0A00088000020DA68002A3FF449AFA4F1040CAC
:10C0B000DCF1000141EB0C0111701A7C42F001022D
:10C0C0001A74FA23C2E7D96800293FF438AF042C68
:10C0D0000A8809D142F4006292B20A801A7C42F0C6
:10C0E00001021A74FA23B1E740F6010092FBF0F066
:10C0F00000EBC020121A92B2EFE7DA68002A3FF490
:10C100001EAF1168042C087812D192F805E086451C
:10C1100002D99279104408701A7C42F001021A7414
:10C120009A68002A3FF40BAF19463046904706E75D
:10C1300092F804E08645EFD29279801A0870EBE716
:10C14000D8680268042C117811D10079884201D98D
:10C15000013111709A6822B1D96803933046904733
:10C16000039B1A7C42F001021A74FA236EE700293D
:10C17000F0D001391170EDE7DA68002A3FF4DFAE44
:10C180001168042C91F9000007D192F905E0864569
:10C19000C2DD927902440A70BEE792F904E0864556
:10C1A000BADAC9E7DA68002A3FF4C9AE1168042C8C
:10C1B000088807D1B2F806E08645ADD91289104447
:10C1C0000880A9E7B2F804E08645A5D21289801A52
:10C1D0000880A1E7DA68002A3FF4B1AE1168042CA8
:10C1E000B1F9000004D1B2F906E0864594DDE5E737
:10C1F000B2F904E086458FDAE8E72A7B3B799B1A9F
:10C20000022293FBF2F3013BDBB20293D5F89030AC
:10C2100003F5C333A03399453B6888BFC5F89090B8
:10C220009B6A384698BF4FF000089847BB791FFAC1
:10C2300080F9002B00F08E80A868002201460B795F
:10C240000E2B02F101047ED13B79D2B2591E9142EC
:10C2500009DC142202FB0303283B6B661B790E2BBF
:10C2600004BF00236B660023BB71A86895F82D30CE
:10C2700059B201EB810200EB820201331279DBB289
:10C28000002AF5D097F9072085F82D10002A0BDB3E
:10C290008A4220D0029B1A44D2B2B64B01213846C2
:10C2A00001F016FFA9EB0009B9F11D0F40F28181E1
:10C2B00095F92D2097F90730934210D0029B1A442C
:10C2C000D2B2AD4B0121384601F002FF95F82D3076
:10C2D000FB71A9EB0009B9F11D0F40F26A81AC684E
:10C2E000002614343B79F2B2023B9A4246DBAE6838
:10C2F0004FF0000B14363B795FFA8BF8023B984500
:10C3000080F2578116F8103C0E2B00F0528116F87F
:10C31000042CD10740F19180029988445FFA88F893
:10C320000D2B00F22381DFE813F017012101210119
:10C330005A005A009000CC00BC00D500D5004D003A
:10C34000DD00AF00A5000A7C42F003020A7414313C
:10C35000224674E7B8F1000F87D02B7BAA6803EB65
:10C36000830302EB83039A423FF67FAF117C4C07B5
:10C3700044BF41F0010111741432F4E714F8103C89
:10C380000E2BB4D014F8041C880718D5002B029B80
:10C390001A4418BF032154F8143C08BF0221D2B23A
:10C3A000384601F095FE14F8043CA9EB000923F08F
:10C3B0000203B9F11D0F04F8043C40F2FA80013683
:10C3C00014348FE756F8083C002B00F0CF807979C1
:10C3D00008394246C9B2384601F07AFE43E097F880
:10C3E00005A0032BAAF1080A2BD156F80C0C50B368
:10C3F00012F008040DD080475FFA8AF103460390DB
:10C400004246384601F064FE0446039823F088FB58
:10C4100082445A4B42465FFA8AF1384601F058FE90
:10C4200016F8043C23F00103204406F8043CA9EB71
:10C430000009B9F11D0F40F2BC800BF1010B14365D
:10C4400059E70024E5E70446E3E756F8080C00281E
:10C45000EDD07979037808390BB3494B4246C9B21C
:10C46000384601F035FE16F8043C23F0010306F8C7
:10C47000043CDCE756F8083C79791A689B68127826
:10C48000083953F82230A4E756F8080C0028CED01B
:10C490000388797913F4006FA1F10801DDD1394BDC
:10C4A00097E756F8080C0028C1D00368187805A94A
:10C4B00011F0E6FC05A820F0F5F9797905AB08390B
:10C4C00087E756F8080C0028B1D0036805A993F94E
:10C4D0000000EDE756F8080C0028A8D0036805A96D
:10C4E0001888E5E756F8080C0028A0D003680089F2
:10C4F0001B78584300F5C33005A9A03011F0C0FCEB
:10C500009DF816209DF815308DF815202E228DF8F7
:10C5100016209DF819208DF81430302A01D02E2ACB
:10C520000DD14FF000028DF819209DF81820302A07
:10C5300001D02E2A03D14FF000028DF81820302BA5
:10C5400008BF202305A808BF8DF8143020F0AAF9F1
:10C55000797905AB09393CE756F8084C44B156F8EF
:10C56000140C23F0DDFA2346C11C32E700205EE7FD
:10C5700020465CE7F4840308F7840308F884030882
:10C58000FA840308FE8403080624FA690132FA617A
:10C59000B7F91820002A7FF79BACD5F884301344F4
:10C5A000019A9B1A3B83AB68D5F88070002B7FF40F
:10C5B00024AED5F88C30019A03F5FA739A427FF6CF
:10C5C00046ACD5F8800003681B6A9847019BC5F804
:10C5D0008C303CE40124D8E70224D6E70324D4E7D6
:10C5E0000424D2E70524D0E7F8B504460E461A4DD8
:10C5F000E1B101F083FD03220521184B204601F033
:10C6000067FD236820465B6A984718F0CDFB18F059
:10C610001BFBC82003F024FE1148FFF791FAAB6A18
:10C62000DB680BB10020984702F044FB2368002729
:10C630005B6885F86C7020469847237AAF62013BAF
:10C64000237216B1074B084ADA60084A137843F0A0
:10C65000010313700020F8BD842500200285030823
:10C660008800002000ED00E00400FA05744F00206F
:10C6700050B110B5064C606020F0D8F802234FF698
:10C68000FF722375A28110BD014A1075704700BF6B
:10C6900014870020064B1A68042A07D0511C196021
:10C6A000044B03EB8203186701207047002070479A
:10C6B000302500208425002070B50446006800F174
:10C6C00020033F2B4BD800F108030F2B2BD8811CE4
:10C6D000032994BF00210121636803F120023F2A4E
:10C6E00000F2B28003F108020F2A1ED89A1C032A16
:10C6F00002D9002908BF0121A26802F120053F2DBF
:10C700002FD802F108050F2D11D900F03F0040F09D
:10C710008000F9F7D3F92079F9F7D0F9207ABDE84C
:10C720007040F9F7CBB90221D6E70221E4E7951C66
:10C73000032D00D911B1012940F0888000F00F00CD
:10C7400040F04000F9F7BAF9A068636800F00F0004
:10C7500040EA0310C0B2BDE87040F9F7AFB96368B2
:10C76000A26802F18001FF2944D902F50041B1F528
:10C77000803F64D302F50002B2F1807F34BF02250E
:10C78000032503F18002FF2A4FEA85050DD903F541
:10C790000042B2F5803F54D303F50003B3F1807F2C
:10C7A0002CBF45F0030545F0020500F18003FF2B87
:10C7B0004FEA850506D900F50043B3F5803F34D232
:10C7C00045F0010565F03F00C0B2F9F777F904F1D3
:10C7D0000C0605F00303022B20781DD0032B11D08B
:10C7E000012B09D0F9F76AF90434B4424FEAA505E0
:10C7F000EFD170BD0025C4E7F9F760F96078F9F76B
:10C800005DF9F1E7F9F75AF96078F9F757F9A07887
:10C81000F9F754F9E078E5E7F9F750F96078F9F7B6
:10C820004DF9A078F9F74AF9DEE700F50000B0F11C
:10C83000807F34BF45F0020545F00305C2E70125BE
:10C840009FE745F00105B0E7A2688AE702293FF4B7
:10C850005CAF01019B0003F00C0301F030010B43BE
:10C8600002F0030243EA0200BDE87040F9F726B97E
:10C87000F0B5C41784EA40047F2C83B046D9434DF9
:10C88000434E95F8C436434F08E0306803681B6890
:10C89000984795F8C436E4097F2C3AD964F07F01B3
:10C8A000022BC9B2F1D1DFF8F0E0DEF8000040F26F
:10C8B000FF1C90F91A308DF806105A1C16D04268E9
:10C8C000C2F30802624502EB43230FD0D9554368F7
:10C8D000E40901337F2C436064F07F012BD990F988
:10C8E0001A30C9B25A1C8DF80610E8D1037E13F035
:10C8F000060F02D090F82830ABB1E4097F2C64F029
:10C900007F0118D9C9B2DEF80000D2E71F4B93F8B7
:10C91000C436022BE1B235D01D4B186803681B6882
:10C92000984703B0F0BD01220DF106010EF0B0FEF4
:10C9300095F8C436AFE7E1B2DEF800008DF80710D5
:10C9400090F91A20531C0FD0436840F2FF14C3F330
:10C950000803A34208D003EB42230E4A99544368CC
:10C960000133436003B0F0BD037E13F0060FD8D04F
:10C9700090F82830002BD4D101220DF107010EF0E0
:10C9800087FECEE7DFF810E0D6E700BF7445002051
:10C990002C870020904F002014870020F0B57F28BE
:10C9A00083B0044646D9434D434E95F8C436434FB1
:10C9B00008E0306803681B68984795F8C436E409B6
:10C9C0007F2C3AD964F07F01022BC9B2F1D1DFF894
:10C9D000F0E0DEF8000040F2FF1C90F91A308DF80C
:10C9E00006105A1C16D04268C2F30802624502EBD8
:10C9F00043230FD0D9554368E40901337F2C4360AA
:10CA000064F07F012BD990F91A30C9B25A1C8DF805
:10CA10000610E8D1037E13F0060F02D090F82830FC
:10CA2000ABB1E4097F2C64F07F0118D9C9B2DEF8FC
:10CA30000000D2E71F4B93F8C436022BE1B235D089
:10CA40001D4B186803681B68984703B0F0BD0122AE
:10CA50000DF106010EF01CFE95F8C436AFE7E1B209
:10CA6000DEF800008DF8071090F91A20531C0FD043
:10CA7000436840F2FF14C3F30803A34208D003EB5A
:10CA800042230E4A995443680133436003B0F0BD1A
:10CA9000037E13F0060FD8D090F82830002BD4D1A5
:10CAA00001220DF107010EF0F3FDCEE7DFF810E0F3
:10CAB000D6E700BF744500202C870020904F00204F
:10CAC000148700200FB42DE9F04FDFF8F49299F8A5
:10CAD000C4368BB0022B149C00F00981B44B18684B
:10CAE000036848211B68984799F8C436022B00F068
:10CAF0005781AF4B1868036820211B68984715AF12
:10CB00000025DFF8C0A20497A84607AE631C059372
:10CB1000217849B3252948D1A31CCDF81880059365
:10CB20006078302863D04FF0000BA0F13003DBB207
:10CB3000092B57D96C282DD0642800F0C2803AD830
:10CB4000252831D079D9582800F0A680632830D123
:10CB500039780020F8F774FF059C631C0593217851
:10CB6000043701350029D5D199F8C436022B6AD093
:10CB70008F4B186803680A211B6898478D4AD2F8C2
:10CB8000943003355D1BC2F894500BB0BDE8F04FF4
:10CB900004B07047059B5C1C05941A78642A00F069
:10CBA000F0802AD8252A6DD1252100200135F8F7FB
:10CBB00047FF059CAAE7732833D05CD9752869D153
:10CBC0003C1D3868334600220A21274621F004F92B
:10CBD000069A00965B465146002021F081F9059C9B
:10CBE000054493E706AA05A911F026F9A2E7E31C7C
:10CBF0000593A0784FF0010B97E7732A11D040F20C
:10CC0000CB80752A54D0782A80D1A2F15802B2FA8A
:10CC100082F23868520933461021043721F0DCF8DB
:10CC2000D6E73B6800930023069A1846514621F048
:10CC300057F904370544059C68E70028B9D199F8ED
:10CC4000C436022B94D15C4B0A2218688DF81C2044
:10CC500090F91A104B1C3BD0436840F2FF14C3F309
:10CC60000803A34234D003EB412354495A54436888
:10CC70000133436082E76E289BD1059C3B680437F3
:10CC80001D6043E740F28480582ABED0632A3FF4F7
:10CC90005FAF3BE778288CD1A0F15802B2FA82F25C
:10CCA000386852093346102121F096F804378FE78F
:10CCB0003C1D3868334600220A21274621F08CF8B3
:10CCC00086E73B1D386831461F4621F057F87FE75D
:10CCD000037E13F0060F3FF451AF90F82830002B7D
:10CCE0007FF44CAF012207A90EF0D2FC46E7324B8D
:10CCF000186890F91A10436848224E1CC3F30803C1
:10CD00008DF80E2040F2FF151DD0AB421BD003EB77
:10CD100041232A495A54436890F91A100133436059
:10CD2000C3F3080320224D1C8DF80F2019D040F2C8
:10CD3000FF15AB4215D003EB412320495A544368F9
:10CD400001334360DBE6027E12F0060FEAD090F872
:10CD50002820002AE6D101220DF10E010EF098FCE8
:10CD6000C2E6037E13F0060F3FF4C9AE90F82830F8
:10CD7000002B7FF4C4AE01220DF10F010EF088FCF0
:10CD8000BDE63B1D386831461F4620F0F7FF1FE720
:10CD9000002A3FF4E9AEB9E66E2A3FF46FAFB5E67C
:10CDA000054B1868426890F91A10C2F30803B9E7F6
:10CDB0002C8700208425002014870020904F00201D
:10CDC00074450020415A00080FB42DE9F04389B0A2
:10CDD00010AE002556F8043BDFF8888102962F46F6
:10CDE00005AC5A1C0392197839B3252935D19A1C00
:10CDF000049703925878302852D04FF00009A0F1E0
:10CE00003003DBB2092B46D96C281CD0642800F013
:10CE1000948028D825281FD067D9582877D0632830
:10CE20001FD131780020F8F70BFE039B5A1C0392A8
:10CE30001978043601350029D7D1284609B0BDE854
:10CE4000F04304B07047039A531C03931278642A8A
:10CE50007AD02BD8252A52D1252100200135F8F788
:10CE6000EFFD039BBDE7732833D041D975284CD122
:10CE700006F1040E3068234600220A21764620F08F
:10CE8000ABFF4B46049A00944146002021F028F85D
:10CE9000039B0544A5E704AA03A910F0CDFFB3E75F
:10CEA000DA1C039298784FF00109A8E7732A10D092
:10CEB00055D9752A37D0782A93D1A2F15802B2FAFF
:10CEC00082F23068520923461021043620F084FF94
:10CED000D7E73368009300231846049A414620F0B0
:10CEE000FFFF04360544039B7BE70028A5D0B8E785
:10CEF0006E28B6D1039B32680436156071E72AD9D3
:10CF0000582ADAD0632A8CD06BE77828A9D1A0F10F
:10CF10005802B2FA82F2306852092346102120F0FA
:10CF20005BFF0436ADE706F1040E306823460022AD
:10CF30000A21764620F050FFA3E7331D30682146D2
:10CF40001E4620F01BFF9CE7331D306821461E461D
:10CF500020F014FF95E7002A3FF46FAF41E76E2AF7
:10CF6000C9D03EE7415A00082DE9F04F0C68DFF8C0
:10CF700014C3C04F2588C04E85B00CFB02F2BC42E2
:10CF8000B6FBF2F603F1FF3C06F1FF36BDF838E0E0
:10CF9000B6B2AAB21FFA8CFC5ED0B84DAC425BD0E0
:10CFA000B4F1804F58D0A5F59835AC4254D005F572
:10CFB0008065AC4250D0B24DAC4253D005F580658F
:10CFC000AC424FD022F4407205F58C3592B2AC429F
:10CFD0002280C4F82CC026850ED0A84A94420BD0DB
:10CFE00002F54062944207D002F58062944203D079
:10CFF00002F58062944201D10022228601256561FA
:10D00000CE79497916F0040731D016F0020F4FF0AF
:10D0100040054FF000060CBF4FF00809B146B0467E
:10D020000296B246B446324601964FF480670395A5
:10D030004FF0040B0C2900F2E280DFE811F0AF00A2
:10D04000E000E000E0008A00E000E000E0006300B3
:10D05000E000E000E0002A00894D22F07002AC42BE
:10D0600092B2ABD12280C4F82CC02685C6E70195C8
:10D070004FF4806506F002020397BB46B9464FF4B1
:10D0800080464FF4805802954FF0100A4FF4807C90
:10D09000D0E7256ADFF8DCC125F480552562256AD2
:10D0A0006768D4F81C9025F4005545EA08086445E3
:10D0B00029F4E64548EA023245F4C04500F0F08024
:10D0C0000CF5006C644500F0EB806760E561C4F826
:10D0D00040E02262E26942F40062E261626C42F482
:10D0E000004262642288254692B242F0010225F88D
:10D0F000342B00226E184381446006606A5005B0EC
:10D10000BDE8F08F256A5B4E25F480752562D4F862
:10D1100020B06568D4F81CA02BF4007B4BEA0C0C03
:10D120002AF0730AB4424CEA02224AF0600A00F084
:10D13000AB8006F50066B44200F0A6806560C4F8D6
:10D140001CA0C4F83CE02262E26942F00802E261FD
:10D15000C4E7256A474F25F010052562D4F820C0A2
:10D160006668A5692CF0200C25F080754CEA0A0A47
:10D1700025F4E645BC424AEA021245F4C0456AD0AD
:10D1800007F50067BC4266D06660A561C4F838E068
:10D190002262A26942F40062A2619FE7266ADFF878
:10D1A000D480019D26F001062662D4F820A067688D
:10D1B000A66926F480362A432AF0020A26F073066E
:10D1C000444542EA0A0246F0600639D02B4DAC4293
:10D1D00036D005F54065AC4232D005F58065AC42ED
:10D1E0002ED005F58065AC422AD06760A661C4F8F0
:10D1F00034E02262A26942F00802A2616EE70C29C3
:10D200003FF66CAF01A252F821F000BFF5D1000843
:10D21000DDD00008DDD00008DDD0000893D1000883
:10D22000DDD00008DDD00008DDD0000849D10008BD
:10D23000DDD00008DDD00008DDD00008D5D0000822
:10D2400022F00C0242EA090227F4407742EA0B027C
:10D2500047EA0C07C9E722F08002039F42EA09125D
:10D2600022F040023A43029F26F4406637433E468E
:10D270008AE700BF002C014000A24A0400340140AC
:10D280000010004040420F0022F4006242EA0922EE
:10D2900022F4806225F440553A4348EA05054DE7FB
:10D2A00027F48047374310E7036803F138422DE93C
:10D2B000F04F920A584DAA5C02F01F055209012452
:10D2C000022A04FA05F400F08C80032A00F08E8014
:10D2D000012A3CD001F003077A1E012AC1F3810C18
:10D2E000C1F300188088C1F3411135D9C60700F198
:10D2F0009780850700F1A380440700F1B180020701
:10D3000000F1BF80C60600F1CD80850600F1DB800C
:10D31000440600F1E980020600F1F780C60500F13D
:10D320000581850500F11381440500F12181020585
:10D3300000F12F81C60400F13D81850400F14B818D
:10D34000440400F15981020455D4BDE8F08F334AFA
:10D3500055692C435461BDE7002422464FF0010E6D
:10D360004FF0030904E00132102A04F10204ECD06A
:10D370000EFA02F636EA0005F5D1D3F808A009FA4C
:10D3800004F5ED430AEA050AC3F808A0D3F808B08B
:10D390000CFA04FA4AEA0B0AC3F808A0B3F804A08E
:10D3A0001FFA8AFA2AEA06069E80B3F804A008FA51
:10D3B00002F646EA0A06B6B29E801E682E401E603D
:10D3C000D3F800A007FA04F646EA0A061E60D3F86E
:10D3D0000CA001FA04F605EA0A0A46EA0A05DD602D
:10D3E000C1E70E4A95692C43946173E70B4AD569EE
:10D3F0002C43D4616EE71A6822F040421A601A6822
:10D4000042EA87771F60DA6822F0404242EA81717F
:10D41000D960BDE8F08F00BF4C6A030800100240DD
:10D420001A6822F003021A601A683A431A60DA682E
:10D4300022F003020A438507DA607FF55DAF1A68C0
:10D4400022F00C021A601A6842EA87021A60DA684F
:10D4500022F00C0242EA81024407DA607FF54FAF06
:10D460001A6822F030021A601A6842EA07121A603B
:10D47000DA6822F0300242EA0112DA6002077FF530
:10D4800041AF1A6822F0C0021A601A6842EA871295
:10D490001A60DA6822F0C00242EA8112C606DA6037
:10D4A0007FF533AF1A6822F440721A601A6842EAB4
:10D4B00007221A60DA6822F4407242EA01228506E5
:10D4C000DA607FF525AF1A6822F440621A601A68A4
:10D4D00042EA87221A60DA6822F4406242EA812234
:10D4E0004406DA607FF517AF1A6822F440521A60DA
:10D4F0001A6842EA07321A60DA6822F4405242EAB5
:10D500000132DA6002067FF509AF1A6822F4404260
:10D510001A601A6842EA87321A60DA6822F44042D6
:10D5200042EA8132C605DA607FF5FBAE1A6822F462
:10D5300040321A601A6842EA07421A60DA6822F436
:10D54000403242EA01428505DA607FF5EDAE1A68A5
:10D5500022F440221A601A6842EA87421A60DA68A6
:10D5600022F4402242EA81424405DA607FF5DFAED0
:10D570001A6822F440121A601A6842EA07521A60C6
:10D58000DA6822F4401242EA0152DA6002057FF5BD
:10D59000D1AE1A6822F440021A601A6842EA875231
:10D5A0001A60DA6822F4400242EA8152C604DA6064
:10D5B0007FF5C3AE1A6822F040721A601A6842EA18
:10D5C00007621A60DA6822F0407242EA016285045A
:10D5D000DA607FF5B5AE1A6822F040621A601A6808
:10D5E00042EA87621A60DA6822F0406242EA8162A7
:10D5F0004404DA607FF5A7AE1A6822F040521A6040
:10D600001A6842EA07721A60DA6822F0405242EA67
:10D610000172DA6097E600BF10B50409013C052CE1
:10D6200017DC0D4B33F8142000F00F0042FA00F322
:10D6300013F001030DD0012303FA00F0013810406C
:10D6400022F0D0FF054A064B125D104403EBC000E8
:10D6500010BD002010BD00BFC06F0308B86F0308E5
:10D66000147600202DE9F04F4A484B4B4B4C4FF0BD
:10D6700090414FF0010A4FF002094FF004084FF0BB
:10D68000080C4FF0100E20274026802530F8022B82
:10D6900012F0010F03D01960A3F804A0083312F0B0
:10D6A000020F03D01960A3F80490083312F0040F9E
:10D6B00003D01960A3F80480083312F0080F03D0D8
:10D6C0001960A3F804C0083312F0100F03D01960DA
:10D6D000A3F804E0083312F0200F02D019609F80F5
:10D6E000083312F0400F02D019609E80083312F008
:10D6F000800F02D019609D80083312F4807F05D01E
:10D700004FF4807B1960A3F804B0083312F4007F53
:10D7100005D04FF4007B1960A3F804B0083312F46D
:10D72000806F05D04FF4806B1960A3F804B0083304
:10D7300012F4006F05D04FF4006B1960A3F804B029
:10D74000083312F4805F05D04FF4805B1960A3F8B2
:10D7500004B0083312F4005F05D04FF4005B196089
:10D76000A3F804B0083312F4804F05D04FF4804B77
:10D770001960A3F804B00833D20B04D04FF4004270
:10D7800019609A80083301F58061A1427FF47EAF71
:10D79000BDE8F08FC06F0308147600200018004821
:10D7A000002867D003682DE9F04F03F138445C4E40
:10D7B000A40A0125345D04F01F066409022C05FA51
:10D7C00006F558D0032C00F0A580012C58D0808895
:10D7D000B0FA80F4C4F11F04A4B2E50803EB850598
:10D7E00004F007042E6AA4000F27A74026EA0706C4
:10D7F0002E622E6A01F00307A2407C1E3243012CE8
:10D80000C1F3810CC1F300182A62C1F341113CD964
:10D81000C60700F18980850700F19580440700F173
:10D82000A380020700F1B180C60600F1BF80850623
:10D8300000F1CD80440600F1DB80020600F1E980B2
:10D84000C60500F1F780850500F10581440500F16A
:10D850001381020500F12181C60400F12F818504A6
:10D8600000F13D81440400F14B81020400F1598133
:10D87000BDE8F08F70472B4CA6693543A561A6E73C
:10D88000284C666935436561A1E7002422464FF0C4
:10D89000010E4FF0030904E00132102A04F10204E2
:10D8A000E6D00EFA02F636EA0005F5D1D3F808A064
:10D8B00009FA04F5ED430AEA050AC3F808A0D3F80B
:10D8C00008B00CFA04FA4AEA0B0AC3F808A0B3F845
:10D8D00004A01FFA8AFA2AEA06069E80B3F804A07A
:10D8E00008FA02F646EA0A06B6B29E801E682E4084
:10D8F0001E60D3F800A007FA04F646EA0A061E6086
:10D90000D3F80CA001FA04F605EA0A0A46EA0A0569
:10D91000DD60C1E7034CE6693543E56157E700BFC9
:10D920004C6A0308001002401A6822F003021A60D1
:10D930001A683A431A60DA6822F003020A4385073C
:10D94000DA607FF56BAF1A6822F00C021A601A6871
:10D9500042EA87021A60DA6822F00C0242EA810287
:10D960004407DA607FF55DAF1A6822F030021A6072
:10D970001A6842EA07121A60DA6822F0300242EAB4
:10D980000112DA6002077FF54FAF1A6822F0C00279
:10D990001A601A6842EA87121A60DA6822F0C00236
:10D9A00042EA8112C606DA607FF541AF1A6822F4B6
:10D9B00040721A601A6842EA07221A60DA6822F492
:10D9C000407242EA01228506DA607FF533AF1A68B9
:10D9D00022F440621A601A6842EA87221A60DA6802
:10D9E00022F4406242EA81224406DA607FF525AFE4
:10D9F0001A6822F440521A601A6842EA07321A6022
:10DA0000DA6822F4405242EA0132DA6002067FF517
:10DA100017AF1A6822F440421A601A6842EA873245
:10DA20001A60DA6822F4404242EA8132C605DA60BE
:10DA30007FF509AF1A6822F440321A601A6842EA88
:10DA400007421A60DA6822F4403242EA0142850550
:10DA5000DA607FF5FBAE1A6822F440221A601A6879
:10DA600042EA87421A60DA6822F4402242EA81429E
:10DA70004405DA607FF5EDAE1A6822F440121A60B0
:10DA80001A6842EA07521A60DA6822F4401242EA3F
:10DA90000152DA6002057FF5DFAE1A6822F4400217
:10DAA0001A601A6842EA87521A60DA6822F4400261
:10DAB00042EA8152C604DA607FF5D1AE1A6822F0DC
:10DAC00040721A601A6842EA07621A60DA6822F045
:10DAD000407242EA01628504DA607FF5C3AE1A68DB
:10DAE00022F040621A601A6842EA87621A60DA68B5
:10DAF00022F0406242EA81624404DA607FF5B5AE0A
:10DB00001A6822F040521A601A6842EA07721A60D4
:10DB1000DA6822F0405242EA0172DA6002047FF5CC
:10DB2000A7AE1A6822F040421A601A6842EA877764
:10DB30001F60DA6822F0404242EA8171D960BDE894
:10DB4000F08F00BF002852D0036803F138422DE95E
:10DB5000F04F920A504DAA5C02F01F0552090124B1
:10DB6000022A04FA05F443D0032A00F09080012A27
:10DB700043D001F003077A1E012AC1F3810CC1F3DF
:10DB800000188088C1F341113CD9C60700F1888094
:10DB9000850700F19480440700F1A280020700F19C
:10DBA000B080C60600F1BE80850600F1CC80440638
:10DBB00000F1DA80020600F1E880C60500F1F68087
:10DBC000850500F10481440500F11281020500F190
:10DBD0002081C60400F12E81850400F13C814404BB
:10DBE00000F14A81020400F15881BDE8F08F7047CE
:10DBF0002A4A95692C439461BBE7284A55692C430E
:10DC00005461B6E7002422464FF0010E4FF003099D
:10DC100004E00132102A04F10204E6D00EFA02F602
:10DC200036EA0005F5D1D3F808A009FA04F5ED436A
:10DC30000AEA050AC3F808A0D3F808B00CFA04FAF7
:10DC40004AEA0B0AC3F808A0B3F804A01FFA8AFA3C
:10DC50002AEA06069E80B3F804A008FA02F646EA0D
:10DC60000A06B6B29E801E682E401E60D3F800A041
:10DC700007FA04F646EA0A061E60D3F80CA001FA79
:10DC800004F605EA0A0A46EA0A05DD60C1E7034A26
:10DC9000D5692C43D4616CE74C6A0308001002403C
:10DCA0001A6822F003021A601A683A431A60DA68A6
:10DCB00022F003020A438507DA607FF56CAF1A6829
:10DCC00022F00C021A601A6842EA87021A60DA68C7
:10DCD00022F00C0242EA81024407DA607FF55EAF6F
:10DCE0001A6822F030021A601A6842EA07121A60B3
:10DCF000DA6822F0300242EA0112DA6002077FF5A8
:10DD000050AF1A6822F0C0021A601A6842EA8712FD
:10DD10001A60DA6822F0C00242EA8112C606DA60AE
:10DD20007FF542AF1A6822F440721A601A6842EA1C
:10DD300007221A60DA6822F4407242EA012285065C
:10DD4000DA607FF534AF1A6822F440621A601A680C
:10DD500042EA87221A60DA6822F4406242EA8122AB
:10DD60004406DA607FF526AF1A6822F440521A6042
:10DD70001A6842EA07321A60DA6822F4405242EA2C
:10DD80000132DA6002067FF518AF1A6822F44042C9
:10DD90001A601A6842EA87321A60DA6822F440424E
:10DDA00042EA8132C605DA607FF50AAF1A6822F4CA
:10DDB00040321A601A6842EA07421A60DA6822F4AE
:10DDC000403242EA01428505DA607FF5FCAE1A680E
:10DDD00022F440221A601A6842EA87421A60DA681E
:10DDE00022F4402242EA81424405DA607FF5EEAE39
:10DDF0001A6822F440121A601A6842EA07521A603E
:10DE0000DA6822F4401242EA0152DA6002057FF534
:10DE1000E0AE1A6822F440021A601A6842EA875299
:10DE20001A60DA6822F4400242EA8152C604DA60DB
:10DE30007FF5D2AE1A6822F040721A601A6842EA80
:10DE400007621A60DA6822F0407242EA01628504D1
:10DE5000DA607FF5C4AE1A6822F040621A601A6870
:10DE600042EA87621A60DA6822F0406242EA81621E
:10DE70004404DA607FF5B6AE1A6822F040521A60A8
:10DE80001A6842EA07721A60DA6822F0405242EADF
:10DE90000172DA6002047FF5A8AE1A6822F04042EF
:10DEA0001A601A6842EA87771F60DA6822F04042F7
:10DEB00042EA8171D960BDE8F08F00BF10B10368FC
:10DEC00082881A85704700BF10B1036882889A6102
:10DED000704700BF38B100298388026814BF002151
:10DEE00010218B409361704730B1036882881B8A90
:10DEF0001A4214BF01200020704700BF2DE9F041F5
:10DF00000B4E346873691C400FD0DFF8288001275E
:10DF1000B4FA84F3C3F11F0307FA03F558F823009A
:10DF200003689847AC437561F2D1BDE8F08100BF4A
:10DF3000000401402C4500202DE9F0410B4E3468CF
:10DF400073691C400FD0DFF828800127B4FA84F3EE
:10DF5000C3F11F0307FA03F558F823000368984735
:10DF6000AC437561F2D1BDE8F08100BF000401400F
:10DF70002C4500202DE9F0410B4E346873691C409C
:10DF80000FD0DFF828800127B4FA84F3C3F11F0310
:10DF900007FA03F558F8230003689847AC43756106
:10DFA000F2D1BDE8F08100BF000401402C45002003
:10DFB0002DE9F0410B4E346873691C400FD0DFF837
:10DFC00028800127B4FA84F3C3F11F0307FA03F58D
:10DFD00058F8230003689847AC437561F2D1BDE857
:10DFE000F08100BF000401402C4500202DE9F041E4
:10DFF0000B4E346873691C400FD0DFF8288001276E
:10E00000B4FA84F3C3F11F0307FA03F558F82300A9
:10E0100003689847AC437561F2D1BDE8F08100BF59
:10E02000000401402C4500202DE9F0410B4E3468DE
:10E0300073691C400FD0DFF828800127B4FA84F3FD
:10E04000C3F11F0307FA03F558F823000368984744
:10E05000AC437561F2D1BDE8F08100BF000401401E
:10E060002C4500202DE9F0410B4E346873691C40AB
:10E070000FD0DFF828800127B4FA84F3C3F11F031F
:10E0800007FA03F558F8230003689847AC43756115
:10E09000F2D1BDE8F08100BF000401402C45002012
:10E0A000084A094808B5936943F0010393610021C8
:10E0B000402226F002FB054B4FF0FF321A60C3F8F6
:10E0C000032008BD001002402C4500206C450020B4
:10E0D00010B404686469A4465DF8044B604700BF4F
:10E0E000036810B504461B689847236820469B6860
:10E0F0009847237A0133237210BD00BF10B503681F
:10E1000004469B689847FF230122E371A27110BD6A
:10E11000F0B484894FF6FF764FF47A745BB3002A2B
:10E120003BD01778013201E0B44219D00589013C97
:10E1300015F00205A4B2F7D007734FF47A7402E029
:10E14000BCB2B4420CD0058915F0010504F1FF37CB
:10E15000F6D0057BEDB209B10D700131013BDDE771
:10E16000104B98420BD0A3F57843984217D003F593
:10E170008063984202D00120F0BC704702250A4B10
:10E1800003EB05156B8901339BB26B81688980B203
:10E19000003018BF0120F0BC7047FF27C6E70125FB
:10E1A000EDE700BF003001401C16002040F2E933CB
:10E1B00000E09BB10289013B12F0020F9BB2F8D044
:10E1C000017340F2E93300E043B10289013B12F0F0
:10E1D000010F9BB2F8D0007BC0B270470C4A90424E
:10E1E00009D00C4B984210D003F58063984201D0BF
:10E1F000FF2070470223084A02EB03135A890132B9
:10E2000092B25A815889C0B270470123F3E700BF28
:10E2100000300140003800401C1600202DE9F0417C
:10E220000701624E624BF259F1199A4206EB07045C
:10E2300004BF01230B730546207A0FF0A3F9237A5C
:10E2400003F01F015B090122022B02FA01F200F028
:10E250008780032B7FD0012B68D0F41901356079BA
:10E26000FFF7DAF9EDB212238371C5718046E079C8
:10E27000FFF7D2F913238371C571A079FFF7CCF9A9
:10E2800014238371C571627A0E214046FFF788FA24
:10E29000E079FFF7C1F9627A0E21FFF781FAA079E0
:10E2A000FFF7BAF9627A0E21FFF77AFA207900288F
:10E2B00046D1F3593F4A934262D03D4A93426AD0D5
:10E2C0003D4A934251D03E44327B62B300242546FE
:10E2D0009A8822F480521204120C9A80998889B28A
:10E2E00041F4805199801A8802F4415242F44572F7
:10E2F00022432A431A809A8822F470621204120C74
:10E3000042F4E0629A809A8B22F400621204120CAA
:10E3100007219A8319821A8892B242F040021A8029
:10E3200048B9BDE8F08101240225D1E7234B996A61
:10E330000A439A6291E7FFF76FF9BDE8F041C3E540
:10E34000FFF76AF91F22C5718271627A0D21FFF70A
:10E3500027FA2079ADE7194B19690A431A617CE75E
:10E36000164BD9680A43DA6077E702F5EA32116999
:10E3700041F400411161116921F400411161A2E7EA
:10E3800002F56042D16841F48051D160D16821F436
:10E390008051D16097E702F5EC32116941F4804178
:10E3A0001161116921F4804111618CE71C16002074
:10E3B0000038004000300140003C004000100240A6
:10E3C000427A02B9704710B504460368406804F108
:10E3D0000A0198470023637210BD00BF437A5A1C9C
:10E3E0000344D2B242729972037A934200D802B9BE
:10E3F000704710B504460368406804F10A01984765
:10E400000023637210BD00BF10B40B49002301E06C
:10E41000272B0CD011F8132082424FEA430403F15A
:10E420000103F5D121445DF8044B48787047002082
:10E430005DF8044B704700BF1C540308024A936800
:10E4400023EA00009060704774450020024A9368F8
:10E4500018439060704700BF7445002038B5134DD5
:10E460002C789C2C01D0002038BD6B88B3F5DD6F73
:10E47000F9D12B79BE2BF6D195F8E636EF2BF2D1F8
:10E4800005220B490B4826F098F90028EBD10A49E0
:10E490002B4602E013F8014F10468B4284EA00023B
:10E4A000F8D1201AB0FA80F0400938BD00F0030816
:10E4B0003C7B0308E1F60308E7F60308F8B5FFF72D
:10E4C000CDFF002800F0F2808F4C13F0D7F92046E2
:10E4D0004FF4DD628D4923F0B7FD94F8E035022B4F
:10E4E00040F2D58000231A4684F8E03540F284419A
:10E4F000742000FB034302F2D24293F8D004844B11
:10E50000844D18700C2313FB002294F8D400824E23
:10E510002144224404282A60316000F0E08040B9A0
:10E52000B4F8D230B3F5F07F84BF4FF4F073A4F8A1
:10E53000D230A368794A1A40002A00F0E080DD0753
:10E5400000F1C880580400F1C080190700F1B880BC
:10E550009A0100F1AF809B0400F1A180704B714FD4
:10E560001F600FF00FFE18B907F1840000F04EFC99
:10E5700000F0AAFB03F0C8FC302200216A486B4D72
:10E5800026F09BF830680FF0C7FD6949694A0D60B5
:10E59000694B94F8B602A5F166011160A5F5817288
:10E5A0001A606421654BC82211FB00210022B4F8D7
:10E5B000160259609A60DA601A615A619A61DA61EA
:10E5C00083F8202083F821200CF09CFAB4F8343230
:10E5D0009FED5B5A3268DFF8B8C194F8F511DFF8A7
:10E5E000B4E19FED586A584E584806EE903AF8EE5E
:10E5F000E66AB4F8F031C5EE265A07EE103A544BED
:10E600001A60B4F8F231534A07EE903A524BC2ED19
:10E61000005A94F8F4211972A5F50D744F49CCF8FD
:10E620000040A5F5087C5A72B8EEC77A4C4ACEF87D
:10E6300000C0F8EEE77AA5F5D57EC1F800E0A5F5B3
:10E640009D71116027EE067A464983ED017A67EEE7
:10E65000867AA5F514743460C3ED007AA5F16904D7
:10E66000414B0F606FF49C770460EF193F4E404CB4
:10E6700040481F60404A41491160A5F1F803D03D70
:10E68000336025600360BDE8F84013F0DFB8C3EBEA
:10E69000C30203EB8202920002F2844128E7384869
:10E6A000FFF7CCFE4020FFF7C9FE57E7042001F03A
:10E6B00037FB09E746F20900FFF7C0FEA3684AE707
:10E6C0003048FFF7BBFEA36842E72F48FFF7B6FECE
:10E6D000A3683AE72D48FFF7B1FEA36832E7B4F824
:10E6E000D030B3F57A7FBFF424AF4FF47A73A4F837
:10E6F000D0300A4AA3681A40002A7FF420AF0120D4
:10E70000FFF7A4FEA3681AE77445002000F0030891
:10E71000E17F0020E47F00204839002009600002EA
:10E7200078730020C8470020B07F00209048002068
:10E730001C2600205839002038910020081B00209A
:10E74000C0C9FB4817B7D138387200205C7200206E
:10E75000C82B0020647300200C39002034440020B2
:10E76000B06D0020006D0020B46D0020BC2B002097
:10E7700098260020AC2B0020303900203661023D65
:10E780000940000201600002092000020860000246
:10E79000407200202C4400202DE9F04F4A4C83B0F9
:10E7A00013F06CF84FF4DD65BE20EF239C210022AE
:10E7B000207184F8E6366580217084F8E726631CB2
:10E7C000601901E013F8011B984282EA0102F9D1B5
:10E7D0003E4B84F8E7261A69120603D53C493D4AA8
:10E7E00059605A60394FDFF8F080DFF8F0A0032459
:10E7F0004FF03409344EC7F80C90002535BB0FF0AC
:10E8000075FC042810D0631E13F0FF04F2D12F4AC8
:10E81000136943F080031361052001F081FA13F0BE
:10E8200015F803B0BDE8F08F3B6943F002033B618C
:10E83000C7F814803B6943F040033B610FF056FC7E
:10E840003B69042823F002033B61DCD100230193E0
:10E8500056F804BB0FF04AFC0428D4D1396905F1FD
:10E86000006303F57C3341F001011FFA8BF239613B
:10E870001A800FF03BFC042804D03B6923F001030D
:10E880003B61C0E705EB0A030193019B4FEA1B4B79
:10E89000A3F800B00FF02AFC3B69042823F0010321
:10E8A00005F104053B61AED1B5F5DD6FA6D13B693D
:10E8B00043F080033B61FFF7D1FD0028ACD012F09C
:10E8C000C5FF03B0BDE8F08F744500200020024072
:10E8D00023016745AB89EFCD00F0030802F0030880
:10E8E0000378202B024600F10100F9D0092BF7D064
:10E8F0002D2B2CD02B2B03BF5378B7EE000A0246EA
:10E90000B7EE000AA3F13001C8B209289FED467A9C
:10E9100010D8F2EE046A07EE901AF8EEE77A12F8D1
:10E92000013FE7EE267AA3F13001C8B20928B0EE24
:10E93000677AF0D92E2B4CD003F0DF03452B0BD098
:10E94000F7EE007A67EE276A20EE260A70475378C2
:10E95000BFEE000A0246D5E710B451782D2959D0F0
:10E960002B290ABF9178501C901C0024A1F1300380
:10E97000092B53D8002303EB830301EB430310F867
:10E98000011FA1F13002092AA3F13003F3D9B3F535
:10E990009A7F28BF4FF49A73072B42D9DFED236A81
:10E9A0001A46F7EE007A083A072A67EEA67AFAD8EE
:10E9B00003F007032BB1F2EE046A013B67EEA67A7F
:10E9C000FBD124B3C7EE276A5DF8044B20EE260A7C
:10E9D00070475378A3F13001C8B2092802F101024F
:10E9E000AAD8F2EE046AF0EE665A07EE901AF8EE34
:10E9F000E77A12F8013F87EEA66AA3F13001C8B2A8
:10EA0000092866EEA56A37EE067AEED994E767EE36
:10EA1000276AD9E7901C91780124A7E7F7EE007ADE
:10EA2000CFE7F7EE007AC5E70000000020BCBE4C3F
:10EA3000B5EEC00ADFED317AF1EE10FACCBF30EE60
:10EA4000270A30EE670ADFED2E7A20EE270A30B56E
:10EA5000FDEEC07A87B017EE904A054684EAE4706E
:10EA6000002303A9A0EBE4700193009302930FF03D
:10EA700007FA002CACBF20232D2303A88DF800300B
:10EA800021F04EF8012803A924D002282DD0032814
:10EA900005BF3023684668468DF8013025F068FED2
:10EAA000684621F03DF80338C4B22246694628463C
:10EAB00025F0BCFE00232B55284621F031F82E22EC
:10EAC000431C2A540DEB0401E81825F06EFE28467D
:10EAD00007B030BD302368468DF801308DF8023024
:10EAE0008DF8033025F044FEDAE7302368468DF8D0
:10EAF00001308DF8023025F03BFED1E76F12033A6A
:10EB000000007A4438B50B4C23688BB15A68821ADE
:10EB1000002A054604DA0CE05A68AA1A002A07DB24
:10EB20009A68226018461A6890472368002BF3D130
:10EB300038BD38BD2C3B00202DE9F0470569C3687E
:10EB40001D4028D00F4606464FF000484FF0000900
:10EB5000B5FA85F328FA03F2D2431B3B3261154024
:10EB6000042B16D8DFE803F03129211903007B6A52
:10EB7000002B32D003F1FF3A1FFA8AFAC7F824902B
:10EB80003C6A34B123682046514698476468002C9B
:10EB9000F8D1002DDCD1BDE8F0873868716B0368CF
:10EBA00089B29847002DD3D1F5E77868B16B036837
:10EBB00089B29847002DCBD1EDE7B868F16B0368B7
:10EBC00089B29847002DC3D1E5E7F868316C036836
:10EBD00089B29847002DBBD1DDE7F36A1FFA83FAAB
:10EBE000CEE700BF174C08B5237803F00502052ACD
:10EBF00024D003F00902092A06D000200EF0E8FE16
:10EC000000200EF0FFFEFEE76568A0682B68E16853
:10EC10004FF6FE7633402B60038823F001031B047C
:10EC20001B0C29260025038008468E71CD714E21CC
:10EC3000FEF7B6FDE068FFF741F9DEE716F0B4F83D
:10EC40002378D6E720260020F0B40D490D4F91F827
:10EC5000E0250D4E742540F2D243022815FB023404
:10EC600028BF022005FB02120C2313FB00430B44B8
:10EC700082F8D0043B603070F0BC03F045B900BFAF
:10EC800074450020E47F0020E17F002010B50228B9
:10EC900028BF0220064B044683F8E005FFF77CFD01
:10ECA000FFF70CFC601CC0B2BDE810400DF0C8BE00
:10ECB0007445002008B5FFF76FFDFFF7FFFBBDE8C7
:10ECC00008400FF0A5BA00BF10B54B4CB4F80432A1
:10ECD000B4F806229A4224BF0023A4F80432B4F800
:10ECE0000A22B4F808329A4224BF0023A4F808325A
:10ECF00094F8FF31A3B1072B12D094F8D42001234C
:10ED00000021062A84F8F83184F8FE3184F80312D1
:10ED100058D994F8D530DFED396A002B3FD110BDBA
:10ED200094F80332002B53D094F8FE3194F8F81184
:10ED3000DFED326A042B38BF042307EE903AB8EEB9
:10ED4000E77A07EE901A27EE267AF8EEE77A84F84B
:10ED5000FE3167EE877A94F8D420062A2FD8284B04
:10ED600003EB8203D3ED006AF4EEE76AF1EE10FAEA
:10ED700011DDC6EE877AFDEEE77A17EE903A102B9A
:10ED8000A8BF1023012BB8BF0123DBB28B4228BFE1
:10ED90000B4684F8F83194F8D530002BBFD0013AF7
:10EDA000032ABCD8B7EE000A80EE260A23F078FBCF
:10EDB000B4F8D230984238BFA4F8D20010BDDFEDCD
:10EDC0000F6AD1E7DFED0F7A1946B0EE677AC6E732
:10EDD00094F8FE3194F8F811DFED0B6A07EE103A63
:10EDE00007EE901AB8EEC77AF8EEE77A27EE267AA1
:10EDF00067EE877AAFE700BF744500206F120338D3
:10EE00006C5403086F12833A6F120339F8B5442229
:10EE10000746002125F051FC64225223A7F8402028
:10EE200087F842300A483B4607F140061421052284
:10EE30000425002401E010F9011B9970DA701D719E
:10EE40009C715A710833B342F5D101233B80F8BD60
:10EE50001D7603082DE9F0432C213A2216262D2495
:10EE60004FF00F0E22250E27352301704270192115
:10EE700021224675047353264FF4FA7480F804E097
:10EE80004FF07C5E4571C773282514274376817146
:10EE900032230274867600224B264485C0F82CE08B
:10EEA00037244FF0010E462185720572077587756C
:10EEB000C372C370C371437480F82830C676467736
:10EEC00044724FF000084FF4827C1D4681704FF071
:10EED0007E534273C275827302764284DFF88C904F
:10EEE000C47480F81EE080F832E080F833404FF0C0
:10EEF000A00E80F8344080F8407064244FF4AF775F
:10EF000080F83560A0F826E00787C36380F83120D9
:10EF100080F83620A0F824C0C0F84490C0F848809B
:10EF2000048480F84140034600F1240E0A2740F291
:10EF3000726683F84E4083F84F4083F8502083F880
:10EF4000515083F8522083F8567083F85720A3F865
:10EF5000586083F8531083F8541083F855100C331D
:10EF60007345E6D180F84C20BDE8F08300002041D5
:10EF70002DE9F04704464FF4DD620021162740F6E4
:10EF8000761525F09AFB40F60C0140F6961240F6F5
:10EF90006C10A4F84674A4F8505481276F254FF4E0
:10EFA000C673A4F84814A4F8522461214222A4F89C
:10EFB0005404A4F85874A1204FF4B177A4F85E5417
:10EFC0004FF4D175A4F85634A4F85C144FF4A1732F
:10EFD0002F21A4F86024A4F86404142240F69800B9
:10EFE000A4F86874A4F86E5440F6C8074FF4C175CD
:10EFF000A4F86634A4F86C140023C82184F87224A1
:10F00000A4F874040A226420A4F84C74A4F84E7482
:10F01000A4F86254A4F86A549C2740F6C415DFF89B
:10F0200074E3A4F85A14A4F87014A4F87624A4F88D
:10F03000780484F87F3484F8803484F8813484F848
:10F04000823484F87C3484F87D3484F87E34C4F8C7
:10F0500008E0A4F80812A4F80A0204215A20277034
:10F06000A4F8F0514FF496773025C74E84F8F81184
:10F0700084F801026E212B20A4F8067284F8FD5159
:10F080002127232584F8381284F83B0201214FF40C
:10F09000C87084F83C7284F83D523727132584F8F1
:10F0A0003922A4F8040284F8E035A4F8F23184F897
:10F0B000FF3184F8003284F8F931A4F81C32A4F846
:10F0C0001A32A4F81E3284F8FC3184F8183284F81D
:10F0D0000E3284F8193284F8FE1184F8FA1184F89B
:10F0E000501284F80F1284F8241284F83A1284F82B
:10F0F0003E12A4F8400284F84B2284F8487284F847
:10F100003F32A4F84232A4F8463284F8441284F81C
:10F11000491284F84A3284F8345306F1DC00374649
:10F12000324602E0072B0BDC9179890704D5E11800
:10F13000157981F835530133824202F11402F1D17D
:10F1400000210523C4F820134FF0310C3225C4F8F8
:10F15000241384F82C333021984640F2DC530022EB
:10F160004FF0010E84F83FC384F8435384F84113F1
:10F1700040F24C4C40F26C75A4F86A32DFF81892F9
:10F18000A4F86CC240F643034FF03F0A40F27531D9
:10F19000A4F86E5284F81DE384F81EE384F83EE37D
:10F1A00084F842E384F840E384F847E384F883E496
:10F1B00084F85DE284F866E284F81C2384F828234E
:10F1C00084F8292384F82A2384F82B2384F82D2318
:10F1D00084F8482384F85C2284F85E2284F85F2255
:10F1E00084F8652284F846A3C4F80890A4F878123D
:10F1F0002546A4F87A324FF01E0C234603E0013274
:10F2000002330EF1010E032ACCBF0121002183F845
:10F210007C1200F01482BEF1120F83F87DC2EED191
:10F2200000234FF0130E40F246524FF002080E2119
:10F2300084F868C284F8673284F8693284F87132DD
:10F2400084F8733284F872E2A4F8762284F870822B
:10F2500084F8741204F5297304F52D724FF47A7E44
:10F260004FF4FA6C23F804EC23F802CC04339342F5
:10F27000F8D10523A4F8D0E04FF0190E84F8B2328B
:10F2800084F8F4E1032340F22E4E0122002184F899
:10F29000B332A4F8CCE04FF4F073DFF800E1A4F847
:10F2A000D230A4F8CEC084F83D1384F8B01284F8AC
:10F2B000B12284F8B52284F8B42284F8D420324BE9
:10F2C000C4F8D8E002E00B290CDC9A79520705D586
:10F2D000621893F804E082F8DCE00131834203F124
:10F2E0001403F0D14FF4C87E40F2DC530121002218
:10F2F000A4F8FEE04FF0320EA4F8F03084F8FC10D1
:10F3000084F80021204BA4F8F2E002E0072A0CDC8C
:10F310009979090705D5A11893F804E081F8F4E07C
:10F320000132834203F11403F0D1322340F2EA5157
:10F3300040F2B45240F27E50A4F8EE30A4F8E80057
:10F34000A4F8EA10A4F8EC2004F5737004F55378DF
:10F35000FCF798FA80220021404625F0AEF92422DD
:10F360000A4904F20C4022F06FFE0B22084904F512
:10F37000866022F069FE0323002284F83C3484F87E
:10F380003B2401230DE000BF546A0308885403089E
:10F39000AC540308038D2C00038DAC00000090409A
:10F3A000B37913F0100306F1140640F040810132E6
:10F3B0000C2AF5D184F83D3404F2CB22104604F235
:10F3C000BF23002102F8011F03F8011F8342F9D176
:10F3D0009C4B0020D91D4FF02B094FF02A084FF00D
:10F3E000130C4FF0120E1A27192699424ED013F91A
:10F3F000012B1F2AF9D80FF2080A5AF822F000BF91
:10F400001BF6000811F6000807F60008FDF50008D5
:10F41000F3F50008EBF30008EBF30008EBF300084A
:10F42000EBF30008EBF30008EBF30008EBF3000844
:10F43000EBF30008EBF30008EBF30008EBF3000834
:10F44000EBF30008EBF30008EBF30008EBF3000824
:10F45000EBF30008EBF30008EBF30008EBF3000814
:10F46000EBF30008EBF30008EBF30008EBF3000804
:10F47000EBF30008EBF3000825F6000881F4000820
:10F48000994284F8D70284F8CB02B0D104F53670E3
:10F4900004F28446FFF7BAFC3046FFF7DBFC6A4B08
:10F4A0006A4A6B49C4F8283200274FF001084FF030
:10F4B0000A094FF0280A1523C4F82C12C4F8302288
:10F4C000A4F82072A4F82272A4F80C7284F8F581D2
:10F4D00084F8253204F515715E48A4F8169284F874
:10F4E000F6A184F8F7A111F07FFF4FF448734FF4B1
:10F4F0007A70642184F84C7284F84D7284F84F82DB
:10F5000084F8367284F8BA7284F8BE82A4F8343271
:10F5100084F84EA284F8B69284F8B792A4F8B802A0
:10F52000A4F8BC1204F1700823464FF4FA6C40F2C0
:10F53000DC5E5A22FF27A3F87201A3F874C1A3F876
:10F5400076E183F8781183F8792183F87A2183F8BA
:10F550007B710E339845EED10423002184F8E3310A
:10F56000002284F8E21104F1C003EA6010359D42E4
:10F57000FBD1394A3949107984F8E50603C9A368F3
:10F58000C4F840041068A4F84414012243F4002590
:10F5900041F26C6E0023C4F8E1064FF0040C022720
:10F5A0002920222184F88C2684F8C22684F8C326D8
:10F5B00084F8300384F83113A560314684F88BC693
:10F5C00084F88D3684F8C53684F8323384F83333C2
:10F5D000A4F88EE684F8C476742204F59F6022F0C5
:10F5E00033FD314604F26C507422BDE8F04722F03E
:10F5F0002BBD84F8D00284F8C402F6E684F8CF026A
:10F6000084F8C302F1E684F8CE9284F8C282ECE674
:10F6100084F8CDC284F8C1E2E7E684F8CC7284F8BD
:10F62000C062E2E684F8D60284F8CA02DDE602EBA4
:10F63000820207EB8202137984F83D34BCE683F83A
:10F640007D82DCE51D7603089A99193F3D0A773FD4
:10F65000F6287C3F9C8A03083C7B0308B8540308C7
:10F6600010B50B4C2046FFF783FC0A4894F8D034C1
:10F670000370094A09490C2000FB034304F2844447
:10F6800003F2D2431460BDE810400B600FF086BF58
:10F6900074450020E17F002048390020E47F0020ED
:10F6A0002DE9F84FF02200218E488F4CDFF8609250
:10F6B0008E4D8F4E8F4FDFF85C8224F0FEFF8E4818
:10F6C0008E49DFF854E2DFF854C200221359834216
:10F6D00000F0F880B3F1804F00F0F680AB4200F00C
:10F6E000F580B34200F0F480BB4200F0F380734534
:10F6F00000F0F280634500F0F180434500F0F080B7
:10F70000DFF81CA2534500F0A7800AF5806A534534
:10F7100008BF092300F0A1801432F02AD6D1DFF807
:10F72000C881774F774D08F1F0064FF0030A4FF08C
:10F73000020998F804301C09013C052C03F00F0362
:10F7400000F3838037F8140040FA03F2D2077CD527
:10F750004FF0010B0BFA03F3013B184020F042FF7E
:10F76000694B1B5D184415EBC0046ED055F8303062
:10F77000664898F8081003F13842920A825C02F059
:10F780001F005209022A0BFA00FB00F09480032AA2
:10F7900000F08A80012A05D1584A584852694BEA3C
:10F7A00002024261B4F804E0BEFA8EF2C2F11F0216
:10F7B00092B2D00803EB800002F00702046A9200C4
:10F7C0004FF00F0C0CFA02FC24EA0C040462046AE9
:10F7D00001FA02F22243002402624FF0010C224699
:10F7E00003E0102A04F102042FD00CFA02F030EAF0
:10F7F0000E0102F10102F4D1D3F808B00AFA04F1C3
:10F80000C9430BEA010BC3F808B0D3F808B0C3F83A
:10F8100008B0B3F804B01FFA8BFB2BEA0000988005
:10F82000988880B29880186808401860D3F800B0B3
:10F8300009FA04F040EA0B001860D868102A01EABF
:10F840000001D96004F10204CFD108F11408464543
:10F850007FF46FAFBDE8F88F082309EBC3034FF0C7
:10F86000010B93F804A00AF01F034FEA5A1ABAF1E9
:10F87000020F0BFA03F30BD0BAF1030F0ED0DA45E7
:10F880007FF44AAFD1F814A043EA0A034B6143E77F
:10F89000D1F818A043EA0A038B613DE7D1F81CA018
:10F8A00043EA0A03CB6137E7144A1448D2694BEAAA
:10F8B0000202C26176E7114A104892694BEA0202DD
:10F8C00082616FE70023C8E70123C6E70223C4E78C
:10F8D0000323C2E70423C0E70523BEE70623BCE7F2
:10F8E0000723BAE730870020546A03080004004069
:10F8F0000008004000100040002C014000100240B1
:10F90000C06F030814760020B86F03084C6A030820
:10F91000CC6F030800400140001400400034014057
:10F920000044014001490248FFF706B9D087002092
:10F930000040014001490248FFF7FEB8A8870020B7
:10F940000034014001490248FFF7F6B8A8870020BB
:10F950000034014001490248FFF7EEB880870020DB
:10F960000004004002494FF08040FFF7E5B800BFB7
:10F970005887002010B5064C06482146FFF7DCF8F2
:10F9800004F1C8010448BDE81040FFF7D5B800BF36
:10F9900030870020002C014000440140014902480A
:10F9A000FFF7CAB830870020002C01402DE9F04154
:10F9B00004684E4DA30AAB427AD00AD94C4DAB42F3
:10F9C0005FD00135AB4277D0043DAB425DD0BDE89E
:10F9D000F081B3F5801F67D04A3DAB4259D14FF05B
:10F9E000700E022647794FEA970C002968D0B000C4
:10F9F000634685190227D4F80C809F400CEB450321
:10FA0000BFB23C4D03F1040C47EA080745F8231048
:10FA100045F82C20E760EFF31281502282F3128820
:10FA2000821905EBC2021369002B34D01362043330
:10FA3000821905EBC202576917B11F60536904337D
:10FA4000821905EBC202976917B11F6093690433ED
:10FA5000821905EBC202D76917B11F60D36904335D
:10FA60000027CAB21F6082F31188304405EBC00042
:10FA7000036A9BB9E3684FF6FE721340E360BDE88A
:10FA8000F0814FF0C00E0426ACE74FF0980E03262D
:10FA9000A8E7BDE8F08105EB0E03C9E7E36843F092
:10FAA0000103E360BDE8F0814FF0480E012699E7BD
:10FAB0004FF0200E002695E74FF0E80E052691E75F
:10FAC000BF08022306FA03F0BB40DB43E768094D99
:10FAD0009BB23B4087190CEB470CE3600CF104032D
:10FAE00045F82C1045F8232095E700BF4B00100087
:10FAF000500010003087002070B503685E4D5F4EE7
:10FB000018885F4C05FB02F20139B4FBF2F4B342F2
:10FB100004F1FF3482B089B2A4B282B266D05948EF
:10FB2000834263D0B3F1804F60D0A0F59830834218
:10FB30005CD000F58060834258D0534883425BD04C
:10FB400000F5806083427CD022F4407200F58C3056
:10FB500092B283421A80D9621C850ED0494A9342E0
:10FB60000BD002F54062934207D002F580629342C7
:10FB700003D002F58062934201D100221A8601224D
:10FB80005A611A883D4992B242F001028B421A80B2
:10FB900061D0B3F1804F60D03C4A93425FD002F510
:10FBA000806293425DD002F5006293425BD002F521
:10FBB0008062934259D002F59032934257D002F5B9
:10FBC0004062934255D002F5806293421ED002F506
:10FBD0008062934208BF092219D002A84FF0012386
:10FBE00040F8043D0DF036FE02B070BD264822F00C
:10FBF0007002834292B2A3D101201A80D9621C857F
:10FC000058611A8892B202431A80C5E70822204B35
:10FC100003EBC20301A85C798DF8044001230022A4
:10FC20008DF805308DF807308DF806200DF012FEA6
:10FC30001B2CD9D1174B019301A80DF00BFE02B07C
:10FC400070BD01201A80D9621C8558611A8892B251
:10FC500002431A809DE70022D9E70122D7E702225A
:10FC6000D5E70322D3E70422D1E70522CFE7062216
:10FC7000CDE70722CBE700BF40420F00002C014038
:10FC800000A24A040034014000100040000400407B
:10FC9000CC6F0308190100011F4B98422CD0B0F122
:10FCA000804F2BD0A3F59433984229D003F580637D
:10FCB000984227D003F50063984225D003F580636E
:10FCC000984223D003F59033984221D003F5406346
:10FCD00098421FD003F58063984207D003F58063F4
:10FCE000984208BF092202D00020704708220B4B1F
:10FCF00003EBC203187970470022F8E70122F6E708
:10FD00000222F4E70322F2E70422F0E70522EEE7FD
:10FD10000622ECE70722EAE7002C0140CC6F03083B
:10FD20002DE9F04F89B0431C0793634D634EDFF814
:10FD3000A481634C0A2305934FF0100A614B197894
:10FD4000614B5B6801F002023BB1002A9A88186897
:10FD50000CBF10270027BA4082615B4A126801F08D
:10FD600001012AB197881068090107FA01F1816140
:10FD70000799029132210391DFF85CC105210491BA
:10FD800033B119689B88888A034218BF1B048B61B2
:10FD900032B1116893888A8A134218BF1B048B61A1
:10FDA0004A4B1A784A4B1B68002A40F0138223B151
:10FDB00019689B88102293408B61039B0693994698
:10FDC0004FF47A7019F1FF39C0F08880D8F8043008
:10FDD000C3F30803002B52D1EFF31283002B4ED153
:10FDE0002968A26800BF2B689942F9D1376800FBE7
:10FDF00007F39B1AB3FBF7F300FB0131D8F804308B
:10FE00000191C3F308030127E3B9EFF31283CBB9E0
:10FE10002B68A16800BF2A689342F9D1D6F800B0D8
:10FE200000FB0BF2521AB2FBFBF200FB0323019A18
:10FE30009B1AB3F57A7FC5D2D8F80430C3F3080310
:10FE4000002BE2D0EFF3128E8AF31288A1682368A8
:10FE5000DB0344BFCCF80070A1682B68DCF80020FD
:10FE60005FFA8EFE8EF31188D6F800E01A4400FB8C
:10FE70000EF35B1AB3FBFEF300FB0233D7E7EFF39D
:10FE800012828AF31288A7682368D90303D5012355
:10FE9000CCF80030A7682B68DCF80010D2B282F3EF
:10FEA00011883268194400FB02F3DB1BB3FBF2F349
:10FEB00000FB0131A2E700BFEC190020607E0020AA
:10FEC00010E000E01E450020204500205C4F00208F
:10FED000584F002000ED00E05C7E00208F4B5B68F7
:10FEE00033B11A689B88918A0B4218BF1B04936137
:10FEF0008A4B1B6833B11A689B88918A0B4218BFE2
:10FF00001B049361864B1A78864B1B68002A40F0CD
:10FF10005A8123B119689B8803FA02F28A61DDF8DD
:10FF200018E04FF47A701EF1FF3E74D3D8F8043015
:10FF3000C3F30803002B52D1EFF31283002B4ED1F1
:10FF40002968A26800BF2B689942F9D1376800FB85
:10FF500007F39B1AB3FBF7F300FB0131D8F8043029
:10FF60000191C3F308030127E3B9EFF31283CBB97F
:10FF70002B68A16800BF2A689342F9D1D6F800B077
:10FF800000FB0BF2521AB2FBFBF200FB0323019AB7
:10FF90009B1AB3F57A7FC6D2D8F80430C3F30803AE
:10FFA000002BE2D0EFF312898AF31288A16823684C
:10FFB000DB0344BFCCF80070A1682B68DCF800209C
:10FFC0005FFA89F989F31188D6F800901A4400FB8A
:10FFD00009F35B1AB3FBF9F300FB0233D7E7EFF346
:10FFE00012828AF31288A7682368D90303D50123F4
:10FFF000CCF80030A7682B68DCF80010D2B282F38E
:020000040801F1
:1000000011883268194400FB02F3DB1BB3FBF2F3E7
:1000100000FB0131A2E7049B002B00F08580013B2F
:1000200004933ED14FF4FA794FF47A70D8F8043043
:10003000C3F30803002B54D1EFF31283002B50D1EC
:100040002968A26800BF2B689942F9D1376800FB84
:1000500007F39B1AB3FBF7F300FB01310127019172
:10006000D8F80430C3F30803F3B9EFF31283DBB914
:100070002B68A16800BF2A689342F9D1D6F800B076
:1000800000FB0BF2521AB2FBFBF200FB0323019AB6
:100090009B1AB3F57A7FE3D3B9F10109C6D1FA23EC
:1000A00003931E4B0CCB6BE6EFF3128E8AF3128890
:1000B000A1682368DB0344BFCCF80070A1682B68FB
:1000C000DCF800205FFA8EFE8EF31188D6F800E08F
:1000D0001A4400FB0EF35B1AB3FBFEF300FB023382
:1000E000D5E7EFF312828AF31288A7682368D90351
:1000F00003D50123CCF80030A7682B68DCF800108A
:10010000D2B282F311883268194400FB02F3DB1B80
:10011000B3FBF2F300FB0131A0E700BF2045002054
:100120005C4F0020584F0020029B013B0293B8D146
:100130004FF47A79DFF824E14846D8F80430C3F365
:100140000803002B6AD1EFF31283002B66D12968D4
:10015000A26800BF2B689942F9D1376800FB07F30A
:100160009B1AB3FBF7F300FB013101270191D8F88B
:100170000430C3F30803002B33D1EFF31283002BB9
:100180002FD12B68A16800BF2A689342F9D1D6F815
:1001900000B000FB0BF2521AB2FBFBF200FB032390
:1001A000019A9B1AB3F57A7FE1D3B9F10109C4D161
:1001B000059B013B05937FF4C1AD264B264ADA60CF
:1001C00009B0BDE8F08F002B3FF4A9AE19689B88F9
:1001D0001022A1E6002B3FF4F0AD19689B880022A5
:1001E000E9E5EFF3128C8AF31288A1682368DB0338
:1001F00044BFCEF80070A1682B68DEF800205FFADB
:100200008CFC8CF31188D6F800C01A4400FB0CF368
:100210005B1AB3FBFCF300FB0233C1E7EFF312827E
:100220008AF31288A7682368D90303D50123CEF87F
:100230000030A7682B68DEF80010D2B282F3118874
:100240003268194400FB02F3DB1BB3FBF2F300FB43
:1002500001318AE700ED00E00400FA055C7E002031
:100260002DE9F04FDFF830C1474A4849484E494D23
:100270008046102718F1FF38C0F08480DCF8043085
:10028000C3F30803002B5CD1EFF31283002B58D18A
:100290000B68946800BF08688342F9D1D6F80090D3
:1002A0004FF47A7000FB09FEAEEB040EBEFBF9FEC4
:1002B00000FB03EEDCF80430C3F308034FF47A7458
:1002C0000120FBB9EFF31283E3B90B68D2F808A061
:1002D00000BFD1F800904B45F7D1D6F800B004FB31
:1002E0000BF9A9EB0A09B9FBFBF904FB0393A3EB98
:1002F0000E03B3F57A7FBDD2DCF80430C3F30803F4
:10030000002BDFD0EFF3128A87F31288D2F808B0FF
:100310001368DB0344BF2860D2F808B00B68D5F837
:1003200000905FFA8AFA8AF31188D6F800A09944FF
:1003300004FB0AF3A3EB0B03B3FBFAF304FB09334F
:10034000D5E7EFF3128487F31288D2F80890136888
:10035000D80303D501232B60D2F808900B682868D6
:10036000E4B284F31188D6F800A04FF47A7400EB5D
:10037000030E04FB0AF3A3EB0903B3FBFAF304FB3C
:100380000E3E97E7BDE8F08F10E000E0EC1900208A
:10039000607E00205C7E002000ED00E0D24B2DE965
:1003A000F0431A68D14E5189B6F906308B4280F27B
:1003B0008A80CF4A4FF07E511160CE4DB6F900C011
:1003C000B5F86A0295F9502295F84CE295F84D720D
:1003D000ACEB000101F2F31840F2E6345242A045C2
:1003E00092B240F2AB804FF4FA71A1EB0E010CB265
:1003F000C14960450C8001DD64420C80B6F902C041
:10040000ACEB000404F2F31940F2E638C1456CD9B4
:100410004FF4FA74A4EB0E0424B260454C8001DD65
:1004200064424C80B6F90460341A04F2F31C40F2C2
:10043000E63EF44500F28F80002CB8BF6442BC4217
:10044000D8BF002700F3898012FB07F7AB4A8F80E3
:1004500086421668BCBF7F428F8016F4805658D003
:10046000B3F5FA6FA8BF4FF4FA63B3F57A7FB8BF5C
:100470004FF47A73A3F57A74A14DA24F85FB042340
:10048000E217C2EB63135A1C6FF0630E37F91220A8
:1004900037F913700EFB0343D21B03FB02F385FBFA
:1004A0000325DB17C3EB65133B449BB2CB8026B11E
:1004B000954A1268D20000F17081944B1B885B064C
:1004C0004ED4BDE8F083B3F5FA6F15DB127AC2F1B2
:1004D000640207EE902AF8EEE77A9FED8D7A844A5F
:1004E00067EE877AC2ED007A67E7002CB8BF6442F6
:1004F000A6458FDB002490E7107A5A1A02FB00F21F
:10050000C1F5FA6192FBF1F2C2F1640207EE902AA2
:10051000E1E7B5F86C229342C0F2BA80B3F5FA6F06
:10052000D4BFC2EB0303C2F5FA634FF47A7404FB41
:1005300003F3C2F5FA64B3FBF4F49DE70029B8BFF6
:1005400049428E45FFF651AF6B49002460450C804F
:100550003FF752AF52E74FF4FA74E71BBFB273E7AD
:100560006C4B6D4AB3F904306C48DFED6D6A00885E
:100570009FED727A82FB0342DB17C3EBA2031B1AC7
:100580001BB207EE903AF8EEE77A67EEA67A77EEBE
:10059000876ABDEEE66A16EE103A2033402B40F231
:1005A0008180DFED606ABDEEE77A17EE103A203306
:1005B000402B74D89FED627AF4EEC77AF1EE10FA10
:1005C00040F30F81DFED585A9FED586A01E0F0EEDD
:1005D000477AF4EEC67AF1EE10FA37EEE57AF6DCF9
:1005E000DFED537AB4EEE77AF1EE10FA40F1FC80D9
:1005F000DFED4D5A9FED4F6A01E0B0EE677AB4EE41
:10060000C67AF1EE10FA77EE257AF6D49FED4B7AA2
:10061000F4EEC77AF1EE10FA3CDC9FED477AF4EE87
:10062000C77AF1EE10FA44BF9FED417A77EE677A10
:1006300067EEA75A9FED435A9FED436A9FED437AB9
:10064000A5EE856A27EEA55AA5EE867AE5EE077A2D
:10065000B1F9023006EE103AB1F9003005EE903AE9
:10066000B8EEC66AF8EEE55A27EEC67A65EEA77AC6
:10067000A5EEA67AE6EE267ABDEEC77AFDEEE77A1B
:1006800017EE102A17EE903A0A804B80BDE8F083EF
:1006900033464EE79FED2A7A77EE677AC8E7DFEDBB
:1006A000217AD5E7F4EEC77AF1EE10FA40F3A28092
:1006B000DFED1D5A9FED1D6A01E0F0EE476AF4EE92
:1006C000C66AF1EE10FA36EEE57AF6DCDFED186A6E
:1006D000B4EEE67AF1EE10FA40F18980DFED125ABD
:1006E0009FED146A36E000BFE47F00206C1A002002
:1006F000647E002074450020241D0020504F0020FF
:100700001F85EB5130260020681A0020061B0020B0
:100710000AD7233C601A002067666666DC2C00203E
:1007200035FA8E3C00000000DB0FC940E4CB1641D7
:10073000DB0F49C0E4CB16C1DB0FC9BFDB0FC93FDC
:10074000DB0F494092E741B99730083C15A82ABE13
:10075000B0EE667AB4EEC67AF1EE10FA77EE256A5C
:10076000F6D41FED0A7AF4EEC76AF1EE10FA2CDD2A
:100770001FED0D7A77EE666A66EEA65A1FED0F5AE8
:100780001FED0F6A1FED0F7AA5EE856A26EEA55ABA
:10079000A5EE867AE5EE076A05E7184AD278002AC0
:1007A0007FF48BAEA3F57A731BB2154C1B0384FB4D
:1007B0000324C0F5FA62DB17C3EBA41312B202FBE9
:1007C00003F300EB2330C88077E69FED0E7AF4EE5A
:1007D000C76AF1EE10FA44BF9FED0B7A77EE666AB6
:1007E000CAE7B0EE677AFBE6F0EE477A0EE7F0EE86
:1007F000476AB6E7B0EE667A68E700BF081B0020DC
:10080000D34D6210DB0FC9BFDB0F49C02DE9F843A0
:10081000144E154835782DED048B90F87112002D8B
:1008200040F07682114C90F870223ABB104B1B8836
:10083000002B00F062820F4B5A888B1CD9B275BB1B
:10084000B4F84A20013A12B2002AA4F84A2000F370
:100850008A800023A4F84A30002D00F04A82064B1B
:10086000B8E000BFDE2C00207445002030260020B8
:10087000061B00209C1C0020241D0020022A00F0E2
:100880003F82032AD7D190F87222C2EB421302EBC7
:100890008302D20092B28B1CD9B2002DD0D0E34B90
:1008A000E34F1B783F68B2FBF7FC0CF101073FB246
:1008B000092BA4F8487000F0B18200294CD0DD4B20
:1008C000B4F85490B3F90080B4F84CE0B4F94A207D
:1008D000A4F85480A8EB09081EFB02FE01299EFB28
:1008E000F7FEC644A4F84CE036D0B3F90280B4F861
:1008F0005690B4F84EE0A4F85680A8EB09081EFB09
:1009000002FE02299EFBF7FEC644A4F84EE023D067
:10091000B3F90480B4F85890B4F850E0A4F85880C3
:10092000A8EB09081EFB02FE03299EFBF7FEC64446
:10093000A4F850E010D0B3F906E0B4F85A80B4F847
:100940005230A4F85AE0AEEB080E13FB02F393FB0F
:10095000F7F77744A4F852700FFA8CF2002AA4F843
:100960004A207FF776AF00293FF476AFB4F84C50B9
:10097000B4F854E0AF4BB4F9487015FB02F5012907
:1009800095FBF7F5AEEB05051D8023D0B4F84E506E
:10099000B4F856E015FB02F5022995FBF7F5AEEB2E
:1009A00005055D8016D0B4F85050B4F858E015FB3A
:1009B00002F5032995FBF7F5AEEB05059D8009D0FF
:1009C000B4F85210B4F85A5011FB02F292FBF7F24D
:1009D000AA1ADA80984ADFEDA06A1268934915785E
:1009E0000F78917807EE905AF8EEE77AB0EE007A39
:1009F00067EEA67AF4EEC77AF1EE10FA40F385813D
:100A0000DFED8E6A37EEC77AB0EE676AA7EE266A28
:100A1000F0EE466AB3F900509FED896ADFF830E2E4
:100A2000DFF830C207EE105AB8EEC77A27EE067A22
:100A3000F0EEC75ACEED005A8CED007A99B106EE71
:100A4000101AB8EEC65A9FED846A67EE074A25EE83
:100A5000065AB7EE006A36EE456A64EEA54AA4EE81
:100A6000856A27EE067A9FED776A557966EE866A83
:100A700026EE877AADB106EE905AF8EEE66A9FED63
:100A8000765A9FED766A66EEA56A66EE856AF4EEA2
:100A9000C66AF1EE10FA40F3A9819FED6B6A27EE6A
:100AA000067A0C2F00F090819FED6D8ADFED6D6A64
:100AB000664DB4EEC87AF1EE10FA98BFB0EE478AF0
:100AC000B4EEE68AB0EE007AF1EE10FAF4EEC77AF0
:100AD000B8BFB0EE668AF1EE10FA85ED008A05DD4A
:100AE00037EEC77ADFED556AE7EE267AB3F9028072
:100AF00007EE108ADFED526AB8EEC77A27EE267A43
:100B0000F0EEC75A8CED017ACEED015A99B106EE9E
:100B1000901A9FED516AF8EEE66A27EE075A66EEE4
:100B2000866AB7EE006A36EE666A25EE255AA5EEAD
:100B3000266A27EE067ADFED436A917967EEA67A98
:100B400067EE877AA9B107EE101A9FED436AF8EEB7
:100B5000C76A9FED427A66EE866A66EEA56AF4EE93
:100B6000C76AF1EE10FA40F34D819FED377A67EED8
:100B7000877A0C2F00F02081DFED396A9FED397AFA
:100B80009FED356AF4EEE67AF1EE10FA88BFF0EEEA
:100B9000667AF4EEC77AF1EE10FAB8BFF0EE477A53
:100BA000C5ED017A517807EE901AF8EEE77AB0EECB
:100BB000007A67EE867A517AF4EEC77AF1EE10FA8F
:100BC00005DD37EEC77ADFED1D6AE7EE267AB3F969
:100BD000043007EE103ADFED1A6AB8EEC77A27EE56
:100BE000267AB0EEC75A8CED027A8EED025A99B190
:100BF00006EE901ADFED185AB8EEE66A67EE076A5D
:100C000026EE256AF7EE005A75EEC65A66EE856A3C
:100C1000E6EE265A27EE257ADFED0A6AD37967EEEB
:100C2000A67A67EE877A002B3ED01DE0387F002041
:100C300030440020241D0020E47F0020D7A3684119
:100C40006F12033B000048430000C842A07E002012
:100C5000C87E0020B87E00200AD7233CA4707D3FC8
:100C600000C0F94400C0F9C407EE103A1FED066A4F
:100C7000F8EEC76A1FED077A66EE866A66EE856A49
:100C8000F4EEC76AF1EE10FA00F3AD80F5EEC06A3B
:100C9000F1EE10FA00F12C81B7EE006A76EE666A8A
:100CA00086EE267A67EE877A0C2F00F095805FED4E
:100CB000146A1FED147A90F87332F4EEE67AF1EECE
:100CC00010FA88BFF0EE667AF4EEC77AF1EE10FA09
:100CD000B8BFF0EE477AC5ED027A43B18F4A126889
:100CE000910004D58E4A1288520640F1A08000235C
:100CF0003370BDEC048BBDE8F883A4F84A30ABE553
:100D0000228B02F57A7292B2C5E5F0EE676A81E64F
:100D1000844A854BD2F8F4201B68844CD3ED0F7ABB
:100D200044F62067BA42A8BF3A46B2F57A7FB7EEDA
:100D3000007AB8BF4FF47A72F4EEC77A92B2F1EE4D
:100D400010FA22837FF76FADDFF810E2784FAEFB29
:100D500002E23F684FF0640E92099EFBF2F2142A01
:100D6000A8BF1422FF04E7694CBFB3F838E0B3F919
:100D700038E0704B04EB470C07F1010748BF4FEA1E
:100D80005E0EBA42E761D8BF0027B3F90630D8BF7C
:100D9000E76104EB4707ACF820303A8C9B1A1BB292
:100DA000002BB8BF5B427345634BD6BF4FF07E52FA
:100DB000C3ED007A1A6036E5BDEEE77A5F4917EEBB
:100DC000108AA1F80280D7E6FDEEC76A5B4D16EEE9
:100DD000908AA5F8008067E6BDEEE77A574B17EEDC
:100DE000102A9A8063E79FED567A5BE7F5EEC06ABA
:100DF000F1EE10FA7FD4F7EE005A75EEE66A85EE52
:100E0000A66A4CE6F5EEC06AF1EE10FA6DD4B7EEC4
:100E1000006A76EE666A86EE267AA8E6454BDFF82B
:100E20001CE11B68CEF80030AEF8062045E594F8CA
:100E30005C209A4262D007EE903AB8EEE79ADFED76
:100E4000417A9FED410A84F85C3029EE279A39EE09
:100E5000000AFDEEC07A17EE903A2033402B58D9A5
:100E6000DFED3A8A3A4BFDEEC97AC3ED008A17EE00
:100E7000903A2033402B49D8B0EE490A1DF070F962
:100E800095ED027A84ED180A60EE477A9FED316A9B
:100E9000DFED316AE8EE287A28EE000AF4EEC67A31
:100EA000A7EE280AF1EE10FA88BFF0EE467AF4EECB
:100EB000E67AF1EE10FAB4EEC60AB4BFB0EE667A86
:100EC000B0EE677AF1EE10FA8CBFF0EE467AF0EEF3
:100ED000407AF4EEE67AF1EE10FAB8BFF0EE667AF8
:100EE00085ED007AC5ED027A01E7B7EE007A3EE6BD
:100EF000B7EE007AD6E6B7EE006AD0E5144B94ED73
:100F0000180AD3ED008AB0EE677ABDE79FED0F0AAD
:100F1000B6E71DF025F9F0EE408AA3E7681A002035
:100F2000061B0020A0100020483900203026002099
:100F3000504F0020241D0020641600203C7F00201C
:100F40000000C84235FA8E3CDB0FC93F00000000AC
:100F50005410002000C0F94400C0F9C4D34D621001
:100F600008B513F071FE024B024ADA60FEE700BFDB
:100F700000ED00E00400FA05024A034B12781978EC
:100F8000F7F7ECBB4E1D00204F1D00202DE9F04F60
:100F9000824D2B78012B8FB0824600F09C82804CD2
:100FA00094F86420002A44D1072BDFF828B200F01F
:100FB000DC81DBF81030002B00F0038394F86D30F7
:100FC0008BBB784B93F8012242BB01232A7884F82B
:100FD0006D30072A00F06383734E306817F0AAFC67
:100FE0002B78072B00F0A282012B00F05C83306885
:100FF00012F04CF96D4B1B68002B40F04F8294F8B7
:101000007430002B40F05A822B78072B00F05C8262
:10101000012384F864300FB0BDE8F08F93F8F83105
:10102000013BDBB2D2E7013B84F86D300FB0BDE885
:10103000F08F072B00F0C783DFF89C91DFF894B1A5
:10104000D9F800305A0552D4594F3B681B0700F1BC
:10105000D782544EFFF7A2F93B6813F0140F06D065
:10106000544B1B8803F40273002B40F00682524B52
:101070001B78C3B1514AB6F86C32B2F906209A42D5
:1010800011DC96F8B332012B00F04983192B00F0E4
:1010900046830E2B07D0082B05D04949494B002227
:1010A000002088809A6096F83602A8B9464EDFF88C
:1010B0002C81FFF7ABFB96F82420531E082B00F27F
:1010C0003881DFE813F06501BB01BE0036014D0039
:1010D0001C00D1013601BD01364B1B889B07E5D0B2
:1010E00014F098FA364AD3881844D080DEE7DBF84B
:1010F0000830002BA8D0354958469847A4E7344B10
:101100001B78002B40F011833368317A4FF48072E2
:1011100003EB012100200CF075FD337A0133DBB2C3
:10112000022B337240F0868100200CF0ADFD0020D0
:101130000CF0AAFDFF200CF0A7FD00F01F00052811
:1011400000F0718514F08CFCF768002F00F0B88275
:101150000022336971680120B84796F82420ACE773
:101160004FF40071306814F02DFC012800F0238347
:10117000C0F01183022840F05D8114F099FC14F056
:101180006FFCF768002F00F09B8200221046336945
:101190007168B84796F824208FE700BF387F002099
:1011A000302600207445002048390020347E00207D
:1011B000601B0020061B00204C1600206C1A00202B
:1011C000241D0020A07E00205C7F002096260020A9
:1011D0007473002070740020504F0020EC19002020
:1011E0001021C54814F0EEFB002840F02181039047
:1011F00001217F2017F02CFE01280990039B40F06D
:1012000017811846022117F023FE002800F06B8496
:10121000012840F00D8116213A2017F019FE431CD9
:101220009B02F36314F044FC3868FCF747FE00218E
:101230000A2014F0E5FB002840F0A082032386F882
:10124000243010210AA814F0BDFB002840F0F280E1
:101250009DF832209DF831009DF834109DF835300E
:101260009DF83370120442EA00620A431B019DF8A4
:1012700036109DF82900DBB243EA111342EA072237
:1012800003F5FA63726333879DF82A209DF83030A6
:1012900042EA002001F00F011A0903F00F0386F85B
:1012A0003A1086F831209DF828109DF82B2086F8FA
:1012B00032309DF82C3086F8281086F82C209DF8C6
:1012C0002D109DF82E2086F82D309DF82F3086F8B1
:1012D0003030708586F82E1086F82F2014F0E8FB49
:1012E000B37E73B9854F3868FCF7E8FD4FF40071A1
:1012F000102014F085FB074614F0DAFB002F40F0B5
:10130000AE807F4A138823F040031B041B0C13801C
:10131000138823F038031B041B0C138013889BB223
:1013200043F04003138000210422316286F8242018
:101330000323DBB2022B40F24E81042A00F0158118
:10134000082A00F012816F4B1B78002B00F04F81B0
:10135000504619F03DFE2B78072B00F0B481002297
:10136000072B84F864207FF424AE03F08BF9DBF8BC
:1013700010300690002B00F024812B78072B7FF48F
:101380001DAE03F07FF9069B5F4FC01A388015E64B
:101390005A4F3868FCF792FD0021084614F030FBE4
:1013A000039014F085FB039B012B43D10023386885
:1013B00073760493FCF782FD40F2AB11082014F021
:1013C0001FFB0528049B00F06183012800F0628365
:1013D00014F06EFB737E002B00F03984022386F834
:1013E00024303868FCF76AFD737E022B14BF00239B
:1013F0004FF0804300213720039314F001FB039B3F
:101400002920194614F0FCFA039014F051FB039BB9
:1014100083B9727E022A00F04983B3763868FCF7FC
:101420004DFD0021092014F0EBFA00283FF4D8AE5E
:1014300014F03EFB96F82420531E7AE72F4FD0E796
:101440000827FF200CF020FCFF2800F09E81013FC0
:10145000F7D17369D8F80020FA339342EAD214F036
:10146000FFFA96F8242028E60827FF200CF00CFC51
:10147000FF286CD0013FF8D1EBE7244B1B7813F029
:10148000100300F02881224A224B5188B3F9000052
:1014900096F9B53200FB03135380E8E510F0B6FD72
:1014A0001D4B1B6893F904300BB10BF0C1FF11F019
:1014B0000DF994F87430002B3FF4A6AD13F052FDF3
:1014C0002B78072B7FF4A4AD03F0DCF8059A0E4BC4
:1014D000801AD8809CE5114B114C1968114A0A4FAB
:1014E00094F86430496A128839807A80002B7FF43E
:1014F000A3ADDFF834B05CE59C7F00207073002062
:10150000003800405C3900203C7F00202E1B00206A
:10151000241D0020D82B00202C4400200C43002048
:1015200030260020FC3900207074002003F0AAF857
:101530002B78079AB14F801A012B788000F0B48085
:10154000072B7FF454AD03F09DF805904FE5336A07
:101550000022012B327640F2A183F269013B013275
:1015600033620823F26186F82430DFF8E08214F059
:1015700041FE98F80130022B00F02981032B7FF403
:10158000E2AE41F2B81318F80330002B40F0F982B4
:1015900041F2A40318F80330002B40F0EE8241F230
:1015A000E80318F80330002B40F0E38241F22C13DB
:1015B00018F80330002B3FF4C6AE91480AF05EF9EC
:1015C000C1E6DBF804308F48984700283FF4D5AED9
:1015D00008F036FFD1E68C4B71691B685B1AC82B8B
:1015E0007FF6AEAE14F03CFA96F82420A5E6D9F8C2
:1015F000003019037FF5ACAE5046F5F75BFBA7E66C
:10160000824A938803F10E0189B21C293AD8804995
:1016100009884E0736D57F497F4EB1F904007F49CE
:1016200086FB00E60988C017C0EBA600401A80B20E
:1016300001B211F1B30FB8BF00F5B4717848794E1B
:101640000078B8BF09B2B329C4BFA1F5B47109B21B
:1016500000077FF5FFAC744896F950E20068CEF1C0
:10166000000E1EFB01F190F808E0704889B21EFBE5
:1016700001F180FB01E00844C917A1EB20110B44E4
:101680009380E7E4634B6449B3F90430634A654EE1
:1016900081FB0301DB17C3EBA1031380DAE402F043
:1016A000F1FF079098E4554F02F0ECFF604A236F7A
:1016B00012680590C31A9A1A2067BB80FA8096E4D4
:1016C00096F82420F9E402F0DDFF089A4B4F2B78BE
:1016D000801AB88043E6A06EC178002900F020820D
:1016E0005449554AB1F90670B2F9001080787A1A57
:1016F000002AB8BF5242824240F34782DFF850E1ED
:10170000424ACEF800308F42D388C8BF404280B2F0
:101710004FF0010E184484F86CE0D080A7E496F8EE
:10172000FC30002B3FF4B9ACBDE4444B19688F0387
:101730007FF506AE4FF400325A60414B1A68414BB8
:101740004FF6FE710A403E490A601A89D20710D44A
:101750000CF002FE0028FBD13A4A938823F00203E2
:101760001B041B0C9380384B1B78002B7FF4DCACE4
:10177000CAE49A891A89D007FBD4E9E714F098F9EA
:1017800014F06EF996F8242097E414F091F90423EC
:1017900086F82430E9E614F08BF9F768042300207A
:1017A00086F824303076002F3FF4DFAE336932689C
:1017B0007168B8473EE67369D8F8002064339342F5
:1017C000FFF4DBAC36E602F05DFF089034E498F8F5
:1017D000023001272646072B00F2EE82DFE813F0E5
:1017E00013012D010601FA008D0073007F0008002F
:1017F0000323344688F80130A5E500BF3C7F002074
:10180000A460002070740020EC190020241D00202A
:10181000061B0020601A002067666666DA2C00202E
:101820002E1B0020744500204839002089888888B4
:10183000304400206C1A0020E02C00200000024000
:10184000580002400038004074730020784F002098
:10185000D42B0020D8F810300622652B564688F885
:101860000220DDF80CA03AD998F80020032A14BF12
:101870006FF0FF026FF07F02A3F1650303EA02033A
:1018800003F1010314BF4FF4807280229A42C8F81A
:10189000103024D22268D8F80C4002321819904235
:1018A00080F06F82C64AC8F80440D16FC8F80800BB
:1018B000490203FB01F30521146042F81C3C42F885
:1018C000183C88F80210D8F80820BE49012019F009
:1018D000A3F9012840F05C82062388F80230002139
:1018E000B94818F027FD012840F0528298F80230DC
:1018F0000133DBB288F802306DE798F8002098F8E1
:101900001430B24CCDF80CA0032A14BF4FF48072EF
:1019100080220492B246002B47D0012BFBD1AC4B66
:10192000D8F804C01B6826685B024FF0FF3E002118
:10193000BEFBF3FE1EEB0C0041F1000100239942B7
:1019400006F1020608BFB04238BF0CEB0E06324665
:10195000A049022014F0FAF9032800F27C81DFE8A4
:1019600000F0020602065446DDF80CA0EBE4D8F8BD
:101970000460D8F80830D8F81020991B914284BF31
:10198000C8F80C60C8F8101003283FF463AF04983F
:101990000133B3FBF0F200FB12320AB103449B1A8D
:1019A0000022C8F8043088F81420226885490232E1
:1019B000002014F0CBF9032800F24D8101A353F865
:1019C00020F000BF671901087D1A01086719010896
:1019D0005518010841F27013344618F80330002BF3
:1019E0003FF4B1AC784809F049FFACE47A4B00937E
:1019F000032088F8020030230522784972483446D3
:101A000019F078F89FE4002334460AAE31461846B0
:101A1000092214F05BF801287FF495AC0A9B93F837
:101A2000FE21552A00F01A8141F2B412022101234D
:101A300008F8021088F8013085E434460AAE41F215
:101A4000FC17314658F807000023092214F03EF82D
:101A500001287FF478AC00220A9B88F80020B3F8B4
:101A60000B20B2F5007F00F0208141F2B412032177
:101A7000012308F8021088F8013064E4D8F8043033
:101A800088F814700133C8F8083048E79DF80C3026
:101A900073769DE4194604220AA80CF0B3F89DF869
:101AA0002B30AB2B04BF0223737691E43868039389
:101AB000FCF704FA039B049319463A2013F0A0FFA5
:101AC000049B0390194604220AA80CF09BF8039B80
:101AD000002B7FF453AE13F0EBFF0A9B1BBAC3F34A
:101AE0008073B3769AE404212C2017F0B1F9032116
:101AF00004904E2017F0ACF90C210390362017F01B
:101B0000A7F9039A049B911C421C09988A409840AB
:101B1000A2FB0023520A42EAC352F263FFF782BBE0
:101B20002F4B304AB3F90030B2F906208078D21A30
:101B300082EAE277A7EBE277874267DD02EBD272B7
:101B400029482A495210026001220A7084F86C2048
:101B50002749284A09680B44B3F5FA6FA8BF4FF428
:101B6000FA63B3F57A7FB8BF4FF47A73D380FFF787
:101B70007EBA214809F082FE18E5204809F07EFE71
:101B80000DE51F4809F07AFE02E594F86C202AB1B1
:101B90001C481D4A006884F86C301060144A154BCC
:101BA00012681144B1F5FA6FA8BF4FF4FA61B1F5AC
:101BB0007A7FB8BF4FF47A71D980FFF758BA00BF67
:101BC0000C6100207C4F0020E86000208061002034
:101BD00088610020804F002081A00208A88A0308A5
:101BE000E02C00206C1A0020CC2B0020DC2B0020E5
:101BF000D82B0020241D0020606000201C600020E5
:101C000030610020A81C0020C42B002094F86C2018
